:109C6A00414952434F544543004256332E33342020
:109C7A0052555300414B4B4D00532F4E21464149FB
:109C8A004C555245005245454E54455221532F4E8C
:109C9A0000434F4E5441435420414952434F544587
:109CAA004300475053004032444000403344400090
:109CBA0042794B21484F42404D45486D000A1600F3
:109CCA000180000300007E0000FE00001E00003636
:109CDA000003E60001C4000000000FFFE0714F66B8
:109CEA00434B404371595420004B6C3650404279E3
:109CFA0043202300504943545552450052414E4B8C
:109D0A00494E4700424150664F20202000364150BC
:109D1A004F6B50414D004D415073505954790036A4
:109D2A006C4E7A4820202000544F744B4E2020203D
:109D3A00004D45544B4E202020004279584F642054
:109D4A002020004D41524B532020200044454641DB
:109D5A00554C5400202020214350642120202020EB
:109D6A006443540020545241434B214F4E2020005B
:109D7A0020545241434B214F464620004D41524BFD
:109D8A000020545241434B2D5550212000204E4F64
:109D9A005254482D5550212000214279584F6401D0
:109DAA00427936404D41507350015943542042790B
:109DBA00434F547901714F6C4554792020686901E9
:109DCA00714F6C4554792042434501544F744B4EB0
:109DDA002020206869014D415073505954796869AF
:109DEA00014149525350414345686901484143542E
:109DFA00504F664B686900594354204279434F5487
:109E0A007900364150404279434F5441200047502F
:109E1A0053204279434F544100514E48202020207C
:109E2A00402148504100464C007A595048416C2024
:109E3A00207159435420003E214558495400214578
:109E4A00584954015245504C41590153454E440119
:109E5A0044454C45544500214279584F6401434FCB
:109E6A004D3A20202020202001544E432031232027
:109E7A0035374B01544E4320312320392E36010108
:109E8A00505743403130234035374B0150574340F8
:109E9A003130234031394B01014D58504031302384
:109EAA004035374B014D58502034232035374B016C
:109EBA004D58502031232035374B014D58504031F1
:109ECA0030234031394B014D58502031232031394C
:109EDA004B00214279584F6401484F422020547464
:109EEA004B014E334D2020544F744B590159644154
:109EFA006C20544F744B590101434F4D3A01714F35
:109F0A006C5974202054744B014F547150202020F6
:109F1A0054744B014F5471404243454054744B01B1
:109F2A0001644E43542054742D54740159646C4096
:109F3A004243454054744B004252472021444953FE
:109F4A005400434F5850200050524553454E542018
:109F5A00504F532E004150584E42202020200020BE
:109F6A0053544F52452157505420002046554C4CCB
:109F7A0020002040434F58502020005345522000D3
:109F8A004952444100555342200055534220004350
:109F9A00714E43004F547150004F734E364B41205F
:109FAA00714550456441744E00214279584F64010D
:109FBA00427936404D4150735001484F42204D502E
:109FCA007354744B014E334D204D41507350200150
:0D9FDA005045425043204D415073015964E1
:109FE7006C204D507354744B015964416C204D41A2
:109FF7005073500143594C20524144495553014332
:10A007004F4D3A01714F6C5974204D415073014FB8
:10A01700547150204D4150735001434845434B20E4
:10A027004D410053454C20524F5554450048404F31
:10A0370040420020484F4240504F534021002140AA
:10A04700504542455043204000504542455043004B
:10A05700214044454C4057505453002144454C201F
:10A0670052544500484520715943544F66200021FA
:10A07700404F547150404D50730020205241444985
:10A08700555300214279584F64014C4F4144404396
:10A0970054522150430156494557404354520144B5
:10A0A700454C40414C4C214354520101434F4D3ADA
:10A0B700015245435620204354520153454E4420F4
:10A0C70020435452005649455720435452002020FC
:10A0D7004D4F56450020204D4F564520544F0053B5
:10A0E70043414C452020582F5920204558495400BA
:10A0F700434C522044495354004155544F43454E15
:10A1070054004155544F204F4646002020205343CA
:10A11700414C450044495354204B4D004449535446
:10A12700204E4D00214279584F64014241504E4F15
:10A1370020202068690158432D48414354506869DD
:10A14700015254452D534554206869014F36764EC8
:10A1570045202020686901504943545552455368AA
:10A1670069010101454153592D534554013341427A
:10A177004F644841435450015445435420714F6C38
:10A1870045540144454C21414C4C21464C49002142
:10A197004279584F640153494E4B544F4E45014342
:10A1A700484E7A212D0143484E7A4050457A014363
:10A1B700484E7A404F365001564152205443402072
:10A1C70020402301564F4C554D4501564152494FAA
:10A1D700204E554C4C015049544348015045524973
:10A1E7004F440156415220415640203040230154EC
:10A1F7004543202020403030402501534F554E44E1
:10A20700434845434B0053494E4B21544F4E45005D
:10A2170053494E4B54214F46460048452064424F10
:10A2270066484F66004F3648596C2042415020001F
:10A23700434F5850403130404D4E4859542020200C
:10A24700004245564F52204E554C4C494E47200030
:10A25700214279584F64015450454B20202020015A
:10A267004142544F6E45485401014350642F644E98
:10A277004354016B6C416664014C2F4401015749FB
:10A287004E4421542D55500143454E5421542D55CC
:10A2970050015741595054214252470021427958A1
:10A2A7004F640153544152544054494D4501464966
:10A2B7005253540144454C544120203A014D554CCA
:10A2C7005449504C45014C4153540143594C53494F
:10A2D7004740202040230153454C40524F55544599
:10A2E7000101010143594C520143594C20542D554A
:10A2F7005000214279584F64010145644E48017668
:10A30700456C744B40302C402023014B4F48545030
:10A31700414354014E4D45412131383301494D5098
:10A327002F414750530101432D564152494F014D8B
:10A33700454D4F525944554D50004D454D4F52597B
:10A3470044554D50004054744B204359764543546F
:0DA3570042594554204000544F744B4120A2
:10A3640020200020204558495420202100524543F4
:10A3740045495645004652454540003C2D204C4930
:10A384005354202D3E2020455849540053454C0039
:10A394004E455854004E4558542054505400505281
:10A3A40045562054505400434C5220404C454700DD
:10A3B400434C52204053554D0042794B20202020DD
:10A3C40020202020002042794B00475053204F7317
:10A3D4004E362000204150584E4220004D415057E7
:10A3E40050004E4145525354004C495354200045AB
:10A3F400544500414C5440300071594354204D4160
:10A404005073500020544F4F404D55434820002175
:10A41400404279364043714E43002053454C4057E7
:10A42400505440210021524543454956454000209F
:10A434002040584F504020202100584F5000564192
:10A44400520046495800474154452158006C4E4833
:10A454002043545054202000535443594C2000406E
:10A4640042794B0054502000406A40494E2000403D
:10A4740067404F555400204F734E364B4120210006
:10A484002045584954004E334D200059404540530F
:10A49400004E334D2020484F422020204150584E3A
:10A4A40042004E4558542053454C4543542045588A
:10A4B4004954005843542D464C49474854200055AC
:10A4C40053454400454E54455220004D4D2E4D4DAC
:10A4D4004D20004D4D2753532E53005747532138D9
:10A4E40034002040554054404D40200055405440D5
:10A4F4004D002055544320004C4F43414C005357CA
:10A50400495353474400414C540053554940580063
:10A514004156474020304023003530300031363436
:10A524003000205D203130404B632F70005D2020CF
:10A53400203140632F2300205D202035404B5453AD
:10A54400005D203230304046504D00406340204B87
:10A5540063004654204B6300406340204E4D004648
:10A5640054204E4D004D2F53003230305E003530B4
:10A57400305E0031220032220033220035220038BE
:10A584002200464C3700464C313600464C333300EB
:10A59400464C3635004631303000463136300046C0
:10A5A400323630005E252640534F47005E25264054
:10A5B40054415300414C540056415200225E2F2412
:10A5C400004B545300532F4E002224004B540022BE
:10A5D4005E004E4D00302C3500312C3000322C30D2
:10A5E40000302C3600312C3200322C3500332C381C
:10A5F40000372C35004031350040333000403630D0
:10A60400005441534B00464C2D4441544500545092
:10A6140000544F46005354410046494E004C414EAD
:10A6240000534554204F4646534554004953412056
:10A63400484549474854004155544F2D474F200041
:10A6440053544152540020434845434B40414C4CE1
:10A65400005241442044495354004053454C40481F
:10A6640045494748543A00475053404241524F40AD
:10A67400414C4C0053494E4B40312D3221632F2322
:01A6840000D5
:1064F400304D2475A7049005C2E0F51CE0F51DE0BD
:10650400F51EE0F51FE0F56DE0F56EE0F56FE0F5E2
:10651400541270B6126AF42275C70375C6E475B9CD
:1065240001E5BCB481431270B61256DC8E628F63EF
:106534007568F97569001265CA203C2D203B2B1241
:1065440066FF1266D3856D1C856E1D856F1E85548E
:106554001F126636203C12203243201D231266FF90
:10656400126AF4E532242850DC22126636203CF903
:10657400203DF6203205201DBD80EF301DB880EA95
:106584001266FF126AF4856D1C856E1D856F1E856B
:10659400541F1266E9126AF4203DCE8099126922D2
:1065A400201D0D7553107400126885203DBB808634
:1065B400E553540FC553C4540F20350512679A8010
:1065C40003126885808BC23CD23B126686FD12663C
:1065D40086FC126686C39573F565EC9574F564EDD7
:1065E4009575600504600A800EE56424E05011800E
:1065F40006E56424204009126686126686026686D1
:10660400126686FD126686FC126686C39576F56769
:10661400EC9577F566ED9578600904600122E566EE
:10662400F48002E5668562F0A474E025F04002C2BD
:0D6634003B22C23C126686A2E7923DA2E620
:10664100921DA2E592324026A2E492E592E692E7FB
:10665100FC1266862565F565EC3564F5641266867F
:10666100FC1266862567F567EC3566F56622A2E4BD
:106671009235540F79C6F712668609F7301D051257
:106681006686F55322E5697023E56860302404408D
:106691002CE56875F004A485F0C7F5C675B901E568
:1066A100BCB4811985BD68756902801E54037010E0
:1066B10005C675B901E5BC056953690F22D23C22B3
:1066C100147004E5BD80F0147004E5BE80E9E5BFF7
:1066D10080E575A7009006F6E56DF0A3E56EF0A3E1
:1066E100E56FF0A3E554F02275A7009006F6E0F5FA
:1066F1006DA3E0F56EA3E0F56FA3E0F55422E56428
:10670100B2E7F56D85656EAB67E566FC30E707C3FB
:10671100E49BFBE49CFCAA62A9631253DCE56630AE
:10672100E707C3E49DFDE49EFEEEB2E7F56F8D54ED
:106731002275380C12698B1269D6D553012275382E
:106741000C12695C1269CCD55301227538001269AB
:0E6751007412699BD553012275380012695CE1
:10675F0012699BD553012275380312698B126A0790
:10676F00D553012275380312695C1269FDD55301A7
:10677F002275380F126974126A2CD553012275389D
:10678F000F12695C126A2CD553262290679F2373D0
:10679F008091807780688059804A803B802C801D53
:1067AF00800E80DA80CB80BC80AD809E808F808011
:1067BF0075381512698B126A4ED55301227538152B
:1067CF0012695C126A43D553012275380912697434
:1067DF00126A14D553012275380912695C126A14B2
:1067EF00D553012275380612698B1269BED5530134
:1067FF002275380612695C1269B3D55301227538B8
:10680F00121269741269E4D5530122753812126994
:10681F005C1269E4D553012202673275381512698B
:10682F008B126A4ED553012275380F12695C126AAA
:10683F002CD553012275380F126974126A2CD55357
:10684F00012275380312695C1269FDD55301227557
:10685F00380312698B126A07D5530122753800125B
:10686F00695C12699BD55301227538001269741245
:10687F00699BD553262290688A2373809E80A980B6
:10688F00B480BF80CA80D580E08010801B802680B6
:10689F0031803C80478052805D806875380C12696A
:1068AF005C1269CCD553012275380C12698B1269B1
:0E68BF00D6D553012275381212695C1269E4B5
:1068CD00D55301227538121269741269E4D553013A
:1068DD002275380612695C1269B3D55301227538D9
:1068ED000612698B1269BED55301227538091269DA
:1068FD005C126A14D5530122753809126974126A33
:10690D0014D553012275381512695C126A43D5539B
:10691D00012202682A78C686040886037AED12538E
:10692D009A78CAA60408A60378C686040886037A50
:10693D006212539A78CCA60408A60378C68604087A
:10694D0086037AB512539A78C8A60408A603227551
:10695D001A6A751B0A78CA8618088619126B9F78F1
:10696D00CC86060886072278C88618088619E4F5AD
:10697D001AF51B126B9F78C886060886072278C603
:10698D008618088619751A00751B01026B9FE51D87
:10699D002519F51DE51C3518F51CC3E51F9FF51FC1
:1069AD00E51E9EF51E22C3E51F9FF51FE51E9EF5F4
:1069BD001EC3E51D9519F51DE51C9518F51C22E561
:1069CD001D2FF51DE51C3EF51CC3E51F9519F51F83
:1069DD00E51E9518F51E22C3E51D9FF51DE51C9EB0
:0969ED00F51CC3E51F9519F51F07
:1069F600E51E9518F51E22E51F2FF51FE51E3EF52F
:106A06001EE51D2519F51DE51C3518F51C22C3E5E7
:106A16001D9519F51DE51C9518F51CE51F2FF51F8D
:106A2600E51E3EF51E22E51D2FF51DE51C3EF51C57
:106A3600E51F2519F51FE51E3518F51E22C3E51DB0
:106A46009FF51DE51C9EF51CE51F2519F51FE51E86
:106A56003518F51E22E51A7009E51B70058C068DA2
:106A66000722ED851BF0A4A2F792D5ED851AF0A4B6
:106A7600AEF0FFEC851BF0A4A2D53FEE35F0FF92F9
:106A8600D5EC851AF0A42FFFE435F030D50104FECD
:106A960022E4F51AF51BEF4E7003051B22EF65196C
:106AA6007006EE65187001227808C3EF33FFEE33E7
:106AB600FEEF9519F5F0EE95184003FEAFF0E51AD6
:106AC60033F51AD8E5F4F51A751BFF7805C3EF33CD
:106AD600FFEE33FEEF9519F5F0EE95184003FEAF85
:036AE600F0E51BBD
:106AE90033F51BD8E5F4C403F51B22E51D9511E523
:106AF9001C9510500BE56E9511E56D95105001220E
:106B0900E51F9511E51E9510500BE5549511E56F9C
:106B19009510500122E51D9513E51C9512400BE5D2
:106B29006E9513E56D9512400122E51F9513E51E3B
:106B39009512400BE5549513E56F951240012253C8
:106B49002CF8C3E51F9554FFE51E956FFE92605022
:106B590007C3E49FFFE49EFEC3E56E951DF519E5A5
:106B69006D951CF5189261500BC3E49519F519E45C
:106B79009518F518C3E5199FE5189E9262500AE524
:106B890018CEF518E519CFF519126A97E52C5407AF
:106B990075F003A4F538E538906BA573026BBD0257
:106BA9006BD1026BDF026BF7026C0A026C1D026C7F
:106BB9002B026C43851C16851D17C3E4951FF5151B
:106BC900E4951EF514026C56851C16851D17851E45
:106BD90014851F158077C3E4951DF517E4951CF5F9
:106BE90016C3E4951FF515E4951EF514805FC3E4FB
:056BF900951DF517E4F5
:106BFE00951CF516851E14851F15804CC3E4951F34
:106C0E00F517E4951EF516851C14851D158039851E
:106C1E001E16851F17851C14851D15802BC3E49524
:106C2E001FF517E4951EF516C3E4951DF515E495AD
:106C3E001CF5148013851E16851F17C3E4951DF5CC
:106C4E0015E4951CF5148000C3E5179513E516950C
:106C5E001210D70122E5159513E514951210D701E0
:106C6E0022E519F92517FFE518F83516FED3EF952D
:106C7E0011EE9510500122E5119517FDE5109516B0
:106C8E00FC402A4D6027126A5BE5152FF515E514B9
:106C9E003EF514E5159513E514951210D70122E56E
:106CAE00199DF9E5189CF8851016851117E5172919
:106CBE00FFE51638FEE5139FE5129E500BC3E51354
:106CCE009517F9E5129516F8E51A700AE51B700688
:106CDE00AA00AB018013E9851AF0A4E5F0FBE88564
:106CEE001AF0A42BFBE435F0FAE5152BFBE5143A6C
:066CFE00FAE5119BE51010
:106D04009A10D70122EB9515FDEA9514FCC3E515FD
:106D14009511E514951010D717E5139BE5129A50B9
:106D240036E5139515FFE5129514FE126FD38027EF
:106D3400EB9511FFEA9510FEAA00C001126FD3D0A3
:106D440003E5172BFBE5163AFAEB99F517EA98F5E4
:106D540016851115851014C2D5E5466002D2D5AA50
:106D640056E98AF0A4ABF0E88AF0A42B30D5047578
:106D7400F00384F8700122E5172513FDE51635129A
:106D8400FCED8AF0A4ABF0EC8AF0A42B30D50475AA
:106D9400F00384FEE5152513FDE5143512FCED8A98
:106DA400F0A4ABF0EC8AF0A42B30D50475F0038486
:106DB400F9E538906DBB73026DD3026DDF026DE8A7
:106DC400026DF1026DF7026E03026E0A026E0FC3CA
:106DD400743E9EFFC3743E99FE8032C3743E9EFF90
:106DE400AE018029AF06C3743E99FE8020AF06AE83
:0D6DF40001801AC3743E9EFEC3743E99FFD9
:106E0100800EC3743E99FF8007C3743E9EFEAF019E
:106E110008EF2437FFE51B7007E51A700CE8800EB8
:106E2100A2E7E51A50030460F488F0A4E5F06001DC
:106E310004F923FA98FBC3E998C333F9906E43E54B
:106E41003873026E5B026E88026EBD026EEA026FDB
:106E510017026F44026F71026F9E05A7800BEB3022
:106E6100E7032A8002291E1FFBEEC45403F583EEBB
:106E71005408C42FF582EE5407243883F5F0E04519
:106E8100F0F0D8DA05A72205A7800BEB30E7032A3B
:106E91008002290E1FFBEEC45403F583EE5408C48F
:106EA1002FF582EE5407240B83F5F0E045F0F0D87E
:106EB100DA05A722804020100804020105A7800BF3
:106EC100EB30E7032A8002291E0FFBEEC45403F5C1
:106ED10083EE5408C42FF582EE540724EC83F5F0B9
:106EE100E045F0F0D8DA05A72205A7800BEB30E7E3
:056EF100032A800229C4
:106EF6000E0FFBEEC45403F583EE5408C42FF5823F
:106F0600EE540724BF83F5F0E045F0F0D8DA05A784
:106F16002205A7800BEB30E7032A8002291F1EFB00
:106F2600EEC45403F583EE5408C42FF582EE5407DD
:106F3600249283F5F0E045F0F0D8DA05A72205A7FC
:106F4600800BEB30E7032A8002291F0EFBEEC454A8
:106F560003F583EE5408C42FF582EE5407246583A7
:106F6600F5F0E045F0F0D8DA05A72205A7800BEB8F
:106F760030E7032A8002290F1EFBEEC45403F58373
:106F8600EE5408C42FF582EE5407243883F5F0E05A
:106F960045F0F0D8DA05A72205A7800BEB30E7030A
:106FA6002A8002290F0EFBEEC45403F583EE540823
:106FB600C42FF582EE5407240B83F5F0E045F0F07C
:106FC600D8DA05A7228040201008040201EC701FC1
:086FD600ED20E740D2E023CFDB
:106FDE0023CF30E7F980357B08801A7B1080167B33
:106FEE002080127B40800E20E4ED20E3EE20E2EFC5
:106FFE0020E1F07B80EE8BF0A4CF8BF0A4E5F02F98
:10700E00FFEC8BF0A4CD8BF0A4E5F02D2499838FAB
:10701E00F0A433E5F033FBE98BF0A4E5F0C88BF078
:10702E00A428F9E435F0F822FFFEFCFAF8F6F4F2A3
:10703E00F0EFEDEBEAE8E6E5E3E1E0DEDDDBDAD901
:10704E00D7D6D4D3D2D0CFCECCCBCAC9C7C6C5C45F
:10705E00C3C1C0BFBEBDBCBBBAB9B8B7B6B5B4B379
:10706E00B2B1B0AFAEADACABAAA9A8A8A7A6A5A465
:10707E00A3A3A2A1A09F9F9E9D9C9C9B9A99999829
:10708E009797969594949392929190908F8F8E8DD0
:10709E008D8C8C8B8A8A898988878786868585845C
:1070AE00848383828281818075A7009070DCE5469F
:1070BE00FA24FA50027A05EA2323F978107F049312
:1070CE00F60809E9DFF99070F4EA93F556227FC2CB
:1070DE00803E7F4680BA7E8C81747D1882E87A303D
:1070EE0085D074608BA08080402010081271000241
:1070FE007356D215D274D273C219C23A1256DC8E9E
:10710E0047757D0075460575520212914612022191
:10711E00E53524EB500E1291467F1990A0F71276AA
:10712E00F012DD1BE55275F016A4F57012730C7596
:10713E007E151271D77F237E0990A0D51277021289
:10714E00DD1B10000810010D10021280E212727F7A
:10715E0075330180DA1272C475330180D2757E00E8
:10716E001271D77E0090A0E61277357F237E0590B0
:10717E00A0DC12770212722812DD1BE55210000FEE
:10718E0010010510028780D5045403F55280CE12EB
:10719E0071D77F237E0B90A114127702E54660070C
:1071AE001460041412411A12DD1BE546100008107B
:1071BE00010B10021180D860D6154680D2B405029C
:1071CE0080CD054680C902711B75320012DEF17F3B
:1071DE00017E1190A0CC1277357E0012D5B2E57EDD
:1071EE00D26612D60975170812DA3C12415975711A
:1071FE0000C20612D759741BFFF5177E0F90A11B04
:10720E00305D0390A123127735129189125D0D1214
:10721E0046BFC20612651C021E03E55260141460BE
:10722E001E1460297F647E2D791C1272721E1FD966
:10723E00F9227F6A7E1F79281272721FD9FA227F75
:10724E00487E2D791C1272720F1ED9F9227F567E3E
:10725E003379281F12DE360F0F12DE361F12DE367E
:10726E001ED9F0221E12DE360E0E12DE361E02DE83
:10727E0036E552605514606814606D800075709E1E
:10728E001272F98003757000E5732540F573E435CD
:10729E0074F574E43575F575227570161272968054
:1072AE000375702DE5762542F576E5773541F57750
:1072BE00E43578F57822E55260CB1460DC1460E199
:1072CE0080007570441272B2800375705AE5739522
:0972DE0040F573E5749400F574A9
:1072E700E5759400F575227570711272DB80037570
:1072F7007088E5769542F576E5779541F577E578F7
:107307009400F57822E54690732293F540FEAD4749
:10731700E4FFFC12546F8E418F4222020C1830603A
:10732700C07F40120E9E121E1912DD1B1275D1EB83
:107337007005909E3A800B1273DF90A43350039030
:10734700A47A7F3F7E0412770212DD1B12DDFC1246
:10735700DE2C75370990A08A121CFF9073667302A2
:1073670002930275260270FA0276020273560273BE
:107377007E0273970273287F2E12168680D17F367E
:107387007E0490A40812770212DD1B12DDFC80BF79
:107397007F37120E9E121E1912DD1B1275B5124889
:1073A7004FD2AC1000A9306DFA12748F203BCF403A
:1073B700ED7568F97516001274DC40FB1276787F5C
:1073C700367E29E51612D39212DD1B05161277A811
:1073D70078C6B6F7E20275AF7C0512484F12DC3566
:1073E700744112DC46745312DC03EB12DC2412776F
:1073F700BA5003DCE5227515F975160010000EE585
:1074070015602512743140051274585002D3227F3B
:107417003F7E29E51612D39212DD1B7F1412DE136D
:107427000516E51664F870D4C322127D7075B9018C
:10743700E5BCB4811AE5BDF51570037516F778C676
:0B744700A616127EB9127EB1127EB1B3
:10745200C3027EB1D3227F0575F019D5E0FDD5F0C8
:10746200FA12484F12DC35744112DC46744212DCC7
:10747200037E0F78C6E60812DC03DEF912DC27125F
:1074820077BA400122DF012275F00080CEC23B12A2
:10749200484FD2AC12DB8E204C3CB440F712DB9347
:1074A200B4400312DB93B4412DF53812DB93B4538D
:1074B2002512DB93FA12DB93E538701A12DB93B4D0
:1074C2000D1412DB93B40A0EC3E5169A4003027739
:1074D2009FC2ACD23B22C2ACD3221277FE12484FDB
:1074E200D2AC1000F112DB8E204CEBB440F412DB74
:1074F20093B4400312DB93B441DCF53812DB93B44E
:1075020042D47E1078C612DB93F608DEF9E53870B5
:10751200C512DB93B40DBF12DB93B40AB9C2ACC37C
:10752200220273567F0A120E9E121E1912DD1B12C0
:1075320075B5124868D2AC1000E712DB93B440F57F
:10754200F53812DB93B46EED12DB93E538600A1264
:107552004868744F12DC0F80DC124868744012DCF9
:1075620046E51612DC0F12DC197568F97516001261
:107572004868D2AC10003912DB93B440F7F53812E8
:10758200DB93B44EC07E1078C612DB93F608DEF9A8
:10759200124868E5386007744F12DC0F80D112760A
:1075A200780516745112DC0F78C6B6F7C21276153A
:0C75B200027356751500751603127D67F4
:1075BE0075B901E5BC30E70205160515E515242061
:1075CE0050EB227B007515F9127D7075B901E5BC83
:1075DE00B481010B0515E515240450EC7515011247
:1075EE007D6775B901E5BCB481010B0515E5152460
:1075FE002050EC227F1C120E9E121E5C400675154A
:10760E00F9127615027356E51560372404401A24D4
:10761E001E5019E515240740028027127D70127640
:10762E00510515E515240450F2751501127D677587
:10763E00B901E5BC30E7031276510515E515242096
:10764E0050EA22127666124EE605C6124EE605C6C0
:10765E00124EE605C6024EE674FF800574048001E4
:10766E00E4F5BCF5BDF5BEF5BF22E568606AF5151B
:10767E000515E5152404501D751501127D6775B9A4
:10768E0001E5BC30E70280190515E515242050EB05
:10769E00751500800C241C60F750E0E5152406508B
:1076AE0037E56875F004A485F0C7F5C675BC81E5AD
:1076BE0015F5BDF56878C6B6F70375BD00081276E8
:1076CE00DB1276D51276D586BC0886BD0886BE0836
:0976DE0086BF08124EE605C62223
:10C0640012AEA012C16312828112C0E81282891238
:10C07400C0F502AEA412AEA012C1631282817F5A2F
:10C08400C23C12816312835F783F79437F607EEA0A
:10C0940012C1571282897F6512816312835F783DD2
:10C0A40079417F207E4E12C157303C2012C31912B1
:10C0B400C174783F794312C0D3783D794112C0D31B
:10C0C40012C31978D7E65480F675370002935BC320
:10C0D400E796FF1819E796FE0809C3E69FF71819B3
:10C0E400E69EF7227F5B7E0690A50E1277351F80B1
:10C0F4000A7F667E14745912D4AB1F127FEC7E390A
:10C10400E402D4CA7866E620E73418C3E6947208D9
:10C11400E694045029C318E6941F08E69404401ECC
:10C124007869E620E71818C3E6940E08E6940150EF
:10C134000DC318E6947508E694004002D322C32286
:10C14400E67D0030E7011D08E62BFB18E63CFCE425
:0EC154003DFD22C3EB9FF6F71819EC9EF6F79F
:10C162002212C108400CE47842F608F67840F6083C
:10C17200F6227864C3E6946AF55708E6944CF556BD
:10C182000808C3E69458F55B08E694AEF55A75398B
:10C1920000AC56AD57EC12B24D784C12B2DBAC5A31
:10C1A200AD5BEC12B24D785012B2DB7F2B7E867DF6
:10C1B200777C1812B212785012B2CF12B11E12B29C
:10C1C20012785012B2CF12B11E12B212785012B2BD
:10C1D200CF12B11E12B2127F367E847D257C64128C
:10C1E200B212785012B2CF12B11E12B212784C12A1
:10C1F200B2CF12B11E12B2127F3F7EA27D607C8B43
:10C2020012B212785012B2CF12B11E12AF0C12AF8C
:10C212000C12B2E77F3F7E807D057CE6053912B1C4
:10C222001E784812B2DB7F2C7E937D477C7F12B250
:10C2320012785012B2CF12B11E12B212785012B24C
:10C24200CF12B11E12B212784C12B2CF12B11E121C
:10C25200B2127F357EB47DF87CDF12B212785012B2
:10C26200B2CF12B11E12B212785012B2CF12B11E58
:10C2720012B2127F3F7EED7D227CCD12B212784C3B
:10C2820012B2CF12B11E12AF1012AF0C784412B21A
:10C29200DB7F317E397D9D7CE712B212784C12B27F
:10C2A200CF12B11E12B212784C12B2CF12B11E12BC
:04C2B200B212784408
:10C2B60012B2CF12AF1012B2127F2C7E377D0C7CD9
:10C2C600A312B212784C12B2CF12B11E12B2127869
:10C2D6004C12B2CF12B11E12B212784C12B2CF1259
:10C2E600B11E12AF1012B2E77F3F7E807D027C9FA7
:10C2F600053912B11E784412B2DB784812B2CF1259
:10C30600B2848E428F43784412B2CF12B2848E40EA
:10C316008F4122753900AC42AD43EC12B24D7848DC
:10C3260012B2DBAC40AD41EC12B24D784412B2DB36
:10C336007F2B7E537D507C0912B212784812B2CF01
:10C3460012B11E12B212784812B2CF12B11E12B238
:10C3560012784412B2CF12B11E12B2127F347EF29C
:10C366007DCD7CA312B212784812B2CF12B11E1242
:10C37600B212784812B2CF12B11E12B2127F3F7EAD
:10C386000A7D2E7CAE12B212784412B2CF12B11EC2
:10C3960012AF0C12AF0C784C12B2DB7F2B7E4F7DA6
:10C3A600AF7CB212B212784812B2CF12B11E12B2DC
:10C3B60012784812B2CF12B11E12B212784812B2D7
:10C3C600CF12B11E12B2127F357EB17D4B7C951213
:10C3D600B212784812B2CF12B11E12B212784412BB
:10C3E600B2CF12B11E12B2127F3F7E497DCD7C457F
:10C3F60012B212784812B2CF12B11E12AF1012AF9B
:10C406000C785012B2DB784C12B2CF12B2848D5532
:10C416008E568F57785012B2CF12B2848D598E5ADB
:04C426008F5B78644C
:10C42A00E557246AF608E556344CF608E55534040F
:10C43A00F608E55B2458F608E55A34AEF608E43502
:03C44A0059F6227E
:1091A90012AEA012983A12AEA47F6690A4F012777C
:1091B900331292177F5A78C41291F31291FB78C631
:1091C9001291F31291DE7F6578C81291F31291FB27
:1091D90078CA1291F37E2DE51B12D4CA7E33E51AA3
:1091E90012D4CA7E39E51902D4CA86040886030254
:1091F90053397E15E51C12D4CA7E1BE51B12D4CA4D
:109209007E21E51A12D4CA7E27E51902D4CA7F5AEB
:109219007E01E53A12D3E07E0B909C2EE53B93024A
:10922900D4DDE6FF08E6FE08E6FD339217E45001B7
:10923900F4FC12B2F875130A75390112B4F678D72D
:10924900E6C2E775F00A84F9303D02A9F012B2F8D6
:109259008913053912B4CF30170A053912B4E2055A
:109269003912B4E2A80302B2DB12AEA012983AC2D4
:109279003C7F5A7E0312851012921712DD1B1000D3
:109289000810011510022080EFE53A146004153A20
:109299008003753A3CD23C80DFE53AB43C05753A27
:1092A9000180F2053A80EE7E0312850B7E0B128552
:1092B9001012921712DD1B10000810011510022060
:1092C90080EFE53BB40205753B158002153BD23CA6
:1092D90080DFE53BB41505753B0280F2053B80EE66
:1092E9007E0B12850B7F5A78C41291F31291FB12EF
:0792F900936412836F78C437
:109300001293BC78C61291F31291DE129396751CDB
:109310000012836F78C61293BC7F6578C81291F3F0
:109320001291FB12936412836F78C81293BC78CAAF
:109330001291F31291DE129396751C0012836F78CE
:10934000CA1293BC303C14E53B24F4500B78C9E6B8
:109350002410F618E63427F61293C212AEA4127E39
:10936000F102DD1BC2247E15E51C128460F51CD2BF
:10937000247E1BE51B128460F51B1023E77E21E58C
:109380001A128460F51A1023E67E27E5191284600C
:10939000F5191023E822C2247E2DE51B128460F506
:1093A0001BD2247E33E51A128460F51A1023E77E5F
:1093B00039E519128460F5191023E622ECF608EB62
:1093C000F622129C4678C8E6FE0886073395E0FD33
:1093D000FC12B2127FE87E037D007C0012B4F6120C
:1093E000B21278CAE6FE0886073395E0FDFC12B497
:1093F000CF12B2127F807E697D677CFF12B4CFEC02
:1094000012B24912B2127F3F7E807D0D7C1D12B1D7
:109410001E12B2127F3D7E407D007C0012B2127897
:10942000BC12B2CF12B11E12B2127F3E7E807D00FE
:109430007C0012AF1012B21278BC12B2CF12B11E61
:0994400012B2127F3F7E807D0014
:109449007C0012AF0C12B21278B412B2CF12B11E54
:1094590012B196783C12B2DB7F407E807D007C00A1
:1094690012B212783C12B2CF12B11E12B37512B2F7
:10947900127F3F7EA87D007C0012B21278B812B22A
:10948900CF12B11E12B11E12B2127F407E007D00B2
:109499007C0012B212783C12B2CF12B11E12B3750F
:1094A90012B2127F3F7EC07D007C0012B11E12AF46
:1094B9001012B21278B812B2CF12B11E12B21278CB
:1094C9003C12B2CF12AF10785412B2DB12B35F78EC
:1094D9005812B2DB12B21212B11E12B21278C012B5
:1094E900B2CF12B11E784412B2DB785412B2CF1245
:1094F900B375783C12B2DB12B21212B11E12B2125B
:1095090078BC12B2CF12B11E783C12B2DB7F3E7E1C
:10951900C07D007C0012B212783C12B2CF12B11E8B
:1095290012B2127F3F7E007D007C0012AF1012B292
:1095390012783C12B2CF12B11E12B2127F3F7E8056
:109549007D007C0012AF1012B21278B412B2CF12A1
:10955900B11E787012B2DB78C4E6FE08860733952F
:10956900E0FDFC12B2127FE87E037D007C0012B49C
:10957900F612B21278C6E6FE0886073395E0FDFCBE
:1095890012B4CF12B2127FE07E5E7DF87CFF12B476
:10959900CFEC12B24912B2127F3F7E7F7DE57CC9C2
:0595A90012B2127870FF
:1095AE0012B2CF12B11E12B196785012B2DB7F3FBB
:1095BE007EF07D007C0012B212783C12B2CF12B156
:1095CE001E12B2127F3F7EC07D007C0012AF1012C1
:1095DE00B212783C12B2CF12B11E12B2127F3F7E7F
:1095EE00807D007C0012AF10783C12B2DB78BC128A
:1095FE00B2CF12B2127F3F7E807D007C0012AF0C84
:10960E0012B212783C12B2CF12B21278B412B2CF9A
:10961E0012B11E12B11E784012B2DB785412B2CFC4
:10962E0012B3AD783C12B2DB12B21212B11E7874C4
:10963E0012B2DB7F417E107D007C0012B21278C028
:10964E0012B2CF12B11E12B2127F407E807D007C0C
:10965E000012B212784412B2CF12B11E12B2127FA1
:10966E00417E207D007C0012AF0C12B212784412A3
:10967E00B2CF12B11E12B2127F407E407D007C002E
:10968E0012B212787412B2CF12B11E12B2127F4001
:10969E007EA07D007C0012AF1012AF1012AF0C1224
:1096AE00B212785012B2CF12B11E12B212785012FC
:1096BE00B2CF12B11E12B2127F3D7E2A7DAA7CABB2
:1096CE0012B11E12B2127F3F7E007D007C0012AFDF
:1096DE000C12B212783C12B2CF12B212787012B2D1
:1096EE00CF12B11E12B212784012B2CF12B1961230
:1096FE00B212785012B2CF12B11E12B212785012AC
:10970E00B2CF12B11E12B11E12B212785412B2CFD3
:0C971E0012AF0C12B2127F4A7E517DD2B5
:10972A007CCB12B11E12B28478AC12B2DB7F407EBF
:10973A00007D007C0012B212787412B2CF12B11EF0
:10974A0012B2127F3F7E807D007C0012AF1012B2EF
:10975A0012784412B2CF12AF1012B212785012B26B
:10976A00CF12B11E12B212785012B2CF12B11E121B
:10977A00B212785012B2CF12B11E12B2127F3E7ECE
:10978A002A7DAA7CAB12B11E12B212785012B2CF45
:10979A0012AF0C12B212785812B2CF12B19612B29C
:1097AA00127F4A7E517DD27CCB12B11E12B2841234
:1097BA00B212AF3AEF3395E0FEFDFC12B2127F40CF
:1097CA007E7E7D057C0012B4F612B2127F607E7531
:1097DA007D587CFF12B4CF12B4CF78B012B2DB78C6
:1097EA00AC751B641298118F1C78B0751B671298A0
:1097FA0011E51C75F00AA42FFF249C50027F007803
:10980A00D7E654802FF62275390012B2CF12B2125F
:10981A007F0A7E007D007C0012B5A2A81BE513F624
:10982A0008E512F608E511F6335004EFF404FF22B6
:10983A00C23D78647BAC12922BD23D78677BB01222
:10984A00922B129C467F007EE47D577C0012B21256
:10985A0078AC12B2CF12B4CF12B2127F007E537D0F
:0E986A00077C0012B5A212B23185133B7F803D
:109878007ECB7DA47C0012B21278B012B2CF12B4A3
:10988800CF12B2127F407E7E7D057C0012B5A212F7
:10989800B231E513F56F04F53A85126E85116D85C1
:1098A800106C7F407E7E7D057C0012B212786C12AF
:1098B800B2CF12B4F612B2127F607E0C7DA27C0089
:1098C80012B21278B012B2CF12B4CF12B4E2786CDE
:1098D80012B2DB78AC12B2CFEC12B24912B2127FDC
:1098E800347E9C7D2B7C5F12B11E785412B2DB1241
:1098F800B35F785012B2DB786C12B2CFEC12B24977
:1099080012B2127F347E9C7D2B7C5F12B11E12B284
:1099180012785012B2CF12B11E784012B2DB7F40DB
:109928007E007D007C0012B212785412B2CF12B1C0
:109938001E12B37512B2127F3D7EC07D007C0012EC
:10994800B21278BC12B2CF12B11E12B2127F3E7E92
:10995800C07D007C0012AF1012B21278BC12B2CFD8
:1099680012B11E12B11E12B2127F3D7E407D007CE4
:109978000012B21278BC12B2CF12B11E12B2127F0C
:109988003E7E807D007C0012AF1012B21278BC12AD
:10999800B2CF12B11E12B2127F3F7E807D007C00D2
:1099A80012AF0C12B212785412B2CF12B11E12AF0B
:1099B8000C12B2127F407E807D007C0012B21278B9
:1099C8005412B2CF12B11E12B37512B2127F3D7E7D
:1099D800707D007C0012B21278BC12B2CF12B11E98
:1099E80012B21278BC12B2CF12B11E12B11E12AF4F
:1099F8001012B21278B412B2CF12B11E785812B245
:109A0800DB785412B2CF12B375783C12B2DB7854BB
:109A180012B2CF12B3AD785412B2DB783C12B2CF87
:109A280012B21212B11E12B21278BC12B2CF12B117
:109A38001E783C12B2DB7F3E7EC07D007C0012B2F5
:109A480012783C12B2CF12B11E12B2127F3F7E00C2
:109A58007D007C0012AF1012B212783C12B2CF1205
:109A6800B11E12B2127F3F7E807D007C0012AF10C3
:109A780012B21278B412B2CF12B11E787012B2DBE1
:109A8800785012B2CF12B21212B11E12B21278C0AE
:109A980012B2CF12B11E784412B2DB785412B2CF90
:109AA80012B21212B11E787412B2DB784012B2CF21
:109AB80012B21212B11E783C12B2DB7F407E807D5A
:109AC800007C0012B212784412B2CF12B11E12B248
:109AD800127F417E107D007C0012AF1012B2127806
:109AE8004412B2CF12B11E12B212787412B2CF124F
:109AF800B2127F407EA07D007C0012AF0C12AF1026
:109B080012B212783C12B2CF12B11E12B2127F3DBD
:109B18007E2A7DAA7CAB12B11E12B2127F3F7E0054
:109B28007D007C0012AF1012B212785412B2CF121C
:109B3800B212787012B2CF12B11E12B212783C1261
:109B4800B2CF12B11E12B11E12B212785812B2CF91
:109B580012AF1012B2127F3F7E7F7DE57CC912B131
:019B68001EDE
:109B690012B2127F4B7E187D967C8012AF1012B212
:109B79008412B2127FE87E037D007C0012B5A21226
:109B8900B23178C8A61208A61308A60608A607784F
:109B99007412B2CF12B2127F3F7E807D007C001218
:109BA900AF0C12B212784412B2CF12AF1012B21225
:109BB9007F3E7E2A7DAA7CAB12B11E12B21278407A
:109BC90012B2CF12B11E12B212783C12B2CF12B138
:109BD9001E12B212784012B2CF12AF1012B2127F17
:109BE9003F7E7F7DE57CC912B212787012B2CF1226
:109BF900B11E12B11E12B2127F487EF47D247C0080
:109C090012AF1012B28412B2127FE87E037D007C7B
:109C19000012B5A212B23178C4A61208A61308A67A
:109C29000608A607223F3F4344454647484A4B4C4E
:109C39004D4E5051525354555657583F3FE4F539FC
:109C4900F5A7909C5A791078B4E493F6A308D9F94A
:109C59002232A5C24A4A19DC3A885CDB3BFFD6DCD2
:019C69003BBF
:10AEA000D2D58002C2D575A70490040078107F0B1C
:10AEB00012AECC78267F0512AECC783C7F2212AE43
:10AEC000CC786A7F0F12AECC75A7002230D506E68B
:10AED000F008DFFB22E0F608DFFB22D2D58002C2B9
:10AEE000D575A7049006FA78737F0612AECC75A7C5
:10AEF0000022DA0CD902800BD906303701B3500595
:10AF000002B07F923702B06BD9F680F9D236800258
:10AF1000C23612B0B0303606C86002B237C89236B8
:10AF2000DAD0D9E4B8000A12B0F7A236923702B0EC
:10AF30005460FBB51300400F12B0F7A23692F7A28F
:10AF4000379236A2F79237C398F40424E740DF24FF
:10AF500019AD29AC28AB277A00C394084008CDCCA2
:10AF6000CBCAE4CD80F424086010F9C3ED13FDECE6
:10AF700013FCEB13FBEA13FAD9F1A236303701B315
:10AF800040308A17E5102BF518E5113CF519E5124C
:10AF90003DF51A501A13F51AE51913F519E51813AA
:10AFA000F518E51713F5170513E5137002051402DC
:03AFB000B00AE400
:10AFB300C39AF517E5109BF518E5119CF519E512F1
:10AFC3009DF51A500DB237C378177F04E496F6083F
:10AFD300DFFA7A047019E513C39408F513500215C8
:10AFE30014E4C517C518C519F51ADAE802B0AB2081
:10AFF300E7BAE5137002151415137817C37F04E637
:10B0030033F608DFFA80E8E51A20E7137817C37FE1
:10B0130004E633F608DFFAE513700215141513E599
:10B02300173378187F03E63400F6500E08DFF77500
:10B033001A800513E51370020514E51420E7547014
:10B0430027E513604E046020851A128519118518AF
:10B05300105326F0AC10AD11A237E51313FFE51220
:10B0630092E7FEA81302B231E4F512F511F510F5DB
:10B07300147513FF5326F043260580D8E5FFF51218
:10B08300F511F510751400F513D2375326F0432646
:10B093000980C15326F0432603E4F512F511F51098
:10B0A300F514F513C23780AC5326F080EC79017A9E
:10B0B300018512F0E513A2F7339237751400F513E7
:10B0C3006002D2F785F012A813B8FF0809E512C28F
:01B0D300E795
:10B0D4006001098C278D288EF0A2F7EF3304700AE3
:10B0E4000AC2F705F00AD5F0011A146002D2F785F6
:10B0F400F02922C88813C512C529C512C511C5284F
:10B10400C511C510C527C51022DA03B8000302B063
:10B114007FD9028002D9F702B06B12B0B030370188
:10B12400B392377004D9E78005DADEB8000302B0C1
:10B13400ABD9E2C3947E500215142513F5135002C3
:10B1440005147815760008B81BFA78277915E608EF
:10B15400FAE8FC78108AF0E608A427F709E5F03746
:10B16400F7500989F00907E760FBA9F0B813E6195D
:10B1740019ECF8B82AD802B00A02B096B8FFFA025D
:10B18400B07FD9FB02B06BDAF6B800F002B0AB12B4
:10B19400B2E712B0B0303701B392377007D9E3B8D1
:10B1A40000E280DBDAE1B8000280E1D9D5C8C398B7
:10B1B40050021514247F50020514F513781A7600F2
:10B1C4007A1A7B80C3E5109527E5119528E5129539
:10B1D400294016C3E5109527F510E5119528F511BA
:09B1E400E5129529F512E64BF67F
:10B1ED00DA0302B00AEB03FB30E703187600C3E580
:10B1FD001033F510E51133F511E51233F51240CA90
:10B20D0030E7DD80B6E53905396010D0F0D0E0C00B
:10B21D0010C011C012C013C0E0C0F08F138E128D7C
:10B22D00118C1022E539146010D0F0D0E0D013D07D
:10B23D0012D011D010C0E0C0F01539227920800C49
:10B24D007910800479087D007E007F003392D550FF
:10B25D000312B2C1EC33400FEF33FFEE33FEED338B
:10B26D00FDEC33FCD9EE22EECCF5F0747E29A2D59F
:10B27D0013FF92F7AEF022EF8EF0A2F7D2F73392D2
:10B28D00D5C3947F5006E4FFFEFDFC2294204004BC
:10B29D0074FF80F304CCFEE4FFFAE5F0CC6012C33A
:10B2AD00CC13CCCD13CDCE13CECF13CF0450EEDABD
:10B2BD00EC30D5D7C3E49FFFE49EFEE49DFDE49CF6
:03B2CD00FC22E67A
:10B2D000FC08E6FD08E6FE08E6FF22ECF608EDF6BF
:10B2E00008EEF608EFF622CFC513CFCEC512CECDAD
:10B2F000C511CDCCC510CC22E4F513F512F511F52E
:10B300001022E493FCA3E493FDA3E493FEA3E4934F
:10B31000FFA322C0E012B21212B11E12B34612B342
:10B3200002D0E0C0E012B21212B33D12B11E12B24E
:10B330001212B30212AF10D0E0D5E0E722AC48AD54
:10B3400049AE4AAF4B228C488D498E4A8F4B2274AE
:10B35000FF7809FFFEFDFCE52654F048F526221291
:10B36000B40604A2E1927F1420E01590B48774041F
:10B3700012B313802912B40630E102B27F20E0EB51
:10B380008C4C8D4D8E4E8F4F90B49B740412B31322
:10B3900012B212AC4CAD4DAE4EAF4F12B11E307F5B
:10B3A00004EF6480FFEE33EF337001FF2212B40626
:10B3B000C0E08C4C8D4D8E4E8F4F90B4BF740312F5
:10B3C000B31312B212AC4CAD4DAE4EAF4F12B11E14
:01B3D000EC90
:10B3D100C54CFCEDC54DFDEEC54EFEEFC54FFF90D2
:10B3E100B4AF740312B313D08212B212AC4CAD4D90
:10B3F100AE4EAF4FE58230E00712B196B27F809D2D
:10B4010012B1938098EE33EF3324605007D0E0D02F
:10B41100E002B34FEFA2E7547F927FFF12B2127C9A
:10B42100837DF97E227F3E12B11EEE33EF332481FC
:10B43100501012B21212B28412B249EFB2E7FF12E7
:10B44100AF10EE33EF33602A2403F8C313FFEE92FB
:10B45100E7FEE82481E4501A12B21212B284EF041A
:10B46100C2E0FCF58212B251EFB2E7FF12AF10E574
:10B471008203FAEE33EF33600B148FF0A2F713FF60
:10B48100EE92E7FEEA2283FA703AE4E9AABCF8E018
:10B49100813EE6E99DBF0000803F1A3C283966697C
:10B4A10099BBE335A33DE75D25BFDB0FC93FCCDB8E
:10B4B1008D41EE3649C43F91C9453DF8B0C5000004
:10B4C100803F34F517C373FA2F45DDFD0AC6EF251A
:10B4D10013FFEE3512FEED3511FDEC3510FC02B215
:10B4E10031C3EF9513FFEE9512FEED9511FDEC952D
:10B4F10010FC02B231EFF88513F0A4FFE513C5F09B
:0AB50100CEF9A42EFEE435F0CDFAD9
:10B50B0088F0E512A42EFEED35F0FDE433CC851367
:10B51B00F0A42CFCE5128AF0A42CFCE51189F0A414
:10B52B002CFCE51088F0A42CFC89F0E512A42DFD71
:10B53B00EC35F0FCE51188F0A42DFDEC35F0FC8A20
:10B54B00F0E513A42DFDEC35F0FC02B231E4CCF8A0
:10B55B00E4CDF9E4CEFAE4CFFB75F020C3E5133369
:10B56B00F513E51233F512E51133F511E51033F54B
:10B57B0010EF33FFEE33FEED33FDEC33FCEF9BEEC0
:10B58B009AED99EC98400CFCEF9BFFEE9AFEED992F
:10B59B00FD0513D5F0C622C2D5EC30E705B2D512A6
:10B5AB00B2C1E51030E70DB2D512B5C512B55812C0
:10B5BB00B2C1800312B55830D515C3E49513F513FA
:10B5CB00E49512F512E49511F511E49510F510229E
:10A68500E57124885002D2191256DC8E4712D1F09A
:10A69500129189125A98305E0F125A361288781222
:10A6A500596712BFF612425412393A1247FB103657
:10A6B50029201F1C301219E412A80B12A82012A978
:10A6C5002012A94230510302A9CC12AC9D20510998
:10A6D500C251E4F552F545F5442275A70075830787
:10A6E500E559C454F0F582E0F538A3E0F518A3A3C5
:10A6F500A3E0F51E74FF12A80B1256DC8E1C8F1BEF
:10A705007510DF751100E51164B4700612A7D675D2
:10A71500111012A7A34028AE1CAF1B12576420329C
:10A725001EAC03AB027A0C125371ED701275A700C3
:10A73500758304851182ECF00583E510F00511D5CC
:10A7450010C412A7D675C70375C6E075A704900592
:10A75500007F0412A791DFFB75A700122B83125A05
:10A7650036E4F5A7F8F559758307E8C4F582E06581
:10A77500387011A3E06518700BA3A3A3E0651E70E4
:10A785000388592208C3E5589850DC22E0F5BCE05F
:10A79500F5BDE0F5BEE0F5BF124EE605C622E510B3
:10A7A50075F004A4F5C685F0C775B901E5BC33405D
:0BA7B5001F05C605C675B90185BE640E
:10A7C00085BF6505C675B90185BC6685BD6785BE53
:10A7D0006885BF69C322E51124FE502E75A7007F4E
:10A7E00010AE111E7583048E82E0FD1582E0CDB59A
:10A7F00005005012F00582CDF00583E0FD1582E0E2
:10A80000CDF00582CDF0DEDCDFD72275A7549004B1
:10A810000005A79005007FB4F0F0DFFC75A70022CB
:10A8200012BE4AC2517B077AFFE4FFF5A7900400ED
:10A8300012A906ED244C4035EC603075A7008D82DE
:10A8400005A712A8CC7583058D82E02410401CF06A
:10A8500005A7E02CF0500505A7E004F0BA000CBBFA
:10A860000009D251EF24DC50027F23DFC3EA6005E8
:10A8700012A87F8006EB600312A8B775A7002230EC
:10A88000E0047553082230E1047553182230E204C5
:10A890007553282230E3047553382230E40475538D
:10A8A000482230E5047553582230E6047553682277
:10A8B00030E7037553782230E0047553882230E185
:10A8C000047553982230E2037553AA22ED54F0C464
:10A8D000232390A8D6735302FE225302FD22530273
:06A8E000FB225302F722E7
:10A8E6005302EF225302DF225302BF2253027F227A
:10A8F6005303FE225303FD225303FB225303FB2281
:10A9060012BD8212BC10E4F5F7C2B2C2B2ADF7F5C1
:10A91600F7C2B2C2B2ACF7D2B22290050078B4E068
:10A926006015FD54F0C4CD7C00540FFE1583E0FF86
:10A9360012546FEFF005830582D8E42275830478FC
:10A94600FF088882E060FAF5D38812E512244C509D
:10A95600012285D3D288D4881279FF0512E51260C8
:10A96600F00908E875F0B484A8F08882E060ECF598
:10A97600D3B9000280D5B9230050D0C395D292D165
:10A986005002F40409FEE4FFFCAD0112547C74018C
:10A99600FA25D475F0B484A8F0AC06AB071253635D
:10A9A600EB30E7010CE5D22C30D1029C9C8882F07A
:10A9B6000AEAB501DCE512244C50012285D3D28582
:10A9C60012D4A812809390040012AA8B8C068B05D1
:10A9D60012AA8BE4FFF512F5118C148B13C3ED9BB1
:0EA9E600F9EE9CFA4012E51199E5129A500A1A
:10A9F4008C148B138A1289118F528F82E0F9C3ED64
:10AA040099FDEE9400FEE582245A5002244C75F020
:10AA1400B48485F082E0FA2DFDEE3400FEEB9AFB5F
:10AA2400EC9400FCE92BFBEC3400FC0FBFB4B0E564
:10AA34005224D3400224B4F552C3E51333FBE51486
:10AA440033FCE511FE2BFBE512FF3CFC1254D1E96B
:10AA5400F890AA9D93F511FDEBF513FFECF514FEA8
:10AA64007C0012546F8F44E890AB9D93FAAB13AC07
:10AA74001412539AAF03AE04AD117C0012546FEF5D
:10AA84007002F552F545227C007B007F5AE02BFBD7
:10AA9400EC3400FC0582DFF522B4B4B4B4B4B4B42D
:10AAA400B4B4B4B4B4B4B4B4B4B4B4B3B3B3B3B367
:10AAB400B3B3B3B3B3B3B3B3B2B2B2B2B2B2B2B26A
:10AAC400B2B1B1B1B1B1B1B1B0B0B0B0B0B0B0AF7A
:10AAD400AFAFAFAFAEAEAEAEAEAEADADADADADAC95
:10AAE400ACACACACABABABABAAAAAAAAA9A9A9A9BA
:10AAF400A9A8A8A8A8A7A7A7A7A6A6A6A5A5A5A5E7
:10AB0400A4A4A4A4A3A3A3A2A2A2A2A1A1A1A0A01D
:10AB1400A0A09F9F9F9E9E9E9D9D9D9D9C9C9C9B57
:10AB24009B9B9A9A9A999999999898989797979696
:10AB340096969595959494949393939292929191D9
:10AB440091919090908F8F8F8E8E8E8D8D8D8C8C19
:10AB54008C8B8B8B8A8A8A8989898888888787875E
:10AB640086868685858584848483838382828281A4
:10AB740081818080807F7F7F7E7E7E7E7D7D7D7CE7
:10AB84007C7C7B7B7B7A7A7A797979787878777729
:10AB94007776767675757574740002030506080970
:10ABA4000B0C0E101113141617191A1C1D1F212239
:10ABB400242527282A2B2D2E303133343637393AA1
:10ABC4003C3D3F404243454648494B4C4E4F505212
:10ABD40053555658595A5C5D5F6061636466676893
:10ABE4006A6B6C6E6F707273747677787A7B7C7E26
:10ABF4007F80818384858688898A8B8D8E8F9091CE
:10AC0400929495969798999B9C9D9E9FA0A1A2A48F
:10AC1400A5A6A7A8A9AAABACADAEAFB0B1B2B3B468
:10AC2400B5B6B7B8B9BABBBCBDBEBFC0C0C1C2C35C
:10AC3400C4C5C6C7C7C8C9CACBCCCCCDCECFD0D06B
:10AC4400D1D2D3D4D4D5D6D7D7D8D9DADADBDCDC91
:10AC5400DDDEDEDFE0E0E1E2E2E3E4E4E5E5E6E7D1
:10AC6400E7E8E8E9EAEAEBEBECECEDEEEEEFEFF027
:10AC7400F0F1F1F2F2F3F3F4F4F4F5F5F6F6F7F794
:10AC8400F8F8F8F9F9FAFAFAFBFBFBFCFCFDFDFD18
:10AC9400FEFEFEFEFFFFFFFFFFC251E4F544F81481
:10ACA400FB900400A9007C0FC2D112ADB8E82405C2
:10ACB400F8B8B4F08B13E5122403FA244C5001FACB
:10ACC400BBFF012275112C8A1912ADEF8F16203D9E
:10ACD40012AA1975112312ADEF8F15751600303DA8
:10ACE400E2801175112312AD97751500303D05E80A
:01ACF4002F30
:10ACF50013F51575111212AD97751400303D05E861
:10AD05002F13F514EA2404F552244C5002F552E4AD
:10AD1500F51AF51BF51CE516600AFB7A00AF137EE4
:10AD2500FF12AD5DE515600AFB7A4FAF137EFF128A
:10AD3500AD5DE516600DFB7A00E5146006FF7ECF7C
:10AD450012AD5DAE1CAF1B7C00AD1A12546F8F4562
:10AD5500EF2513F544D25122EFF5F0A4FCADF0EB4D
:10AD6500F5F0A49CFCE5F09DFDEB8AF0A4FAABF0B0
:10AD7500EF8EF0A49AF8E5F09BF9E833F8E933F99A
:10AD85007B00125515051AE51B2BF51BE4351CF543
:10AD95001C22EA2511F9244C5001F9C2D112ADB695
:10ADA500303D428F00C3EA9511F9500324B4F9D21E
:10ADB500D17C09E4FDFEFF8982E060062FFFE43EB9
:10ADC500FE0D09B9B4027900DCEDED20D118F51EB0
:10ADD50024FE923D500F12547CEFB50300500685BA
:10ADE5001E1FFB881222F51D80E612AD97203D43FC
:10ADF500740212AE8E12AD97203D38740412AE96D1
:10AE050012AD97203D2D740612AE8E12AD97203DE2
:10AE150022740812AE9612AD97203D17740A12AE31
:10AE25008E12AD97203D0C740C12AE9612AD972084
:10AE35003D0122C3E89F605088148F158A1640088B
:10AE45001ABAFF0A7AB380060ABAB4027A0012ADBA
:10AE550097303D34C3E89FF9602EC3E5149515FB83
:10AE65006930E7D4E930E703F404F9EB30E702F49D
:10AE750004C3995002AA16E5142515C82F28FFE426
:10AE8500FC33FE7D0412546F222AFA244C5001FA39
:0BAE950022C3CA9AFA500324B4FA2228
:10BBD700758000C2B212DE11D2B275F830227580BC
:10BBE70000C2B2F5F7C2B2C2B2D2B222758000C2A9
:10BBF700B2F5F7C2B2C2B2856CF7C2B2C2B2856BF8
:10BC0700F7C2B2C2B2856AF722758000C2B275F771
:10BC170003C2B2C2B2856FF7C2B2C2B2856EF7C2B3
:10BC2700B2C2B2856DF72212BC67740612BBE57407
:10BC37000212BBF38FF7C2B2C2B2D2B222909F5F99
:10BC47007F631276F012DD1BD214120E9412766EF9
:10BC5700124EE612BC67740612BBE574C712BBE549
:10BC670012BC6D40FB22758000C2B275F705C2B2E7
:10BC7700C2B2C2B2C2B275F705C2B2C2B2C2B2C2D2
:10BC8700B2E5F7D2B2A2E022120E9485BF6C85BE50
:10BC97006B756A00E56B7015E56A701112BC677405
:10BCA7000612BBE574D812BBF3D2B2D21F22E54B02
:10BCB7000475F03C8485F04B12BF72852E72E55FE8
:10BCC700030354C0F8E55E543F28F57C3055012244
:10BCD70012BD0C12BC6D40F7E54C60F312BC671245
:10BCE700BD2312BCF180F112BC67C21F740612BBE0
:10BCF700E5740212BBF3787086F708B880FAD2B2FF
:10BD070012BD40808F787075A704758304E54CC415
:0CBD1700F5827F10E6F0DFFC054C80197F
:10BD2300787075A704758304154CE54C30E701E47E
:10BD3300C4F5827F10E0F6DFFC75A700227410259E
:10BD43006A54F0F56AE4356BF56BE4356C540FF522
:10BD53006C22E54B75F010A4256A54F0F56AE5F002
:10BD630080E4E56A24F054F0F56AE56B34FFF56B83
:10BD7300E56C34FF80D7E56A24FF80ECC380EBE5F4
:10BD83006D24F054F0F56DE56E34FFF56EE56F3418
:10BD9300FF540FF56F2212BDF112BE19C22DC2540A
:10BDA300C255E57F7002D255147002D254E54A3071
:10BDB300E00122B4061C20540D12BD6512BEC1124F
:10BDC300BF5112BF892212852F7E0412DE09754AE4
:10BDD300012220550D12BD4012BF3012BF7212BE98
:10BDE3009A2212852F7E0412DE09754A05227403F6
:10BDF30012BBF37870E4F5F7C2B2C2B2A6F708B883
:10BE030080F3D2B222740312BBF3E4F5F7C2B2C2D9
:10BE1300B2E5F7D2B222E575F8541F30E40244E0EC
:10BE2300F57585722EA2779226E57C543F30E502A4
:10BE330044C0F55EE57C54C02323F55FE57FC2E78C
:10BE430079BCF709A77E22856C6F856B6E856A6D59
:01BE530022CC
:10BE5400856F6C856E6B856D6A22E4FEFF740775D1
:10BE6400A704F5838E8274FFF0DFFD75A7002274AA
:10BE7400067E007FB012BE63E4F55AF55B2275A717
:10BE840004758306E55A600A75F00A84E5F07002C9
:10BE9400740AC4F58222307720E55A240240020550
:10BEA4005A12BE82E55AF0E573F0E574F0E575F0D8
:10BEB400E576F0E577F0E578F075A700223077F9BC
:10BEC40012BE827F1074FFF0DFFDE55A24F55003A3
:10BED40012BEEC155AE55AB4FF02055AC3E55A9549
:10BEE4005B50D6755B0080D112BE4A7F0A056D0592
:10BEF4006D12BC10E4F5F7C2B2C2B2E5F7D2B230AB
:10BF0400E704DF02800512BD8280E2056D12BC10D9
:10BF140012BE82E55A24F6F07F06E4F5F7C2B2C2F7
:10BF2400B2E5F7F0DFF4D2B275A70022053FE53F92
:10BF3400B43C17753F00053EE53EB43C0D753E002C
:10BF4400053DE53DB41803753D00024ABB153FE5C8
:10BF54003FB4FF17753F3B153EE53EB4FF0D753EFC
:10BF64003B153DE53DB4FF03753D17024ABB054251
:10BF7400E542B43C0F7542000541E541B43C05750A
:0CBF840041000540221542E542B4FF0FC9
:10BF900075423B1541E541B4FF0575413B15402213
:10BFA000AC40AB41A842EC75F03CA42BFBE435F06F
:10BFB000FC7A3C125363EB28FBE43CFC22AC3DAB27
:10BFC0003EA83F80E178AE8604AB3EE53FC313F860
:10BFD000800C7800120E5DE5BE75F005A4FBE5BF90
:10BFE00075F03CA42BFBE435F0FC7A1E125363EB96
:10BFF00028FBE43CFC2212BFD2AE04AD0312BFC545
:10C000008C148B13120E67E5BFFF24F650027F01DC
:10C01000E5BE75F096A4AAF0F9C3ED9513FBEE9575
:10C0200014FC924E4B701120110E30480B75364B9C
:10C030003003037536FFD22E304E02DF1F7A021214
:10C04000536375A7009004EEECF0A3EBF0C3E5BFDB
:10C050009F04BF0102D2E79005CBF022ED29FDEE4F
:04C060003AFE80B56F
:10DDF60012DDFF12DDFF12DDFF7E0480067E02804B
:10DE0600027E017F0080087F6480027F017E00EF32
:10DE16004E6012E4FD0D1D0DEDC394AD40F7EF1FEE
:10DE260070ED1E80EA22753500C200C201C20222D0
:10DEDD00F5D8D2DCE5F520E7FBE5DA540FFEAFD936
:04DEED0075D80022C2
:10DAE4007F767E06909C7E127702740412DEDD7CC3
:10DAF400007D5212546FEFF875F00A84C0F07F76FF
:10DB04007E2312D4CA7E29742E12D4DD7E2ED0E058
:10DB140012D4CA7E35745612D4DD7F6B7E1190DB2D
:10DB24004D12D509E824E04001220423F824E750EB
:10DB340002781812DB3DD8FB227F6CE82411FE79B1
:10DB44000512DE360E0FD9F922071DFFFFFFE08014
:10DB5400000020C0000038E0000008F0000038F8A1
:07DB6400000020FFFFFFE0BD
:10DB6B0012DB9330E6022409540F75F00AA4F51565
:10DB7B0012DB9330E6022409540F25152212DB9396
:10DB8B00540F2275F000800875F044800375F00780
:10DB9B00E4206D09D5E0FAD5F0F7D24C229247C2BA
:10DBAB00ACE54F623885504FA26E926D859950C28D
:10DBBB006FD2ACC24CA2472212DBCDC4FA12DBCD22
:10DBCB002A2212DB9320E603540F22540724092246
:10DBDB00E612DBE218E608FAC412DBE8EA540F445B
:10DBEB0030F924C6E950112407800D75F00A84C062
:10DBFB00F012DC01D0E0443030530975F00085E0C1
:10DC0B00E0D5F0FA3099FDC299F599623822E538E2
:10DC1B0080F2E53812DBE2800812DC03E53812DC17
:10DC2B0003740D12DC03740A80CE744012DC03748F
:10DC3B004080C5742C80C1742E80BD75380080B8AF
:10DF030085A0835383FE438380858384F0758400D7
:01DF130022EB
:10D9920074A212DF0374A112DF0374A612DF0374F0
:10D9A200A412DF0374C012DF03742512DF0312DA3C
:10D9B2002275C70375C6FC75B90112B5DB7408126E
:10D9C200DEDDEE75F020A4FEEF54F80303032E24EF
:10D9D20092C313FE24EA50027E16EE90DA0B9325D0
:10D9E200BCFE24E6501F24E8401B748112DF03EEC4
:10D9F20012DF0312DA2F744012DF03742F12DF03D7
:10DA020074AF02DF037E2680E1F7F7F8F8F9FAFB3C
:10DA1200FCFDFEFF000000000101020202030303FD
:10DA2200A8BCA9BDAABEABBFACC7ADC62288BC8983
:0ADA3200BD8ABE8BBF8CC78DC622D3
:10DD1B00C006C007C5F075A7019000007EB7E58C63
:10DD2B00240340FA12DD3D1EBEAFF3C5F0D007D081
:10DD3B00062275A700EE12DF03741012DF037404C2
:10DD4B0012DF0385A08343838185838475A7517F6D
:10DD5B0020E0F0E0F0E0F0E0F0DFF6E4F5A7F5848A
:01DD6B002295
:10DEF10075A711900000E4C583F0C58330E2F8F501
:02DF0100A72255
:10DE3600EF20E723EE20E71F20E61C05A7C45403C6
:10DE4600F583EE5408C42FF582EE5407240983F5B2
:10DE5600F0E045F0F005A7228040201008040201FA
:10DE6600EF20E723EE20E71F20E61C05A7C4540396
:10DE7600F583EE5408C42FF582EE5407240983F582
:10DE8600F0E055F0F005A7227FBFDFEFF7FBFDFEC0
:10D48A00FDA42582F582E5F03583F583ED229060CF
:10D49A00AC7A0475F00512D48A7D05805E7A05801F
:10D4AA00027A04547FC0E0C083C082C39420500132
:10D4BA00E490605C12D49D802E9061BA7A05800552
:10D4CA009062777A0675F00712D48A7D07802C7AE3
:10D4DA000580027A06C0E0C083C082C3942050014E
:10D4EA00E490620712D4CFD082D083D0E022905F3A
:10D4FA00D075F00A12D48A7D0A7A07C2D18002D284
:10D50A00D1C0A7C082C083C007C006C0E030D1091D
:10D51A0075A704E493FDE493FAEEFB75A704EBFE0A
:10D52A00EAFC7901D9067908E493F5D4E5D423F520
:10D53A00D420E01612DE660EDCEA0FDDE1D0E0D080
:10D54A0006D007D083D082D0A72212DE3680E89098
:10D55A005F1075F00E12D48A7D0E7A0812D50590E6
:10D56A005FB875F00212D48AE493FDE4A393FACE6D
:10D57A002408CE7C0812D5867C06AD02ED23FD2058
:0ED58A00E00712DE660FDCF42212DE3680F7B8
:10D37500F5D2C2D58036F5D2D2D58030F5D224F695
:10D3850050090E0E24A650030E0E0EE5D2F5D275E9
:10D39500F0648485F0D3C2D57009D2D5742012D437
:10D3A500DD800312D4CACE2406CEE5D375F00A84F7
:10D3B50085F0D3700A30D507742012D4DD800312AE
:10D3C500D4CACE2406CEE5D312D4CAE5D222F5D2EC
:10D3D50075F0648485F0D3C2D58022F5D2C2D5809C
:10D3E50025F5D2D2D5801FF5D275F0648485F0D3AA
:10D3F500C2D57009D2D5742012D4DD800312D4C3EE
:10D40500CE2405CEE5D375F00A8485F0D3700A30B5
:10D41500D507742012D4DD800312D4C3CE2405CEE3
:10D42500E5D312D4C3E5D222F5D2C2D58035F5D2E3
:10D43500D2D5802F30E70DF404C0E0742D12D4ABA3
:10D445000E0ED0E0F5D275F0648485F0D3C2D570A8
:10D4550009D2D5742012D4AB800312D498CE2404FB
:10D46500CEE5D375F00A8485F0D3700A30D50774FC
:10D475002012D4AB800312D498CE2404CEE5D31267
:05D48500D498E5D2225D
:1076E700909F5F1276F002DD1B7E00800E7405FE10
:1076F700F51EE4FFF51DF51F203C3375A700E49345
:10770700700122A3B40204051D8003B4010A051FFA
:10771700EF2409FFAE1E80E612D4DD7D06B44002D9
:107727007D03B421027D02EE2DFE80D27E0075A777
:1077370000E493700122A3B40204051D8003B40181
:107747000F051FEF2407FFAE1E80E612D4A780089F
:10775700B45B0050F612D4AB0EB4210280D30EB442
:10776700400280CDB42C0280C80E0EB45F0280C1E7
:10777700B45B0040BC0E0E80B8E60812D4DDEE24E0
:1077870006FED513F422909CAC307409909CB0305F
:107797007303909CB502770275F019D5E0FDD5F01B
:1077A700FA12484F12DC35744F12DC46744B12DC68
:1077B70024C322C2501277FE12484FD2AC12DB8E7E
:1077C700304C1212DB8E304C0C12DB8E304C06D252
:1077D70050C2ACD322B440E512DB93B4400312DBB2
:1077E70093B44FED12DB93B44BE712DB9312DB93A9
:1077F70012DB93C2ACC32230530975F008D5E0FD04
:10780700D5F0FA227F0575F019D5E0FDD5F0FA120B
:10781700484F12DC35745712DC46745012DC03747F
:097827008112DC03E56312DC03AD
:10783000E56212DC0378D0E612DC0308B8D7F8E67C
:10784000F8795F30E702792FE912DC0312DC0312CA
:10785000DC0312DC03745812DC03744312DC03E40F
:1078600012DC03E8C2E775F00A84C425F012DC03D9
:107870007864E612DC0308B869F8E612DC241277B3
:10788000BA400122DF02800A20508B75F000808010
:10789000D250C2ACD3221277FEC25012484FD2ACA3
:1078A0002002EF12DB8E204CE7B440F412DB93B4DD
:1078B000400312DB93B457DAF53812DB93B450D29D
:1078C00012DB9312DB93F56312DB93F56278D0122F
:1078D000DB93F924A0500353015FE924E0400279CF
:1078E0005FA60108B8D8E8780612DB93D8FB12DB54
:1078F00093FC53040FC4540F75F00AA42CFC249C71
:1079000050027C0078D78601E4B92F02D2E72CF62A
:10791000786412DB93F608B86AF812DB93E53860F6
:107920000302789212DB9312DB93C2ACC32290A3C2
:107930004C8003909FA37F2012773312DD1B02DE61
:1079400007753400C26B1279FD12DE07127DADE5BA
:1079500016600312795902025912800F121E461244
:10796000DD1B10002010010280F8127E1850131247
:107970001E5112792E10000D10010280F8121DF315
:0579800080D7127B9D81
:1079850022C26BD22775480A122B77753400127EF6
:10799500E5C26A1233CF106A0512024A80ED12025F
:1079A5004A127D3F127E97127EF178D0E6642660FA
:1079B5004412800F121E4612DD1B10003810010202
:1079C50080F8127E18501BE965156018121E5112B9
:1079D500792E12DDFF10001D10010280F8121DF333
:1079E50080BCD26B127EC3751607855917122BF012
:1079F5007535008096020259127DAD127A1F127EEE
:107A0500F17F19127A3990A3797E121277357E2388
:107A1500E51602D44990A4C380EF7862E4127A3067
:107A250078D0745F127A3018E4F6227F08F608DF02
:107A3500FC227F7B7E007810742012D4ABCE240408
:107A4500FED8F5227F197E081277357E28909F850E
:107A5500305303909F8A027735C26B127A1F127AD0
:107A650069020259C251127EF190A371127A49122C
:107A75001E19127DAD7F20127A0812DD1BE51670E6
:107A85000512DDFC803675A6FF3051031277A8126A
:107A9500484FD2AC200025306DFA127899400C126F
:107AA5007E184011127B9DD25180BB105003127974
:107AB50033C25180D1D25112792E80CAC2AC22D2A2
:107AC5002775480A122B77753400C26B127EE5C202
:107AD5006A1233CF106A0512024A80EB12024A126B
:0D7AE5007D3F127E97127EF1127AF550DA85
:107AF200020259909F9E127A49121E2B12DD1BC35D
:107B020010001310010510020E80F412780B4001D0
:107B12002212793380DDD3C2AC22D227C26B7548E0
:107B22000A122B77753400127EE5C26A1233CF1027
:107B32006A0512024A80EDD26B127D3F127E9712C5
:107B42007D6775B901E5BCB2E7F5BC124EE6751664
:107B520007855917122BF080CB127DADE516601FF9
:107B620078D0E53D127B8EE53E127B8EE53F127B9F
:107B72008E765A08765F12C80E127EC3027D7E7F11
:107B82003E7E11909F7512770202DD1B75F00A840A
:107B92004430F608E5F04430F60822D26B127EC378
:107BA200127D7EE51775F01084240AF54824E8500A
:107BB2000375480A122B838558592275320012BE6A
:107BC2005E75A704900700751500127D6775B901EF
:107BD200E5BC20E705E515F0801004600D648260C5
:107BE2000975BCFF75B90575B9020515E51524209F
:107BF20050D8E58224FE4003027C96A882187F00BA
:107C020075A7007583078882E0FE75F004A4127DD3
:107C120012A9BCAABDABBEACBF1582E0FD75F004D3
:107C2200A4127D12C3E995BC404C7052EA95BD4046
:0D7C320045704BEB95BE403E7044EC95BF95
:107C3F004037703DEE75F004A404127D12A9BCAA62
:107C4F00BDABBEACBFED75F004A404127D12C3E949
:107C5F0095BC4015701BEA95BD400E7014EB95BE98
:107C6F004007700DEC95BF5008EEF00582EDF01552
:107C7F0082E5826009C3EF95825003027C0A0FC32D
:107C8F00E89F4003027C0275A70490070075C703A5
:107C9F0075C6A8E0F5BCE0F5BDE0F5BEE0F5BF7533
:107CAF00B90575B90205C6E58224204006E5C6244C
:107CBF002050E00875C70375C68075B901E5BC1281
:107CCF007CFCF5BCE5BD127CFCF5BDE5BE127CFC71
:107CDF00F5BEE5BF127CFCF5BF75B90205C6E5C65A
:107CEF00245850D6E5320470FB75A70022B4FF016B
:107CFF0022F975A704900700E582686005E06970B6
:107D0F00F7E922F5C685F0C775B901E5BC645F7068
:107D1F000375BC27E5BD645F700375BD27E5BE64C1
:107D2F005F700375BE27E5BF645F700375BF2722C1
:107D3F0075C703E54875F004A42480F5C6E55975A9
:107D4F00F00484A8F00825C6F5C675B901A9BCAA28
:077D5F00BDABBEACBF8615F1
:107D660022E515242050037515DFE51575F004A4EA
:107D760054FCF5C685F0C722E51724204028E517F0
:107D860075F00484A8F00824A8F5C675C70375B96C
:107D960001A9BCAABDABBEACBFA61589BC8ABD8B6A
:107DA600BE8CBF124EE622E4F516F51579FF127D5C
:107DB6006775B901E5BCB4FF040516A9150515E5F7
:107DC60015242050E9891579FF75C70375C6A8756E
:107DD600B90109E5BC04601B09E5BD04601509E5A8
:107DE600BE04600F09E5BF04600905C6E5C6242088
:107DF60050DD09891722751600751501127D677504
:107E0600B901E5BC20E70205160515E51524205045
:107E1600EB227900E975F004A454FCF5C685F0C799
:107E260075B901E5BC20E73078D066702B08E5BD52
:107E360066702508E5BE66701F08E5BF6670190501
:107E4600C675B90108E5BC66700E08E5BD66700822
:107E560008E5BE667002D32209E9242050B6C32283
:107E6600127E86127E6EA8017F08E0F608DFFB22EE
:0B7E7600127E86127E7EA8017F08E6C7
:107E8100F008DFFB2278D0796275A704758307EBD0
:107E9100C454F0F58222127D6778D0127EB1E5BC20
:107EA100F9C23C20E702D23C127EB17862127EB167
:107EB10075B901A6BC08A6BD08A6BE08A6BF0805DF
:107EC100C622127D6778D0127ED3127ED3786212D9
:107ED1007ED386BC0886BD0886BE0886BF08124EC2
:107EE100E605C622125A3612DEF112866E02DD1B3B
:107EF10012DEF17F007E0990A35E1277027F0A7E77
:107F010012E5150412D3817F1412C9F8121DF37FF3
:107F1100277E0875130778D0127780E6793E30E71F
:107F210002792F7E34E912D4DD7F3D7E0190A4DFFA
:107F310012773520311B3030031291A9C23B1281D7
:107F4100A1127F57D23B1281A1127F691281E88071
:107F51007C12C06480E6C23B7F44745320170274D4
:107F61004E7E0012D4DD8017D23B7F4F745720170D
:107F71000274457E0012D4DD7E06E51E12D4CA7E4F
:107F81000CE51D12D4CA7E12E51C12D4CA7E1774E8
:107F91008112D4DD7E1CE51B12D4CA7E22E51A12A1
:107FA100D4CA7E28742E302602742712D4DD7E2D89
:107FB100E51912D4CA7E33E51812D4CA7E393026A7
:0F7FC10007742C12D4D97E3BE53702D4CA742D35
:107FD000201702742B7F707E1512D4DD127FEC7E89
:107FE0003A12D32A7E0190A50A0277027E1BE51C75
:107FF00012D4CA7E21E51B12D4CA7E27E51A12D4F8
:10800000CA7E2DE51912D4CA7E33E51802D4CA12ED
:10801000808D1280B812838F127EF11283E72017B1
:108020001E10021B1248F012C80E128075121DFE9F
:108030007F347E2F12778D127F2A12DD1B80E21291
:108040001DF3203026203128C23B1281A11280CDA1
:1080500078661282A1D23B1281A11280E278691265
:1080600082A11281E812815C02834412927280F232
:1080700012C07980EDE57D75F01084AAF075F00AE4
:10808000A42A547FFA78D7E654802AF6227F277EE6
:108090000879D08700C001D224B9D002C22412844A
:1080A0006ED001A70010230909EE2406FEB9D7E31C
:1080B0002219EE24FAFE80DB7E3479D7E7A2E7921C
:1080C0001712841B79D7E7A21792E7F722C224C2BE
:1080D0003B751E007F447E0012842B801E1023ED12
:1080E000802AD23BC2247F4F7E00128433D2247E6A
:1080F00006E51E128460F51E1023E7D2247E0CE5EF
:108100001D128460F51D303BD41023E1D2247E1271
:10811000E51C128460F51C1023E17E1CE51B128413
:0381200060F51BEC
:108123001023E67E22E51A128460F51A1023E87EF6
:108133002DE519128460F5191023E87E33E5181232
:108143008460F5181023E87E393026027E3BE5373C
:10815300128460F5371023E3227F707E1512842387
:10816300C2247E1BE51C128460F51CD2247E21E50B
:108173001B128460F51B1023E77E27E51A12846027
:10818300F51A1023E67E2DE519128460F5191023E4
:10819300E87E33E518128460F5181023E82278D7B7
:1081A300E6C2E775F00A847866F537303B057869EF
:1081B30085F03712821130262BE53775F003A404BE
:1081C3000475F00584FBE51975F00AA4251875F00C
:1081D30006A42BFBE435F0FC125585F537125585C3
:1081E300F5188B1922E563FC339217AB6250031227
:1081F30055F6305C0A7AD21253717840125513AE99
:1082030004AF037C277D1012547C8F1C8037E6FD5E
:1082130033921718860418860350031255FE7A0901
:10822300792778C01255108B1EADD3ACD2AB06792B
:10823300EA786012550E8B1DAF06AED27C177D70A7
:1082430012547C8F1CAF05AE047C037DE812547C72
:0F8253008F1BAF05AE047C007D6412547C8F1A24
:10826200ED75F00A84F51985F01822EC3392175057
:10827200031255F6751D30301786751D2D808178D5
:10828200427B607CEA800678407B207C4E12C144AF
:108292007927781012550E8B1CAF06AED280AB3008
:1082A200262AE51975F00AA4251875F00AA42537BF
:1082B200FBE435F0FC7A051253638C068B077C00D5
:1082C2007D0312546F8E048F031281DBE51E75F05D
:1082D2000AA4251D75F00AA4251C75F006A4251B09
:1082E200FBE435F0FC7A0A125363EB251AFBE43CFB
:1082F200FC7A0A125371EB2519FBE43CFCE43DFDC8
:108302007A0A125383EB2518FBE43CFCE43DFD3072
:1083120017031255FEA60518A60418A60378D7E679
:10832200A2E7923DC2E775F00A84FCABF0303B0E47
:10833200AB37EC75F00AA42BA23D92E7F622AC37DC
:1083420080F012835F305C0A7A4012537178D21245
:1083520055133017031255F68C638B622212836F0A
:108362007A0A125363EB2518FBE43CFC22E51C75E8
:08837200F00AA4251B75F00AB6
:10837A00A4251AFBE435F0FC7A0A125363EB25199B
:10838A00FBE43CFC221283C112DE03C202C22312A6
:10839A0083C110000810010510021B80F51031ED91
:1083AA0010300D102604D22680E3D230C23180DD8F
:1083BA00D231C23080D7227F3590A4C81277339049
:1083CA00A4E620300F90A50220310990A4D72026D8
:1083DA000390A4CF1F7E1712770202DD1B7F357E22
:1083EA0001909F521277357F347E3A128510744E6F
:1083FA0012D4DD12DD1B12DE03C2027F347E3AD2B2
:10840A001775115975124E802675112E751227800F
:10841A001E75113E75122F801675112B75122D803F
:10842A000E75114E75125380067511457512571245
:10843A008510E511301702E51212D4DD12DD1B108A
:10844A00000810010510020B80F5D23C1017E3D288
:10845A001780DF02850B4430F812846AE8540F2231
:10846A00C2218002D221A22492229223128510E8EC
:10847A0030E709D23C7430302102745FF812D4DD3F
:10848A0012DD1B10003410010510025D80F5D23C8C
:10849A00102266102367B43909745F2021DF743013
:1084AA0080DBB45F04742D80D4B42D04744180CD74
:1084BA00B45A04743080C60480C3D23C30240610F7
:0F84CA002237102338B44104742D80B1B42D042F
:1084D900745F80AAB45F04743980A3B43009745AF4
:1084E90020219B74398097148094B48908D223E899
:1084F90012D4DD800DF8C223800874898001E80256
:1085090084879085258003908521C007EF2408FF83
:1085190012D509D00702DD1B0205F8F80205000093
:10DCBB0075A70090DCED75F02D84C2D5C2D160172D
:10DCCB00D2D1146007D2D514600DC2D1E5F093FC0C
:10DCDB00742D95F093FB22E5F093FB742D95F09347
:10DCEB00FC220009121B242C353E474F58606870EC
:10DCFB007880888F969DA4ABB2B8BEC4CACFD4D956
:10DD0B00DEE2E6EAEDF0F3F6F8FAFCFDFEFFFFFFCC
:10DDB500D23D8002C23DED8BF0A430E70205F0C3F1
:10DDC500E895F020D50425F025F0FEED8CF0A43083
:10DDD500E70205F0C3E995F030D10425F025F0FF01
:10DDE500203D0B2487500122EF24CC40012202DE86
:01DDF50036F7
:10D75900203A7A7E1C7F5312DE367F5912DE361E3E
:10D769007F5712DE367F5512DE367E2312DE367F74
:10D779005712DE361E7F5912DE367F5312DE361FF0
:10D789007E2012DE367F5A12DE367E1E12DE367F8C
:10D799005212DE36120E67E5BD20E0143006117F05
:10D7A900357E1C90D815E571700390D81F02D509F4
:10D7B900E5716018E57012DCBB781F79567D091296
:10D7C900DDB9303A0312D7E80DBD16F3227E1C7F6E
:10D7D9005390D7FE12D509200CD612CA5480C0C066
:10D7E900060E30D5021E1E12DE36D0061F30D102BB
:10D7F9000F0F02DE36070700386C446C3800050548
:10D809002070D8702005057088A88870080710381E
:10D819007CFE383838000807102844C62828380004
:10C8330090A5147F717E23127735120E67E5BC7EB7
:10C843003112D49830121AC23C120E67E5BCFB7544
:10C85300F00AA4F904FAC23D12BE4A12CAD1303D0D
:10C863000122DAF712C9D87C00EBF4042E4019AD8B
:10C873000312546FEFA2D1203C077E237F6502D0C1
:10C88300F7AE16AF1702C979AD0112546FEF12D18B
:10C89300E5203C077E237F6502D11BAE16AF17024E
:10C8A300C99D7F567E0512CA047F3D12CA177F6F4A
:10C8B30012CA1712CA547E0A7F4112CA877E227F88
:10C8C3005912CA872012012212BE4A857A1D855E3B
:10C8D3001C857B1B855F1A7AC0C23D12CACD203DE1
:10C8E3005212C9D87C007D1412546F74562F20D174
:10C8F300029F9FFF24CB40028037EF2488500280A1
:10C9030030EA1475F00384FE12DE36C3E51B957B13
:10C91300FEE51A955F92D55004EEF404FEEEC313C0
:10C92300FE24E0400C741F2E30D5029E9EFE12DEC4
:10C9330036DAA8227F5212C9497F5A12C94975179C
:10C9430053751600802B7E0012DE660EBE12F9228E
:10C953007F157E28742012D4DD7F1C7E2812DE66AC
:04C963000EBE40F9CB
:10C96700223012E712C95375171575162DD23C02DE
:10C97700C84CC23D6002D23D92D175F080305C0454
:10C98700F5F08001A4A2E792D5E5F075F03284F8BE
:10C99700E5F075F00584C0E0E5F0A2D533C0E0E826
:10C9A700601E12D4CAEE2406FED0E0F8D0E012D4FE
:10C9B700CAEE2406FE742C12D4DD0E0EE802D4CA89
:10C9C7007420303D07742B20D102742D12D4DD80E2
:10C9D700D4C3ED957AFFEC955EFE92D150031255C4
:10C9E700E6227F1512C9F07F327E3E12DE36DEFB6D
:10C9F700227E0912DE360EBE36F9227E0112DE369F
:10CA07000E0EBE3FF8227E3312DE360EBE40F922EE
:10CA17007E047D1112DE360E0E0EDDF81F1F7E35E9
:10CA270090A51D305C057E3190A5210277357405F0
:10CA3700305C097E32740112D49874067E3612D4A3
:10CA4700987E3A740012D4987E3D02D4987F417E36
:10CA57001F7D0F12DE360F0F0FDDF8227F687D0373
:10CA670080047F677D0512DE360FDDFA227F667D43
:10CA77000780F37E1F7F5012DE361F1FBF3EF8224E
:07CA87007D0A12DE360E0EDF
:10CA8E000F0FDDF722203D07123C767003D23D22B8
:10CA9E00056D12BC10E4F5F7C2B2C2B2ABF7F5F7F2
:10CAAE00C2B2C2B2E5F7FA30E411EB251DF51DE472
:10CABE00351CF51C0519EA30E3010ED2B28015784B
:10CACE000380027801203D07123C767003D23D228E
:10CADE00D8F3056DE56D2409F56D12BC10E4F5F77C
:10CAEE00C2B2C2B2ADF7F5F7C2B2C2B285F71BF54C
:10CAFE00F7C2B2C2B2E5F7FCD2B2543F30E50244FF
:0FCB0E00C0CC54C02323F51AE56D24F6F56D2233
:10D680007E017F0990D6FE12D5092051097E037FC5
:10D6900000743F02D4DDE4FEFFC3E54512CF4FFD29
:10D6A000940AED403D9464ED4002746312D37B7E96
:10D6B000017F09E552240575F02D84AAF075F00567
:10D6C000A4CA75F00B842A90D6E99312DCBBBCB8CF
:10D6D000027BB87D04EE2DF8EF2DF90D12DDB5DDDE
:10D6E000FB227E0312D4CA80C6000C1622222D39DA
:10D6F000444F4F5A66707C7C87939EA9A900090904
:10D700000800410000000000888000000000410087
:10D710000800120E7BE5BCB4F8339004C3E0602C23
:10D72000FA24F340277F137E0012DE360F0F12DE3D
:10D73000360E12DE661F1F12DE660EDAEC7F147ED6
:10D740000012DE360E12DE660EBE12F5229005CCF9
:09D75000E0C3941240F60480C706
:10CF4F00305D0A75F08AA42480E5F0340022207445
:10CF5F00157F017E1190CFD712D5097F0A7E0AE582
:10CF6F002E540702D3927F087E1190CFE712D50976
:10CF7F0020730C7F0A7E1712DE660E0E12DE667F9E
:10CF8F00007E0BE57112CF4F12D3817F0C7E11E51E
:10CF9F0071602F0EE57064B4602864B475F032844C
:10CFAF00C0F012D4C3CE2405CED0E075F00584C0F6
:10CFBF00F012D4C3CE2405CED0E023302D010402CD
:10CFCF00D4C390886A027702070FFFFFC473BDAF07
:10CFDF00A463B5FBCDE7FFFF030F0100FFFE038046
:10CFEF00306701227F357E00748812D4DDE55160F1
:10CFFF001712CF4F75F06484F87E06E5F012D3E078
:10D00F00E860E07E0002D4CA7E003074D63073161A
:10D01F0079BCE7FC09E7FB12530B781D201704E6D8
:10D02F0070011802D2AB909CB0027702202C012223
:10D03F0090D04502D509050EFFF0E01CF004F81C56
:10D04F00FFF0301201227F637E00909CC712D5093A
:10D05F007F1512C9F07F1F12C9F07F2912C9F07F07
:10D06F00177E06E53F30E00B90A531305C0390A5AD
:10D07F004580132074077E01909CE7800990A526B8
:10D08F00305D0390A53B127702307306E54E6002C8
:10D09F00154E205718E54EB40113120E8AC3E55CE6
:0DD0AF009560F5BCE55D9561F5BD124EE69E
:10D0BC007F217E01E53F30E021305705909E0C80AA
:10D0CC0016E54E7005909E18800D909CF312770219
:0BD0DC007E30E54E02D3E61277022200
:10D24D0012530B7F207E05751900781DC2D5E6306F
:10D25D00D51712D4C3EE2405FE18B818F17E1F742D
:10D26D0063305C02748202D4DD7005B8191880E257
:10D27D00D2D5CE24FACE7484301702742D12D4DD9B
:10D28D00EE2406FE80C8742012D4D980C8781C8084
:10D29D000D7F007E23AC5EAB7A12530B781DC2D589
:10D2AD00E630D50C12D4CAEE2406FE18B818F122B9
:10D2BD007005B8191680EDD2D53017E4CE24FACE0C
:10D2CD00742D12D4DDEE2406FE80D5742012D4DD2B
:10D2DD0080D512530B781DC2D5E630D51612D498D1
:10D2ED00EE2404FE18B818F10E745E305C0274273B
:10D2FD0002D4A77005B8191680E3D2D53017DACE4F
:10D30D0024FCCE742D12D4ABEE2404FE80CB7420FD
:10D31D0012D4AB80CBC23D12D3350F0F0E0E7463FA
:10D32D00305C02748202D4DD12530B781DC2D5E637
:10D33D0030D50C12D4F8EE2408FE18B818F122706E
:10D34D0005B8191680EDD2D5301716740BCE24F80A
:10D35D00CE12D4F8EE2408FE80D5740C12D4F880C9
:08D36D00D5303DCB740A80E5C8
:10D829007F797E24E55F30E70122AC5F1CAB7B1278
:10D839005339E51B700E742012D4DDEE2405FE1257
:10D84900D877800C12D877E51B12D4C3EE2405FED5
:10D85900E51A12D4C3EE2405FE742C12D4DD0E0E83
:10D86900E51912D4C3EE2405FE745E02D4DD742DCD
:10D87900201702742B12D4DDEE2406FE22E55F3058
:10D88900E70122AC5F1CAB7B125339E51B700E74A8
:10D899002012D4ABEE2404FE12D8D0800C12D8D0BA
:10D8A900E51B12D498EE2404FEE51A12D498EE244E
:10D8B90004FE742C12D4AB0E0EE51912D498EE2482
:10D8C90004FE742A02D4AB742D201702742B12D4CF
:06D8D900ABEE2404FE2268
:10D0E7007F097E2530040512D1E18028A275E579F4
:10D0F700C23D6002D23D92D175F080305C04F5F0FC
:10D107008001A4A2E792D5E5F075F03284F8E5F046
:10D1170075F00584C0E0E5F0A2D533C0E0E8602AE9
:10D1270012D4F8EE2408FED0E0F8D0E012D4F8EEDE
:10D137002408FE0F0FE52B5403701F746012D4DD13
:10D147001F1FEE2404FEE802D4F8740C303D067469
:10D157000A20D1010412D4F880C9205904742E8002
:10D16700DC205804747F80D5748080D13004051288
:10D17700D1E18028A275E579C23D6002D23D92D106
:10D1870075F080305C04F5F08001A4A2E792D5E544
:10D19700F075F03284F8E5F075F00584C0E0E5F04D
:10D1A700A2D533C0E07F3E7E1CE8602012D559D05F
:10D1B700E0F8D0E07F3E7E2812D5597F447E327456
:10D1C7002E12D4DD7F3E7E37E802D559303DE0741C
:10D1D7000A20D1010412D55980D59005CAE075F00F
:10D1E7000A84F8E4C5F0C2D522301105E54AB40235
:10D1F70050C39006E9E0957AFB9006E8E0955EFC5F
:06D2070050031255F6EC85
:10D20D00C31360047B63800FEB13FB249C40F52458
:10D21D004F4004C20480079005CAEBF0D20490067B
:10D22D00E6E09006E8F09006E7E09006E9F0E55EAE
:10D23D009006E6F0E57A9006E7F02212D22B80DE1A
:10CB1D00E54424F64001227800E552206607C395CE
:10CB2D0070500224B40475F00384F9E928FE24C47E
:10CB3D005001FE12CB5F12CB6B1E12DE36C3E9988D
:10CB4D00FE5003243CFE12CB5F1E12DE3608B81FCA
:10CB5D00DA22EE2420FE24C250032402FE22E82411
:10CB6D00F1E8C2D55006D2D5E8F4241F23FF90CBAF
:10CB7D00ED93CF0493FAE545F5F0A4ACF0FB125319
:10CB8D009AE544F5F0A49BFBE5F09CFCEB2420FB1F
:10CB9D00EC3400FC12CBCEFAE5458FF0A430E70261
:10CBAD0005F0E5F020D502F4042A75F005201903EF
:10CBBD0075F00384FF24DF50027F20C374329FFF82
:10CBCD0022EC24F0500BEB2460EC340090CC3D9320
:10CBDD0022EB33FBEC33FCEB33EC3390CC0D932297
:10CBED00FF00FF03FA0BF318EA2ADE40CF58BE739D
:10CBFD00AB8D96A880C068D64FE835F51BFD00FFBC
:10CC0D0000080B0E101214151718191B1C1D1E1FD2
:10CC1D0020212223242526262728292A2A2B2C2D9C
:10CC2D002D2E2F2F303131323333343435363637D4
:10CC3D00373839393A3A3B3B3C3C3D3D3E3E3F3F30
:10CC4D004042444648494B4D4E5052535556585903
:10CC5D005B5C5D5F60616364656668696A6B6D6E80
:10CC6D006F7071727374767778797A7B7C7D7E7F45
:10CC7D00808182838485868788898A8B8B8C8D8E33
:10CC8D008F9091929394949596979899999A9B9C3D
:10CC9D009D9E9E9FA0A1A2A2A3A4A5A6A6A7A8A95A
:10CCAD00A9AAABACACADAEAFAFB0B1B1B2B3B4B489
:10CCBD00B5B6B6B7B8B9B9BABBBBBCBDBDBEBFBFC3
:10CCCD00C0C1C1C2C3C3C4C5C5C6C7C7C8C8C9CA08
:10CCDD00CACBCCCCCDCECECFCFD0D1D1D2D2D3D456
:10CCED00D4D5D5D6D7D7D8D8D9DADADBDBDCDDDDAC
:10CCFD00DEDEDFDFE0E1E1E2E2E3E3E4E5E5E6E607
:10CD0D00E7E7E8E8E9EAEAEBEBECECEDEDEEEEEF68
:10CD1D00EFF0F1F1F2F2F3F3F4F4F5F5F6F6F7F7CF
:10CD2D00F8F8F9F9FAFAFBFBFCFCFDFDFEFEFFFF3E
:10CD3D00E54524FD400122E552206607C39570505C
:10CD4D000224B40475F00384241FFE24C25003246E
:01CD5D0002D3
:10CD5E00FE12CD98EEFD241EFE24C250032402FEC8
:10CD6E0012CD98E544240275F00520190375F003E1
:10CD7E0084F4042432FF24EE500F12CD8DAE051E26
:10CD8E001E7C0512DE360EDCFA227F1512DE360F01
:05CD9E000FBF2DF8227B
:10D598007E00206615E5700475F0B484E5F075F03A
:10D5A8000384FE6004C3743C9EFE745312D5C37496
:10D5B8005712D5C3744E12D5C374457F2F12D4ABFE
:10D5C800BE00077E3C12D4AB7E00EE240875F03C0A
:10D5D80084AEF00F0F0F12DE360E12DE360F12DE9B
:10D5E800361E12DE36EE240775F03C84AEF022308B
:10D5F800745C301259E54AB4040122B4060122E5EC
:10D608007112CBB78F057C037E1E30662AE5700445
:10D6180075F00384241EFE24C6501C24FB500424E9
:10D62800038013C00612D63FD0E024C67C016006F2
:10D638000C1460020C14FE12D64B0EEE24C14002EC
:10D64800DCF5228D0712DE360FEF24CE50F722E5E7
:10D6580053206607C39570500224B40475F0038400
:10D66800241FFE24C250032402FE12D6760E7F2306
:08D6780012DE360FBF2DF9226E
:10DD6C00AF177E00E53C12D3757E0C742E12D4DDF9
:10DD7C007E12E53B12D3757E1E742E12D4DD7E24EA
:10DD8C00E53A02D3757E0E78ADE612D3E07E1874B8
:10DD9C002C12D4DD7E1B18E612D3E07E25742C12D7
:09DDAC00D4DD7E2818E602D3E064
:10CDA3007F797E00E54012D3E07E0A743B12D4D92A
:10CDB3007E0CE54102D3E07F797E16743B12D4D911
:10CDC3007E18E53F12D3E07F797E0078AEE612D37A
:10CDD300E07E0A743B12D4D97E0CE53E02D3E030E8
:10CDE3005EE52043E27F6D7E0078AEE612D3E07EFF
:10CDF3000A743B12D4D97E0CE53E12D3E07F757ED4
:10CE03000075F00A84E5F012D4F80F0F7E08743A27
:10CE130012D4D91F1F7E0DE53F75F00A84C0F012AE
:10CE2300D4F8EE2408FED0E002D4F8851C1E851B3E
:10CE33001FAB1BAC1C305D0A7A1B12537178321284
:10CE43005513C3EB33FBEC33FC923D125342303D9D
:10CE5300087409F51DF51CF51B7F75E51D60157E2E
:10CE63002412D4F87E2CE51C12D4F87E34E51B1270
:10CE7300D4F8803D7E22E51C601912D4F87E2AE5A1
:10CE83001B12D4F87F787E31742E12D4D97F75E5C6
:10CE93001A8019E51B12D4F87F787E29742E12D4D8
:10CEA300D97F757E2DE51A12D4F8E5197E3512D493
:10CEB300F87F777E3C125CCC851E1C851F1B227F6E
:10CEC300397E1F12DE360FBF40F9781F79567A007C
:10CED3007D1A12DCBB12DDB9EA2406FABAAEF37886
:01CEE3001B33
:10CEE400C3E5119570500224B4FA604214603E14F4
:10CEF400603A2450603A146036EA24A540278A1E1A
:10CF0400751D007D1912CF140D30740312CF140D4A
:10CF1400781F7956AA1DEA12DCBB12DDB90AD3EADE
:10CF2400951E40F2228A1D751EB380D70808080892
:10CF34007F367E1C90D815E571700390D81F12D5EA
:0BCF4400097F3CAE0090852102D5095A
:10DA3C00787512DA8C7453201702744E207406E534
:10DA4C002E54074430AF1712DAB67E3BE57DC45432
:10DA5C000F12D4CA2074077E07742012D4DD787894
:10DA6C0012DA8CE5172409FF74572017027445202D
:10DA7C007402742012DAB67E3BE57D540F02D4CAD0
:10DA8C00E6FD3392171886041886033017031255D7
:10DA9C00FE7917787012550E8B13AF06AED27C0040
:10DAAC007D6412547C8F148D15227E0012D4DD7E81
:10DABC0007E51312D3927E19748112D4DD7E20E512
:10DACC001412D3757E2B742E2073030E742C12D467
:08DADC00DD7E2FE51502D37574
:10DC4B00E54A602E7A2420E00E7A26141460087AB6
:10DC5B0028141460027A297F667E01EA12D4DD2033
:10DC6B005505205406800B745B8002745C7E001299
:10DC7B00D4DD20110778A9B60007802130261EC2FB
:10DC8B0026909D867F681276F07F66A85AE54AB487
:10DC9B00060108E875F06484E5F012CE1C20080F2D
:10DCAB00E537640260097F367E2E744112D4AB22B5
:10D8DF0020144F740512DEDDEF33EE33F9EF03033F
:10D8EF00541FF5F090D932E993A4C5F013C5F01386
:10D8FF00C5F013C5F013C5F0135403FCE5F013FB8B
:10D90F00E9242093C9244093C39BC4540FFBE99C83
:10D91F00C4FC540FF9EC54F02B2446F57BE934F694
:10D92F00F55F22FFFFFFFFFFE6C5AD9C8F857D777B
:10D93F00726E6C6A696A6A6C6F747A828D9DB4D9E3
:10D94F00FFFFFFFAE9DCD3CEC9C6C3C0BEBBB9B770
:10D95F00B5B4B2B0AFADABAAA8A6A4A2A09E9C9935
:10D96F0096918C00381CE735D137246F00C5B3C1B1
:10D97F00E61F66B60E68C21867AADBF4EDB94675E6
:03D98F0010A200E3
:10DEBD00D2A27408D2A1D2A300C2A3C2A1D2A30040
:10DECD00C2A3D5E0EF7405D2A300C2A3D5E0F8221A
:10DE9600C2A3D2A2D2A1D2A300C2A375F008339224
:10DEA600A1D2A300C2A3D5F0F5C2A175F003D2A3F7
:07DEB60000C2A3D5F0F82221
:10C44D0012DE96D2A300C2A3C2A175F008E4D2A356
:10C45D0000C2A3A2A233D5F0F5FE75F008E4D2A375
:10C46D0000C2A3A2A233D5F0F5FFD2A300C2A3222E
:10C47D00E478806608B88BFB70012274D512C44D28
:10C48D007881C3EE13FEEF13F692D118EE2460F609
:10C49D0074D612C44D7888EF33CE33CE33CE33CE2F
:10C4AD0033A2D192E25407FCEEFB7A08125363ECEF
:10C4BD00244FF608EBF674D912C44DEF543F788231
:10C4CD00F67886EF33CE33CE33CE33CE335403F6F8
:10C4DD0008EEF618161608E6C4FF54F0F618E6C472
:10C4ED00CF540F2FF674DA12C44DEF232354FC787A
:10C4FD0083F67884EEF608EF54C0F67880E466088B
:10C50D00B88AFBF62212C4557889C3EF96FF18EE50
:08C51D0096FEA2E792165010F1
:10C525001255E6740FF8F91253B0EF2CFFEE3DFEED
:10C53500788BEEF608EFF622E6182016072CF7E6BC
:10C545003D19F722C39CF7E69D80F66A405E80564A
:10C55500E050F04B0044803DC0384031D02BA02541
:10C56500601F2018D014000F000AA00144015801D3
:10C57500680178018801A001B401D001EC02100224
:10C5850038026802A002DA030C034D78BE802085CC
:10C595008E8A9D8F4D95BA9A97A0BEA631AC53B29F
:10C5A5002AB801BD6AC1EDC4D1C78812C455788DBA
:10C5B500EEF608EFF67887798C1253B07883799088
:10C5C50012C53D7885798C1253B07881799212C560
:10C5D5003D788DE624E4FE08E63392D13392D554B6
:10C5E500FCFFEEA2D133A2D533FE780F7992125318
:10C5F500B078947990C3EC97F61819ED97F679947D
:10C6050090C5507F1F7D11EF93C3971F19EF939727
:10C615001F091DED600240EF0F90C570798DEF93F6
:10C62500F7090FEF93F7788E79941253B090C59070
:10C63500EF93C39BFB1FEF939C2420FC7897E62B7D
:10C64500F618E63CF618E436F6740612DEDDD23747
:09C65500EE24F740062402500215
:10C65E00C237EEFCEFFD740712DEDDC3ED9FFFEC7B
:10C66E009EFE78B7E6FD337C0050011CEF2DFFEEE9
:10C67E003CFE789CEF26F618EE36F6222014122099
:10C68E00370F789DE6B4050912C74212C77712C755
:10C69E00C02220145E7897799A12C7F112556EC394
:10C6AE00EE9420FE924550031255E67C007D051255
:10C6BE00547C3045031255E6E531B40C3612DA22BD
:10C6CE00120E80E5BC2FF560E5BD3EF56120E71149
:10C6DE0024F8500DFAC3E5609AF560E5619400F513
:10C6EE0061120E8AE5BC2560F57AE5BD3561F55E11
:10C6FE0012DA2F7897799AC3E697FB1819E697FC0A
:10C70E007A0212536330370B7A02125363ECFEEB4C
:10C71E00FF800312C74212C77720140312C7C078D6
:10C72E00957998E6F776000809E6F776000809E6A7
:10C73E00F7760022799CE77700FB19E77700FC7803
:0CC74E009DE6B40506EB33FBEC33FCEC7D
:10C75A00A2E792D550031255F67A32125371ECFBC6
:10C76A00EDFC30D5031255F6ECFEEBFF22EE240861
:10C77A00FE74042037167406307511789DE6B405E8
:10C78A0004740C8007F42406C323540FFD7C0012A2
:10C79A00534F789FE6FC08E6FBC374109DFA1253C8
:10C7AA0071EFF8EEF912556EE878A02FF6FF18EE41
:10C7BA0039F62480FE22927540031255E678BBE6CC
:10C7CA00F5F02438400375F0E1EF33EE3378A8F63C
:10C7DA00A485F07930E7020579C276307508E579E3
:10C7EA0024F15002D27622E627FB1819E637FC1804
:10C7FA0019E637FD2212BDF17F087871793A12C81D
:10C80A001A024ABB855E63857A62787379647F0609
:10C81A00E6F70809DFFA227864797380F178737988
:09C82A00AF80EB78AF797380E573
:1052E900E4FEFFFC7D0A791DE7540F2FFFE43EFE23
:1052F900B9190280061912534F80ED301703125560
:10530900E622305C2BEC33921750031255F6EC244D
:10531900D950047C277B007AD2125371EB33CC33FA
:10532900CD33CC33ED33FBEC33FC3017031255F698
:10533900EC33921750031255F67919125585F7096E
:10534900B91DF8A70322EFF88DF0A4FFEDC5F0CE43
:10535900A42EFEEC88F0A42EFE22EB8AF0A4FBE535
:10536900F0CC8AF0A42CFC22EB8AF0A4FBE5F0CC6B
:105379008AF0A42CFCE435F0FD22EB8AF0A4FBE5CD
:10538900F0CC8AF0A42CFCE435F0CD8AF0A42DFDF4
:1053990022EB8AF0A430E70205F0E5F0CC8AF0A40C
:1053A9002CFBE435F0FC2286F0E7FDA4FAABF019FA
:0653B900E786F0A42BFBC7
:1053BF00E435F0FC18E68DF0A42BFBEC35F0FCE4A3
:1053CF0033FDE687F0A42CFCED35F0FD22EB89F0E0
:1053DF00A4CBAEF08AF0A42EFEE5F03400FDEC89EC
:1053EF00F0A42EFEE5F03DFDE433CC8AF0A42DFDB4
:1053FF00E5F03CCEFC22EB89F0A4CBAFF08AF0A411
:10540F002FFFE5F03400FEEC89F0A42FFFE5F03E0E
:10541F00FEE433CC8AF0A42EFEE5F03CFCED89F0DF
:10542F00A42EFEE5F03CFCE433CD8AF0A42CFCE581
:10543F00F03D8E058C068F04FF22C2D5EC30E705B8
:10544F00B2D51255EEEE30E70DB2D51255E6125425
:10545F007C1255EE800312547C30D5031255E62290
:10546F00C3EC13C0E0ED132FFFD0E03EFEBC000BEA
:10547F00BE0029EF8DF084FFADF022E4CCF975F07A
:04548F0008EF2FFFF4
:10549300EE33FEEC33FCEE9DEC994005FCEE9DFEF5
:1054A3000FD5F0E9E4CEFD22EDF9F5F0EE8420D23C
:1054B3001CFEADF075F008EF2FFFED33FD400799AB
:1054C3005006D5F0F222C399FD0FD5F0EA22EC3352
:1054D300EE3400FEEF3400FF7D007A007900780996
:1054E300C3ED9AFDEE9BFEEF9CFFB392D54009ED11
:1054F3002AFDEE3BFEEF3CFFA2D5E933F9ED33FD88
:10550300EE33FEEF33FFD8D92279007A00C380153A
:1055130079007A00C3EA13FFE913FEE8132BFBEECD
:105523003CFCEF3DFDE4F5D2F5D333FE7F19C3EE2A
:1055330098FEE5D299F5D2E5D39AF5D3B392D54047
:105543000DEE28FEE5D239F5D2E5D33AF5D3A2D54F
:02555300EB3338
:10555500FBEC33FCED33FDDF0122EE33FEE5D23308
:10556500F5D2E5D333F5D380C3EDC454F0FEECC4D6
:10557500FF540F2EFEEF54F0FFEBC4540F2FFF2204
:10558500EC75F00A84FCEB54F025F0C475F00A8440
:10559500C4CBC454F025F0C475F00A842BFBE5F0A8
:1055A50022AC10AB11125585A904AD03FA7C197B09
:1055B50099125363AE04AF03EA75F006A4F8AC1272
:1055C500AB131255852875F00A8485F014F8EF2B76
:1055D500FFEE3CFEEF28FFE43EFEE43DFDE439FC32
:1055E50022C3E49FFFE49EFE22E4C39DFDE49CFCF0
:1055F50022C3E49BFBE49CFC22C3E49BFBE49CFCF0
:10560500E49DFD2275D4107B807A0079807800EACC
:0A561500F5F0A4FCADF0EBF5F0A4F5
:10561F00FEAFF0EB8AF0A4C333C5F033C5F092D5DB
:10562F002DFDC5F03EFEE430D501043FFFB5150D4D
:10563F00EEB51409EDB51305ECB51201224006EADB
:10564F0098FAEB99FBD5D40ABB0001220ABA0001E4
:10565F000B22C3E913F9E813F8EA28FAEB39FB80B8
:10566F00A478087B807D807C00EDF5F0A4FAE5F04E
:10567F008EF0B5F007EA8FF0B5F001224003ED9BF5
:10568F00FDD827BDFF0122EDF5F0A4F9A8F0ED0438
:10569F00F5F0A4C399FAE5F09813CA1329F9E83A7B
:1056AF00F8C3E99FE89E50010D22C3EB13FBED2BCE
:1056BF00FD80B6C374689511FB74019510FC8004CE
:1056CF00AC10AB117A0B79B81253DC80177473F8E6
:1056DF00F9E627FB0809E637FC0809E637FD30E74E
:0556EF00031255FEEB63
:1056F40033FBEC33FCED3323FD242083F8ED241C31
:1057040083FFED241883FAED241483F9EF99F9E863
:105714009AFA1253DCEF9DFFE89EFE22FFFFFFB6CC
:10572400FED7FD63FB5DF8C4F59BF1E3ED9EE8CF86
:10573400E379DD9ED743D06BC919C153B91CB07945
:10574400A7709E06943F8A237FB674FF6A045ECBDB
:10575400535B47BB3BF1300423FB17DE0BB2FF80E6
:10576400C21DC232532CF8C3E5679576FBE56895F4
:1057740077FCE5699578FD30E705D2611255FE2482
:10578400F05003125838AA06A907125405EC2480D5
:10579400E43DFBF9F51AE43EFCFAF519E43F600236
:1057A400D2321253DC8B128C138D148E15C3E56424
:1057B4009573FBE5659574FCE5669575FD30E70525
:1057C400D2621255FEEBF9F51FECFAF51DED6002FD
:1057D400D232303201221253DCEB2512F512EC35B1
:1057E40013F513ED3514F514EE3515F51540E102F6
:1057F400560912576420323BEB242E40D3EA24018D
:10580400CB3400FC7A07793D1253DCC010C0118EF2
:10581400108D118C128B13E4FCFD7E077FD012B522
:0E58240058851203851302D011D010BB000569
:10583200BA0002D21D22B261C374809BFB74F59C34
:10584200FC74209DFD22204D69204866303F637F15
:10585200697E0112CA047E1F12CA7475A7009004E1
:10586200EDE0A2E792171392E7FC1582E013FB30FA
:1058720017031255F6BC003AEB603720E73420E6F6
:105882003110E513201707C3741F9BFE80027E1F91
:1058920012CA690EDBFA22FB2017097E00C37420AC
:1058A2009BFB8008EB241FFE74209BFB12CA630E35
:1058B200DBFA2275A700758307E559C4440FF58208
:1058C200E0A2E792522212C8271258B5C2E775F039
:1058D2000A84FEAFF075A7045382F1786412593E30
:1058E200AE07786712593E75A700E57DC4540FFED6
:1058F200E57D540FFF7873125932AE07787612594C
:105902003274AF1256DE1257F68B148A1312092024
:10591200ACCCAB017A0A125363E5139B9004ECF012
:10592200FBA3E5149CF0FCA2E7923DD23F02C82DF6
:10593200860308860408860518188006E0FBE0FC4A
:0A594200E0FD7A0A12538320E70CFF
:10594C00EB2EF608E43CF608E43DF622C3EB9EF69B
:10595C0008EC9400F608ED9400F622204D0920483E
:10596C0006C23F302A0522C23380F6E54824F640B1
:10597C00F5E5580460F075A700758307E559C42454
:10598C0008F582E0FEA3E0FF1209207437125A2AB0
:10599C00500B30381BC23878C586468013743212CF
:1059AC005A2A400C203809D23878C5A646754600CC
:1059BC00740D125A2A404A1258C8303D3820112210
:1059CC00204D1F20481C204019BCFF16EB243250E0
:1059DC0011D240120E62E5BF75F019A4F536D22E25
:1059EC00D22F205238E55965586032204D2F20486F
:1059FC002CD2338028201109204D062048037536FF
:105A0C0000303319204D1220480F1291460559C30E
:105A1C00E55895595003855859C233C2402229FB89
:105A2C00E435CCFCC3EB9FEC9E22E558B4FF01227D
:105A3C0085581175A704758307E54824F650028034
:105A4C005C201259202905202A02805112C827E413
:105A5C00F516F517751000125AC2E510700312C82E
:0B5A6C0021125ADB302910E51B251722
:105A7700F517F51BE51C3516F516F51C125AE81235
:105A8700C8210510C3E511951050D175A70002C8AC
:105A97002DE55AF51124F6500375110A75A70475FB
:105AA7008306751000125AC2125ADB125AE8051003
:105AB700C3E511951050EE75A70022E510C4F582D5
:105AC700E0E0F564E0F565E0F566E0F567E0F568C8
:105AD700E0F5692275A701125ED4123ED775A704B7
:105AE70022E9F0E51CF0E51BF022E510C454F0F5BF
:105AF70082E0F512E5822406F582E0F511E0F51C57
:105B0700E0F51B22E512B426157F757E34740D125D
:105B1700D4F820442575110012CEC2025C397F6D7E
:105B27007E3BE012D4DDE5137E3512D4DDE5127E2F
:105B37002F12D4DD20440312CEC212CE2E025C39BE
:105B4700202852E558B4FF012275A704758307E59D
:105B570059F51030330965586005204802051012C1
:105B67005AF1E0F513305E07204304E5376095E00E
:105B77007F797E3D12D4ABE5137E3912D4ABE512A3
:105B87007E3512D4AB30480B7F7F7E3512DE360E62
:105B9700BE40F980392012012275A7047583068556
:105BA7005B10125AF1305E0A204307E53770030293
:025BB7005D5B34
:105BB900E512700B7E3A7F79745D12D4DD800D7524
:105BC900F06484E5F07E397F7A12D42DE537B4028A
:105BD90005128FDE8045B403028040E51C7006E59E
:105BE9001B24FB5036E511F964B4602F20062CE51F
:105BF90037600D200C0AC3E99570F9500324B4F9F4
:105C0900E912DCBB781D79547D1D90D807E53F204A
:105C1900E00390D80E12DDB912D5097517797516FA
:105C29001930280375161DE51264266003125C7C81
:105C390075A7009006E3E511F0A3120E7BE5BC758C
:105C4900F01970040475F014A4951BFBE5F0951C7C
:105C5900FC922450031255F6ECF0A3EBF0C24FC2AC
:105C690063EC700EEB24E64002D24FEB24C84002ED
:105C7900D26322E51C24ED402BAE1CAF1B125E9EA5
:105C89007C007D3212547CC005EFAF17AE1612D3DB
:105C9900E6CE2405CE742C12D4DD0E0ED0E02312EC
:105CA900D3E0801B125E95125CD6CE2405CE742CEF
:105CB90012D4DDCE2402CEE875F0058412D4C3CE09
:105CC9002404CE7422305D02748302D4D9EE243DBB
:0D5CD90050047EC37F4B7C017DF412547C8F
:105CE600C004C005EF6007AF17AE1612D3E6D007A3
:105CF600D0067C007D3212547CA805EFAF17AE1695
:105D0600CE240ACE02D4C3125E95EE2450305D0333
:105D1600EE24A150047EC37F4B7C017DF412547C9B
:105D2600C004C005EF6007AF177E2F12D433D0072B
:105D3600D0067C007D3212547CC005EFAF177E374B
:105D460012D4987E3B742C12D4AB7E3DD0E075F015
:105D5600058402D4987F6D7E2F746312D4DDE5121C
:105D660075F06484E5F07E3512D37512CEC202CE8C
:105D76002E30480320740122E4FCF5A79006E3E0E8
:105D8600F9A3E0FE24FE40EFA3E0FF7D78E537604F
:105D960008304FE3200C2A800B120E67E5BD20E089
:105DA60010304F0DD206E57124FE5015125E8B8021
:105DB600107D3CE546600A7D141460057D0A14706A
:105DC600B6891112534F7D6F12546FBE00A9EF248E
:105DD600E240A4AD07E51112DCBB202404B2D5B223
:105DE600D1781F795612DDB9A806A907E511242D29
:105DF60075F0B484E5F012DCBB7407304F02740E04
:105E0600FDFA12DDB9B2D5B2D112DDB9B2D5B2D131
:075E1600DDF0AD0212DDB961
:105E1D00850616850717B2D5B2D112DDB985061ED6
:105E2D0085071F7A03304F027A06E511241675F0A7
:105E3D00B484E5F012DCBBA816A917AD0212DDB9CA
:105E4D00DDFBE51124EA400224B412DCBBA81EA937
:105E5D001FAD0212DDB9DDFBE5377021304F1E900D
:105E6D00A5E9305D0390A5E57F3C7E3312773512B1
:105E7D000E67E5BD20E00612CA7A12D7A822C3E943
:105E8D009570500224B4F922E51B2402FFE4351C61
:105E9D00FE305D1ABEC305BF4D028012AC06AB07C6
:105EAD007A1B1253717832125513AE04AF03227858
:105EBD007379641256E01257F6751CC3751B4B208F
:105ECD0032048B1C8A1B22125EBC30320122AC19AB
:105EDD00AE1AA91DAF1FB90005BC00028010C3E9A1
:105EED0013F9EF13FFC3EC13FCEE13FE80E8BF298B
:105EFD00005006BE2900500122C3EF13FFC3EE135D
:105F0D00FE80EB3E7FE3E3E3E3E3E3E3E3E3E37F01
:105F1D003E0C1C3C7C7C1C1C1C1C1C1C1C7F7F3EDA
:105F2D007FE3E3E3070E1C3870E0E3FFFF3E7FE302
:105F3D00E3030F0E0F03E3E3E37F3E070F1F3F77EE
:105F4D00E7E7FFFF0707070707FFFFE0E0E0FEFFBA
:105F5D00030303E3E37F3E1E3F73E0E0E0FEFFE358
:105F6D00E3E3E37F3EFFFFE3E30303070E1C383853
:105F7D003838383E7FE3E3E37F3E7FE3E3E3E37FBF
:105F8D003E3E7FE3E3E3E37F3F030303E77E3C0015
:105F9D000000181818FFFF18181800000000000066
:105FAD00000000FFFF0000000000003FF00000387F
:105FBD001C38F00180C1F020F0FC0038F03FE0000B
:105FCD000000007CC6C6C6C6C6C6C6C67C183878D4
:105FDD001818181818187E7CC6C60C183060C0C664
:105FED00FE7CC6C6061C0606C6C67C0C1C3C6CCCCC
:105FFD00FE0C0C0C0CFEC0C0C0FC0606C6C67C3CDC
:10600D0066C0C0C0FCC6C6C67CFEC6C6060C18302F
:10601D003030307CC6C6C67CC6C6C6C67C7CC6C6FD
:10602D00C67E060606CC78000018187E7E1818006D
:10603D0000000000007E7E00000000000000000057
:10604D000000000000C6E2E2D2D2CACAC6C6C20033
:10605D000000000000000000008080A0C0A0003003
:10606D004020C08080C0A0A0000060A0600000A003
:10607D0040A05098D090882050A850888850A850A3
:10608D002060806000000040E040000000000080C3
:10609D000000E000000000000040002040800040B3
:1060AD00A0A0A04040C04040E0C02020C0E0E020C3
:1060BD004020E02060A0E020E0C02020C06080E013
:1060CD00A0E0E020404040E0A0E0A0E0E0A0E02023
:1060DD00C0004000400000800080002060E0602093
:1060ED0000E000E00080C0E0C080E0E0E0E0E00023
:1060FD000000000040A0E0A0A0C0A0C0A0C040A033
:10610D0080A040C0A0A0A0C0E080C080E0E080C022
:10611D0080806080A0A060A0A0E0A0A0E0404040F2
:10612D00E0202020A040A0A0C0A0A080808080E022
:10613D00A0E0A0A0A0A0E0E0E0A040A0A0A040C0F2
:10614D00A0C0808040A0A0C060C0A0C0A0A0608002
:10615D004020C0E040404040A0A0A0A060A0A0A072
:10616D00A040A0A0A0E0A0A0A040A0A0A0A0404062
:10617D0040E0204080E02020A870202070A8202042
:0D618D0008F030D0100000F0A8A8000000BD
:10619A00E0000000902048708898984000E0E0E015
:1061AA0000A0E0E0E04060301030604040E0404055
:1061BA0060909090909060206020202020706090E5
:1061CA0010204080F06090102010906010305090A5
:1061DA00F01010F080E010109060609080E09090D5
:1061EA0060F0102020404040609090609090606085
:1061FA00909070109060C0E0F0F8F0E0C0000000ED
:10620A000000000000000000000000506050007014
:10621A007050000078807008F000F8888888F800CC
:10622A00C0C8102040981800C0B098B0C0006020C4
:10623A0040000000000090D8FCD8900000246CFCBC
:10624A006C24000020A870A82000002020F820203C
:10625A000000000000000080000000F000000000C4
:10626A0000000000606000081020408000708888EC
:10627A00888888702060202020207070880810206C
:10628A0040F8F810201008887010305090F810105C
:10629A00F880F008088870304080F0888870F80824
:1062AA00102040404070888870888870708888788C
:1062BA0008106000606000606000000080000080DC
:1062CA0000002040F84020000000F800F80000001C
:1062DA002010F8102000708808102000200000000C
:1062EA000000000070888888F88888F08888F0881C
:1062FA0088F070888080808870E09088888890E034
:10630A00F88080F08080F8F88080F0808080708843
:10631A0080B8888878888888F888888870202020BB
:10632A00202070381010101090608890A0C0A090A3
:10633A0088808080808080F888D8A8A88888888803
:10634A0088C8A898888870888888888870F088881B
:10635A00F080808070888888A89068F08888F0A08B
:10636A00908870888070088870F82020202020206B
:10637A00888888888888708888888888502088884B
:10638A0088A8A8A85088885020508888888888506B
:10639A00202020F80810204080F800CCAC9CACCC1F
:1063AA000000CCD4E4D4CC0004781828C800FC40FF
:1063BA00A04018202018000000000000F80000008B
:1063CA0000A040A05000788888986870884030887B
:1063DA0070200000F0A8A8A8A878484848487888FB
:1063EA0070888080887020A88898A8C8888880507B
:1063FA0048FC485080304C5C6060603C00E0F0082B
:10640A000808F88044485C484480F880808080808E
:10641A008078484848484888B8A8A8E8A8A8B8880A
:10642A0088888888F808500070888888708080F08A
:10643A0088888888F8888888888888F090909090DA
:10644A0090F0A8A8A8A8A8A8F8888888F808080832
:10645A0050008888888878A8A8A8A8A8F808000002
:10646A000000000000000000000000008888888802
:10647A00E8A8E8A8A8A870A8A8A80000000000003A
:10648A000000000000000000000000000000000002
:10649A000000000000000000006000606000600072
:1064AA0060006060205020000000005090B890D03A
:1064BA0090886050500070705000882020887000CA
:1064CA000080C0A090F8003048B4B448300030488A
:1064DA00B4B44830FC0098D02058C800F8E8D880F6
:0A64EA00D8E8F8404050F850404058
:0300000002005E9D
:03000B0002B5E853
:0C000E00206E06859950D26E32D26F32FF
:0E00230010990AC298206DE385994FD26D3274
:10003800E4F537F534F52F12DE2CC229C22AC2683E
:09004800C227C214C215022D9C4E
:03005B00022B2A4B
:10B5DB008530F0C5F065308530F060F722C0D0C003
:10B5EB00E0C0F0C0A775A700C083C08275D00875F6
:10B5FB008A00300503758A7A758CEA0532E532705C
:10B60B000215320530E530640A6026201520E5313D
:10B61B00B40C0BE530B4010612BA6312D8DFE53176
:10B62B00B4180BE530B4060612BA6312D8DF02B8B1
:10B63B0002C2AFD2C075C07AD2AFF5300531E53159
:10B64B0064197040F531201529C225C22C7D0A746E
:10B65B000412DEDDEF33EE339005CCF0EE24F54033
:10B66B00112402400B24014005DDE4022B2AD225D4
:10B67B00D22CE5A6600215A678B5E660011678B661
:10B68B00E6600116302E0BE5367007C22FC22E1264
:10B69B00B990E5367004C24B8002153678A9E66086
:10B6AB00011678D8E66001160535E53570021535BB
:10B6BB00E590307B0B30E008D278C27BC200801A59
:10B6CB00307C0B30E108D279C27CC201800C307D1A
:10B6DB000930E206D27AC27DC202E59044F8F470DA
:10B6EB0003753500304A09E53324FA5003753305E9
:10B6FB00E5336005153302B7A7E590F454077003E3
:0DB70B0002B7A7A2E09200A2E19201A2E223
:10B71800920230100320143D75330820001B2010BE
:10B728000C2011098013E59030E10E8006E53724DE
:10B73800FC40F3E543541FF53320100375A6FF20A2
:10B748002E5D301004E536705620100C201109E5E6
:10B758003524F55003753304D21BD2A5D2A612B9ED
:10B768009075B44075B24078D8E670020534202749
:10B778002E20682B202928202A25A2107211501F5C
:10B78800E52054076019E53424375004C24A800F75
:10B798002401400B200026200119D27D7534C820D1
:10B7A8001558E531702412DEBD74E812DE96802A41
:10B7B80002B8D5E53724FC40E6D27C80DF3011DFC3
:10B7C800E53724FC40D9D27B80D275F00384E5F0BC
:10B7D80070DE12C51274E812DE96E531B406051261
:10B7E800C68A8016B40C0512C6A0800EB4120512C3
:10B7F800C68A8006B4180312C6A0E59030E1053069
:10B80800E202800620100820110520103C807D20CF
:10B8180027F82068F52029F2202AEFE53424304063
:10B82800E9240750E5600B205E088590F020F202BD
:10B83800740190B84A93D2A5201002C2A512B97B10
:10B84800806FC8A08269554646202F12E536603CB5
:10B8580024AA500AE53675F01984E5F06040D2A6AE
:10B86800201002C2A6D2A5202F0C7418304B0274E7
:0EB878006412B97B803BE53675F00C30480356
:10B8860075F00684A2E0744640E9743780E5E52B3E
:10B896005403600C20100E301106E54A6402600560
:10B8A60012B996800312B8ED101B08A25892A5A2F1
:10B8B6005992A675A700D082D083D0A7D0F0D0E049
:10B8C600D0D0201009C5A67003022B2AC5A632C205
:10B8D60018B40202D21812C5B030180874E412DE89
:10B8E6009602B7E202B7DD78A7E5B4600924E04026
:10B8F60005760002B996E534702920412220751F8D
:10B90600300D1CE57924CE40167AFFE5B110E7012B
:10B916000A2325B3F5B3EA35B4F5B4C313F5B2E695
:10B9260060021622C2412075028075E579FF6058D3
:10B9360020120424FD5051206502C21CD265FF244A
:10B94600B050027F4FEF90BA139375C70375C6FCCC
:10B9560075B90185BFF0A4E5F0F624F44002760C33
:10B96600301C2DE5BEC39FF5F0A4E5F024E04003AE
:10B9760075F020E5F0C21C79AA770375B300F5B41B
:10B98600C31375B100F5B222C26578A77680D2419D
:10B9960079AA7703D21CE4F5B3F5B4F5B1F5B22272
:10B9A600C26579A1E57924CE500DE720E7E2762835
:05B9B600301CDD7432BD
:10B9BB0080BE7680E720E7D3E5799740CE79AAE77A
:10B9CB00FAE5792323B4C500400274C42437300E42
:10B9DB0031F42437300D15F7BA0302FA0AC39AF57E
:10B9EB00B175B300EAF5B4C313F5B222101C07D23C
:10B9FB001C76C802B97D763274FF200E02749B024E
:10BA0B00B97DC313247E80CCFFF3E8DDD3C9C0B866
:10BA1B00B0A9A29A948F8A85817D7975716E6B68B6
:10BA2B0065625F5C595653504E4C4A4846444240FF
:10BA3B003E3C3A383634333231302F2E2D2C2B2AD4
:10BA4B0029282726252524242323222221212020AF
:10BA5B001F1F1E1E1D1D1C1CD2B5C28EAE8DAA8DA6
:10BA6B00AF8BAB8BE4F58DF58BD28E301401227836
:10BA7B00B6BE0007EF24E24002800806E624EC5035
:10BA8B00027614206705E624F64005E4FEFAFFFB78
:10BA9B007C007D0A12534F7C007D5E12546F8F51D8
:10BAAB00EE60037551FFEAFC7A33125363EBF5F04A
:10BABB00A4E5F0CB8CF0A425E0C5F035E0CB92D516
:10BACB0025F050060BBB0002D2D530E7060BBB00AE
:10BADB0002D2D5ECF5F0A42BFBE5F03400FC30D50D
:10BAEB00010C78A6E6C39BFF18E608F6EB18F618D0
:0EBAFB00E69CFE18E608F6EC18F63014012260
:10BB09007A0050040A1255E67C007D6E12546F8F3C
:10BB1900F078A2E6A4FBACF0125585EBBA0002F46A
:10BB290004FAE4F8FFEA30E70118E57960062075C0
:10BB3900031FF4042AF579EF38D27520E70860036A
:10BB49007579FF02C7E3C2750470F5E579F40460FD
:10BB5900EFF57980EE120E5D78BBA6BC120E7BE57F
:10BB6900BE78A2F624F65007E4F5BEF6124EE612A8
:10BB79000D46E5BEF54824F65008E4F5BEF5481231
:10BB89004EE6E5BFF54324F3503924F34035120E50
:10BB99007178A1A6BCE5BF789DF61424FB50087402
:10BBA90003F6F5BF124EE678B7A6BE120E67E5BDDD
:10BBB900A2E39266A2E49267035403C253B401025A
:0EBBC900D25322740DF5BFF543124EE680C034
:10005E0078FFE4F6D8FDF4F5A6D2B4D2C075C07A16
:10006E0075D75075AE1375AF017581D87590F8754B
:10007E00EFBC75FDFFD2A412DE03C2A47450122B86
:10008E0042758951D28C75A882D2BC12BBD712DEB2
:10009E00BD12C48812BB5E12D992122A087F407E0E
:1000AE0001909C73127702124D4A12DE0312DAE4AB
:1000BE0012DD1B12DE2C7C1412DE0D300003022B1F
:1000CE002ADCF512489F753A001248EDE53A701693
:1000DE0012DEF17F437E0690A3CE12770212DD1B55
:1000EE003000FD022B2A75A6FF12489F12BB5E122E
:1000FE002A0812DD1B12DDFF12DE2C78B5761E12D9
:10010E00D99212C47DC215C214122A08909CBA7FCD
:10011E00781276F0205E0A7F767E12909CC712D5FA
:10012E00097F4012DD917F497E0978AEE612D375C4
:10013E007E15743A12D4DD7E1AE53E12D3757E26F4
:10014E00743A12D4DD7E2BE53F20E00805A6E5A625
:10015E00700215A6E53F12D3757F5312C9F87F576B
:10016E007E0B12D2A212D32A7F60207303020208E2
:10017E007E0BAC5DAB5C12D2A612D32A7E31127707
:10018E008D7F697E1212D82D3025087E1290DB4DA0
:10019E0012D509E5A60303543FFDFE0D7F7312DE53
:1001AE00360F12DE361EDDF478B5E57124F6400208
:0801BE00761E307419E660564C
:1001C6007F727E16744012D4AB7E17E612D4337E4D
:1001D6001F745312D4AB12DD1B10003710013710F9
:1001E600023712483FD2AC75369612DB93B4E0055F
:1001F600124935800AE53670F112488D12DDFC028F
:10020600010D2074097E2BE52E540712D4CA7E17E1
:1002160002018C022B2A022D628072E53524C85019
:1002260049E59020E244D0E0D0E012027102735614
:10023600E53524D25034E59020E22FD0E0D0E0120C
:10024600DEF18038E53524D25020E59020E21BD03F
:10025600E0D0E012DEF1306B0B7F091276E7124F29
:100266001E127BBD1202710206BE2212DEF190A49E
:10027600847F001276F012DD1B02DDFC12DEF190A7
:10028600A4847F001276F012DD1B12DDFFC215C2B8
:1002960014C227C26812DE2C753701909DA3121C6A
:1002A600FF9002AB730200F70217C2020B56021F41
:1002B60012021F0E0206BE0206FB0273560202C699
:1002C60012DE2C75370790A12B121CFF9002D673F5
:1002D60002029302096B0209A50209D90202FA0277
:1002E60005AD0202C60202C60203180202FF024B55
:1002F600B30203261248F0805A7F517E00747212B0
:10030600D4D9121E5C40B9124E3512D99212BB5E78
:1003160080AE7F49A25E120D31925E120D5080A012
:100326007F64120E9E121E5C401DE5352480F47516
:0C033600F0198460157F727E1F12D4CA7B
:1003420012DD1B1001E810000280E30202C612BC9B
:10035200440202C6124EE612DE2C75370290A2F952
:10036200121CFF900369730202C6020EA8020F0D4F
:10037200020F61020FB6020FFA02100902035902BC
:10038200051302038980D0D21412DEF17F147E0598
:1003920090A341127702121E1912DD1B12486875D2
:1003A200A6FFD2AC1000DE12DB93204CF2B405EFB4
:1003B200E4F511F514F5151204411204D51248683A
:1003C20075A6FFD2AC1000BD12DB93204CF2B4151F
:1003D200051204C880E7B406E712047FE51424FC82
:1003E20050D5E4F56FF56EF56D12048B1204D5123B
:1003F200486875A6FFD2AC10004212DB93204CF283
:10040200B415051204C880E7B406E71204B5E56F17
:1004120024F050D5124868743B12DC0F7A47909C46
:100422006A1224C9742A12DC03909C731224C974C0
:100432002A12DC03DAF912DC2C12DE0D020359ACAB
:1004420014AB157A0412536375A704900400E4F008
:10045200ECF0EBF08514C78515C67F08120467DF40
:10046200FB75A7002275B901E5BCF0E5BDF0E5BE5C
:10047200F0E5BFF005C6E5C6700205C722E5152402
:1004820008F515E43514F5142275A704900400E567
:100492006F4410F0E56EF0E56DF0740312BC107F4E
:0404A20020E4F5F766
:1004A600C2B2C2B2E5F7F0DFF4D2B275A700227489
:1004B60020256D54E0F56DE4356EF56EE4356FF587
:1004C6006F2205117F287E00E51112D3EC8006907D
:1004D6000402E070177F287E15900400E012D3EC2A
:1004E6007E2A900401E012D3EC12DD1B12486874D8
:1004F6003A12DC4675A7009004007F23E0A312DBC6
:10050600E2DFF912DC1D3099FD2202035912DEF1F9
:100516007F0F90A6781276F0121E1912DD1BC214F8
:10052600C21512DDFC7510651000DFE53170F9E5C6
:10053600106465700D855E14857A15E4F512F51361
:10054600800C78A8E51326F513E43512F5127F1E04
:100556007E19E51012D392C3E57A9515F517E55E77
:100566009514F5167F287E0BAC16AB1712D2A61281
:10057600D32A12DD1B12DE0DD510ADAB17E516FC26
:1005860030E7031255F67A0A79001253DCA912A84D
:1005960013125515EBF510243840037510C8120ECA
:1005A6005D8510BC02035612DEF1909CFE7F017E33
:1005B60009127702909D067F0A7E091277027F1341
:1005C60012C9F0751700120E6CE5BC12068DE5BD5A
:1005D60012068DE5BE12068DE5BF12068D909D565C
:1005E6007F5F7E06127702121E9E12DD1B751700B4
:0605F60012066D10000862
:1005FC0010011510024880F20517E51724F7500377
:10060C0075170075100080E2E51764087015120E5E
:10061C006C75BC0175BD2375BE4575BF67124EE682
:10062C000205ADE51012069F12DD1B12064D0510DA
:10063C00531007E51724FE400353100380AC02024D
:10064C00C6A9BCAABDABBEACBFE5171304F8E64007
:10065C00085407C42510C4800454702510F6027D7C
:10066C00A17800E875F009A42417FF7E3B7D20E8F3
:10067C00651770027D89ED12D4DD08B809E502DD3D
:10068C001BF8C4120693E812069F7E030517E517A4
:10069C0002D4CA540775F009A4909D0E2582F582E8
:1006AC0050020583E51775F009A42417FF7E0C0290
:1006BC007702C26812DE2C753705909EDC121CFF87
:1006CC009006D073020293027941027986027B1C58
:1006DC000206BE0206F4027A5E027AC402178B028C
:1006EC0006BE021771020C627F2E12168680C31290
:1006FC00DE2C753706909FB3121CFF90070B73020C
:10070C0002930217C802182A0218A30219700219C0
:10071C00A2021A19020750020749021A62021B07A9
:10072C0002072F7F64120E67E5BDA2E7120D31128E
:10073C000E67E5BD92E7F5BD124EE680B27F491219
:10074C00168680AB12090C122B6912DEF1121DF306
:10075C00E55804607790A0811207F912871E12DD0C
:10076C001B10000810011310021C80F50559C3E57D
:10077C0058955950D575590080D01559E55930E721
:10078C00C985585980C4E559B40F02802FB51F0292
:10079C00802A75F007A42408F51775162774B82558
:1007AC0059F987001207E712DD1B100028100128E9
:1007BC0010020280F574B82559F9A700E53524FA22
:1007CC00508878C7A64812090312DEF112DD1B12FD
:1007DC00DDFF0206FB1880CC0880C9E875F005A483
:1007EC0085F01CF51BC000125C7CD000221287AF78
:1007FC00B4FF0122751000751FFF1287C6E5106447
:10080C000F6017120830401274B82510F8E675F016
:10081C0005A485F01CF51B125D0D0510C3E558955C
:10082C001050D7221211AEF8602E6404602AE8141E
:10083C00B51025F51F120E7BE5BC70060475F0147F
:10084C00800375F019A485F01CF51B125D0D7E223A
:10085C0090A619127735D322C322E558B4FF012292
:10086C00751000E510640F602EE51075F007A424D8
:10087C0009FF74B82510F8E61208ED75F00A84C06B
:10088C00F07E2012D4337E28742C12D4ABD0E07EB0
:01089C002A31
:10089D0012D4981208AD0510C3E558951050C32217
:1008AD001211AEF8603964046035E8146510702FCC
:1008BD00120E7BE5BC1208EDF8C313923D7E1C129F
:1008CD00D4497E28742C12D4ABE4303D067405B89F
:1008DD000001147E2A12D4987E18742312D4AB22F0
:1008ED00305D1275F036A42432FBE435F0FC125560
:1008FD0085125585EB221209151276D5DFFB2212D2
:10090D000915127EB1DFFB2275C70375C6F078B8E5
:10091D007F042275C70375C6F375B901E5BFB548E8
:10092D0031E55924F1402BE55975F00484A9F024E3
:10093D00F0F5C675B901C5F0A9BC600CA9BD146070
:10094D0007A9BE146002A9BFE975F005A4F985F0E9
:10095D00CC22120E7BA9BD75CC0022124EE612DE02
:10096D002C75370390A196121CFF90097B73020220
:10097D00C6020C7B02131F020C90020C9B0216E6A2
:10098D000213A6020D5C0213DA02142002173802BC
:10099D00138E021465124EE612DE2C75370490A2EA
:1009AD0057121CFF9009B5730202C6020CAA020C65
:1009BD00B50209A5020CCB020CD60210230209A523
:1009CD00020CE5020CC0020CFF124EE612DE2C7575
:1009DD00370B90A2A3121CFF9009E9730202C60205
:0B09ED0010D10210D1020A6F020AAD07
:1009F800020A10020A330217CE02117602123E02D0
:100A080011E70212CF020D19120E67E5BF1470C16B
:100A18007F2E120E9E1F120E67E5BDA2E6120D3143
:100A2800120E67E5BD92E6F5BD80A37F37120E9ED4
:100A3800120E62A8BFE8120A6712DD1B1000081028
:100A4800010D10021280EE18B802EA780A80E60852
:100A5800B80BE2780380DE120E6288BF0209D67FE7
:100A6800367E2CE802D37B7F1C120E9E120E67A8DE
:100A7800BE120AA112DD1B10000810010D1002148D
:100A880080EF18B800EB780B80E708E824F450E111
:100A9800780180DD88BE0209D67F1B7E35E875F0B7
:100AA80005A402D3757F25120E9E120E67A8BF12E9
:100AB8000ADF12DD1B10000810010D10021480EF70
:100AC80018B800EB780980E708E824F650E17801C7
:100AD80080DD88BF0209D67F247E3BE802D4CA1293
:100AE8000E5DE5BF75F03CA4ACF0FDE5BE75F00504
:100AF800A42DFDE5F03CFC120E67E5BF14603675C9
:100B0800F005A485BEF0A42DFFE5F03CFE7C007D39
:100B18003C12547CC005EF75F01884E5F07F2D7EFB
:100B28002412D3757E30743A12D4DD7E35D0E012AB
:070B3800D37502DD1B7F2DC8
:100B3F007E0590A63B127702120E67E5BDA2E67FF7
:100B4F002D12161502DD1BD25712DEF1121DF312F4
:100B5F000B640202937F177E02909E011277027F31
:100B6F004C7E02909E18127702AC5DAB5C7F577E75
:100B7F000412D322120E8A85BC6285BD63E56124FF
:100B8F00F84044909E237F371276F0AE61AF607CC1
:100B9F00017D5E12547CC3741F9FFAAC63AB62EC91
:100BAF0033921750031255F6125363AB047C003087
:100BBF0017031255F674F52BFB74033CFC125339D3
:100BCF007F377E1512D29A909E307F697E0F1277F3
:100BDF0002E560240FFBE43561FCA25C923BD25C22
:100BEF007E1E12D2A6A23B925C7E30742012D4DD00
:100BFF007E36742012D4DDE5602562FBE561356336
:100C0F00FC7F227E0412D322E56245637016742E98
:100C1F007E3A12D4DD12DD1B10000D1001151002EB
:100C2F0026020B8C742080E81562E562B4FF0C1568
:100C3F006380080562E56270020563E53524F550AF
:100C4F0003753301020B8C120E8A8562BC8563BD5E
:100C5F00024EE67F637E00747212D4D9121E5C407E
:100C6F00087F631276E7124EED0206BE120E71E593
:100C7F00BCA2E77F0A120D34E5BC92E7F5BC02096E
:030C8F00687F1C5F
:100C9200A20D120D31920D80097F25A20E120D3187
:100CA200920E120D5002096B7F0AA20F120D3192A1
:100CB2000F802A7F13A208120D319208801F7F52E3
:100CC200A20C120D31920C80147F25A20B120D3151
:100CD200920B80097F2DA209120D319209120D503B
:100CE2000209A57F49120E67E5BDA2E3120D31127A
:100CF2000E67E5BD92E39266F5BD0209A27F5B1223
:100D02000E67E5BDA2E5120D31120E67E5BD92E553
:100D12009243F5BD0209A27F6D120E67E5BDA2E006
:100D2200120D31120E67E5BD92E0F5BD0209D61231
:100D32000D468F1F9217120E9EAF1F1F7E3912840F
:100D42000BA21722120E7685BC2B85BD2122120E14
:100D520076852BBC8521BD024EE6203714120E711A
:100D620085BE12120D89120E718512BE124EE680D8
:100D7200057F3F120D7B02096B7E0390A221127741
:100D82000212DD1B02DDFC75A6FF12DEF112B5DBDD
:100D9200740712DEDD8FF0740612DEDDEF2512C35A
:100DA20095F0A2E7923D4010FD24CD50027D32AC79
:100DB20005C3743F9DFD800FF404FD24C850027DDD
:100DC20037AC0574402DFD7F4012C9F07E1212DE51
:0F0DD200360EBE1EF91F303D020F0FEF6D70ED94
:100DE100E536700A753606EC2513F5148C13120ED0
:100DF1000712DD1B1000071001083002072215122F
:100E01008002051280827F377E28742E12D4DD7F06
:100E1100347E21740A303D010412D4F8E514FC2417
:100E21009C50027C637F347E2DEC12CE1C7F437E6E
:100E31001E12D2A27E00E51212D4397F057E0290E5
:100E4100A22C1277027F6D7E0190A2371277357F37
:100E5100747E0490A248127735021DF375C6F480A2
:100E61003575C6F5803075C6F6802B75C6F78026B8
:100E710075C6F8802175C6F9801C75C6FA8017758C
:100E8100C6FB801275C6FC800D75C6FE800875C64E
:100E9100FF800375C6FD75C70375B9012274721F02
:100EA10012D4D90F02DD1B7F0A120E9E7E2A124830
:100EB100F0120E7BA8BF120EDC10001210010510FB
:100EC100021580F508E824E750EC781880E818E866
:100ED10030E7E3780080DF88BF805F7F097E05907F
:100EE100A4FCB80C0390A4F61277027E27E53D28F6
:100EF100240C75F01884E5F012D3757E33743B121F
:100F0100D4DD7E35E53E12D37502DD1B7F13120E53
:100F11009E120D46120F3E10000810010510021717
:100F210080F2105C07205D0BD25C80E8105DE5D299
:0D0F31005D80E1D25C80DD852BBC020356A3
:100F3E00205C10205D1890A54F7F127E2312770241
:100F4E0002DD1B90A563205DF090A55680EB90A569
:100F5E005C80E67F1C120E9E120E76A8BF120F98B2
:100F6E0010000810011110021A80F2E824F250034A
:100F7E001880EA780D80E6E824E740030880DE78E2
:100F8E001980DAE8F5BFF54380A37F1B7E26E412B5
:100F9E00D4CAE82323B464087E26740112D4CAE4AA
:100FAE007E2E12D37502DD1B7F25120E9E120E852C
:100FBE00A8BCE8120FF112DD1B10000810010D1075
:100FCE00021F80EEE824E050E9188006E824CF40A6
:100FDE00E108120E8588BC124EE6D21512D9928007
:100FEE00D180157F247E3724E202D3E67F2EA20A1B
:100FFE00120D31920A120D500203597F37120E67ED
:10100E00E5BDA2E4120D31120E67E5BD92E49267C2
:10101E00F5BD0203567F367E00747212D4D90F7E50
:10102E0016743F12D4AB120E71A8BD12109C12DDB5
:10103E001B10000810010510021080EFE8248750E5
:10104E0004240A800224E8F880E17F377E1674209B
:10105E0012D4AB7E2C743F12D4AB12109C12DD1B3B
:10106E0010000810011410022080EF18B80904783F
:10107E007880E7B878E478E780E008B87904780AF1
:10108E0080D8B8E8D5787980D188BD0209A2E82445
:10109E0087923DE8500224917F367E30C313923BF7
:1010AE0012D3E67E3CE4303B02740512D4C37E1AA2
:1010BE0090A442303D0390A4461277027F3C7E3AC4
:1010CE0002DE367F127E00747212D4D90F7E207427
:1010DE003F12D4AB120E5D85BE1085BF1112115892
:1010EE0010000810011110021B80F21511E511B449
:1010FE00FFEB75111780E60511E51124E850DE753A
:10110E00110080D91211587F137E20742012D4AB97
:10111E007E31743F12D4AB12DD1B1000081001118A
:10112E0010021B80DF1510E510B4FFD875100B8070
:10113E00D30510E51024F450CB75100080C6120EA6
:10114E005D8511BF8510BE0209D67F127E24E51182
:10115E0012D3757E30743A12D4DD7E35E51075F0FB
:10116E0005A412D37502DD1B7F49120E9E1211AE1D
:10117E00F81211B410000810010D10021280F218AE
:10118E00B8FF02780480EA08B80502780080E212FF
:10119E000E5D88BD124EE6B800030209D902123E5A
:1011AE00120E5DE5BD227F487E0590A45C1277028B
:1011BE00E8601CB4040A7E0590A451127702800CDC
:1011CE0090A4681277027E38E812D4CA02DD1B9012
:1011DE00A4637E2912770280F31211AE601D64049F
:0211EE00601986
:1011F0007F5B120E9E120D46121219120E7610000F
:101200000B10010810020C80EF0209D9105FE9D21F
:101210005F80E5852BBC0209D61211AE601F640405
:10122000601B7F5A7E0590A45C1277027E2390A4F7
:101230006C305F0390A47312770212DD1B2212112F
:10124000AE70030209D97F527E11120E9E120E7BE0
:10125000A8BC12127E120E7B1000081001081002AA
:101260000880EF1880EC0880E9120E7B88BC124ED3
:10127000E6120E85E875F005A4F5BD0209D6121137
:10128000AE604BE875F03270040475F028A4ADF040
:10129000FC305D11ACF0FB7A8A125371EB30E7053C
:1012A0000CBC00010DAE05AF047C007D6412547CC3
:1012B000C005EF7F517E1A12D3927E2C742C12D46B
:1012C000DDD0E07E2F12D3751241B712DD1B227FD5
:1012D00064120E9E120E7BA8BD121300100008109F
:1012E000010F10021680F218E824CD50EC783280FD
:1012F000E808E824CD50E2780080DE88BD0209D6F7
:101300007F63E823C2E012CF4F75F06484C0F07EA3
:101310002612D4CA7E2C742C12D4DDD0E080A47F97
:1013200013120E9E120E71E5BCA2E7923DC2E7F8C1
:10133000E812135E12DD1B10000810010D100212DE
:0313400080EE1824
:10134300B800EA783280E608B833E2780180DEE854
:10135300A23D92E7F5BC79A1F78079547F305C0117
:10136300237F127E2375F00A84C0F012D3E67E2D0C
:10137300742C12D4DDD0E07E2F12D4C30F7E3590AF
:10138300A569305C0390A5C50277357F64120E9E74
:10139300120E7BE5BE7F637E2C128460F5BE79A2BC
:1013A300F780317F37120E9E120E76A8BC530003CE
:1013B3007F367E32E812D4CA12DD1B1000081001FA
:1013C3000710020780E718180880E2E5BC54FC48C0
:1013D300F5BCF52B0209687F49120E9E120E85A8F3
:1013E300BE12141112DD1B10000810011110021A95
:1013F30080EFE8240AF8242450E778DB80E3E8242C
:10140300F6F8247F40DB788180D788BE80C6E8F475
:1014130024DC75F00A847F487E3B02D4CA7F5212D3
:101423000E9E120E85A8BF12145812DD1B10000861
:1014330010011110021A80EFE82408F8245750E72E
:1014430078A880E3E824F8F824A040DB786080D70C
:1014530088BF0213D7E8F424A923C47F517E3B023B
:10146300D4CA122C74754A00D210C211D214D27588
:1014730075791475340012DEF17F007E0290A202AA
:101483001277029041E07F087E2612D509E52B549E
:10149300030F7E3912D4CA121E0E12D173128ED1CB
:1014A30012DD1B10000810011A10022480C52075DC
:1014B30004057980BE1579E579B4FF05C2757579A0
:1014C3000180B02075EB1579E57970A7D27580A3FB
:1014D300C210C21402096B120E76E5BE7F097E3A72
:1014E30002D4CA120E7BA8BF120EDC120D46120FD5
:1014F3003EA8BF120F98120E85E5BC120FF17F2D87
:10150300A20A1216157F36A267121615120E5DE592
:10151300BC7F487E3202D3EC120D467F1BA20D1214
:1015230016157F24A20E121615120E71E5BC1213A6
:101533005E7F09E5BCA2E7121615A8BF121724E5C2
:101543002B54037F367E3212D4CA120E7BE5BE7F44
:10155300637E2C12D4CA120E85A8BE121411A8BF22
:10156300121458120E67A8BC021769120D467F09A0
:10157300A20F1216157F12A208121615120E67E596
:10158300BDA2E37F48121615E5BDA2E57F5A1216E8
:10159300157F51A20C1216157F24A20B1216157F6C
:1015A3002DA209121615120E71A8BD02109C120E5F
:1015B3005D85BE1085BF11121158120E67A8BE12A9
:1015C3000AA1A8BF120ADF120AE7120E76E5BE7F50
:1015D3003F7E3A12D4CA120E62A8BF120A67120ED5
:1015E3005DA8BD1211B4120E7BA8BC12127E120E9E
:0415F3007612121941
:1015F700120E7BA8BD121300120E67E5BDA2E07F95
:101607006C800B7F098040120D467F48A25E744EA6
:10161700400274597E3A02D4DD127DAD7F73127A8F
:101627000B127DFC7F6C127A1A7F2D801A120E67BF
:10163700E5BDA2E77F63121615120E76E5BE7F0998
:101647007E3A12D4CA7F4812166EB40104BF09014C
:10165700E4F51075F005A47E1E909F852582F5821E
:1016670050020583027702120E67E5BD035403C2D9
:1016770034C25330E103D2342230E002D253221273
:101687000E9E1F12164E12DD1BE5101000121001E0
:101697000610020280ED22045403B4030AE4800713
:1016A700145403B403011423C5BD54F925BDF5BD76
:1016B700124EE680CE1275D1EBF516F5147F6C123B
:1016C7007A1A1275B57F647E23E51612D449C3E5ED
:1016D700169514F5167F73127A0B7F2D02164E7F1F
:1016E7002E120E9E120E71A8BFE824FA400330375F
:1016F70002780312172412DD1B10000810010D10C9
:10170700021280E518B800E1780580DD08B806D92F
:10171700780180D5799DE8F7F5BF0209687F2D7EAE
:101727002C7420B80502742E12D4DD7E32E802D460
:0C173700CA7F5B120E9E120E67A8BCE871
:1017430012176912DD1B10000810010D1002128020
:10175300EE18B800EA780380E608B804E27801805E
:10176300DE88BC0209687F5A7E2CE802D4CAD2689C
:1017730075480A1248F0D214122B77127EE5123301
:10178300CFC26B12024A80F3D214751501127D6722
:1017930075B901E5BC20E71C127E9775A6FF127E82
:1017A300F1121E1912DD1B12780B10000F500512D7
:1017B300793380E70515E515242050D10206BE12C2
:1017C30017D40202931217D40206FB1217D402098C
:1017D300D91217E0120E768548BE024EE6122B6927
:1017E300122B83125A3612DEF190A02AD2491287A5
:1017F3004B128704121DC912DD1B100014100105C2
:1018030010021B80F50548E548640A7002F548801C
:10181300CF1548E54864FF700375480980C28548C1
:1018230049122B83E558221248F0122B6985484947
:10183300C250E558B40F02D250125A36803AD2271A
:1018430075480A122B77125A3612DEF112866E9001
:10185300A41320290390A41E121E8BC26A1233CF35
:10186300106A0280E1C227127D3F854948121C3667
:10187300122B83D229125A3612DEF1909F4212871D
:101883004920500E121E7512DD1B1000101001AE00
:1018930080F8121E1912DD1B10000280FB0206FBEA
:1018A300122B69E55830E7137F1B90A3FD7E0512C9
:1018B300770212DD1B12DDFF0206FB122B83125A85
:0A18C3003685594912DEF1121E03AA
:1018CD0090A41E12874912870E12DD1B10000810FE
:1018DD00010A10020C80F512193B80DB12194880A9
:1018ED00D612DEF1121E0390A03A12874912870E0E
:1018FD0012871212DD1B10000810010A10020C8055
:10190D00F512195480DB12196280D6121BFC122BB2
:10191D0083125A3612DEF190A367128749121E41C7
:10192D0012DD1B10000510028880F80206FB055918
:10193D00C3E55895595003755900221559E5596459
:10194D00FF7003855859220549D3E5491495584030
:10195D0003754900221549E54964FF70058558490D
:10196D00054922122B69E55830E7057F240218AD91
:10197D00122B83125A3612DEF190A04512874912AE
:10198D001E8012DD1B10000A10010280F8121CA52A
:10199D0080DE0206FB122B69E55830E7057F2D022C
:1019AD0018ADC26B7559FF125A3612DEF1121DF3C6
:1019BD00E55930E703121E0E90A057128749128782
:1019CD001E12DD1BE55820E706100008100111104E
:1019DD00021B80F00559C3955950CF7559FF80CA28
:1019ED001559E55964FE70C285585980BDE55920D9
:1019FD00E711D26B75A700758307C4F582E0B2E7D6
:101A0D00F080A7306B03121C530206FB122B69E505
:101A1D005830E7057F360218AD122B83125A361255
:101A2D00DEF190A062128749121E5C4009121C9AC9
:091A3D00121CCF121A460206FB2E
:101A4600120E7BE5BD75F00584F5BCF5BDF5BEF55A
:101A5600BF120915124EE605C6DFF922122B69E5FB
:101A66005820E7087F5190A06B0218B012DEF19063
:101A7600A429128749121E1912DD1B12484FD2AC37
:101A860010001FE55830E7F8306DF5121B9C7E20DC
:101A96007F00501390A47A12773512DD1B12DDFFFA
:101AA60080CAC2AC0206FB1B8B13909F5F12773570
:101AB60012DD1BC26B7B007514B8121C8F127E667A
:101AC600127E185025A814E824384004A6010514EF
:101AD6000BC3E5139B50E678B8121CD1306B03128A
:101AE6007BBD122B83125A368082127DADE51660BD
:101AF600E6D26B127EC3C003127D7ED003A9158089
:101B0600C4122B69E55830E7057F5A0218AD122B2F
:101B160083125A3612DEF190A076128749121E36CB
:101B260012DD1B10003510010280F8754605121BE8
:101B36006450157F007E357407954612D44912DD30
:101B46001B12DDFFD546E7D390A433500390A47A49
:101B560012874912DD1B12DDFF80B30206FB124815
:101B66004F12DC35745212DC46745412DC03E5580D
:101B76000475590012DC241277BA4016127D3F1202
:101B86007E9712780B400B0559C3E558955950ECD2
:101B9600C322C2ACD32212484FD2AC12DB8E204CE9
:0D1BA600F1B440F712DB93B4400312DB935F
:101BB300B452E2F53812DB93B454DA12DB93FA60D1
:101BC300D424EF40D012DB93E53870C912DB9312B3
:101BD300DB9312779F7B007E031278965010205080
:101BE300B412DB93204C03B440F7DEED80A7127EE2
:101BF300760B12779FDAE0C322121CE0E55924C862
:101C0300F88602E54924C8F9986013146010500F50
:101C130018E608F618E86970F7A702121CCF22E548
:101C230059640F60F91908E618F608E86970F7A710
:101C33000280E8121CE078C8C250E6B4FF028007B5
:101C430008B8D8F6D25022B8D702D250A615807C55
:101C530078B8121CE2E4F9F5A7758307E9C4F582A5
:101C6300E030E70AE924B8F82438400276FF09C3D4
:101C7300E5589950E7121C9A78B879C8E6B4FF0280
:101C83008002F70908E8243850F2804079B877FFDA
:101C930009E9243850F82279C877FF09E924285044
:101CA300F822121CE0C23D78D7B6FF04A900D23D4A
:101CB30018B8C7F5203D0279D81978C8B6FF0122B4
:051CC300C3E899500781
:101CC800C6C7C6081980F478C8121CF1127ED31250
:101CD8007ED3127ED3027ED378C8121CF1127EB155
:101CE800127EB1127EB1027EB175C703E54875F068
:101CF80004A42480F5C62212DEF1C23C1276F4E573
:101D080037605314604D14604514603D14603514F9
:101D1800602D14602514600E14600B14600D14609F
:101D28001414600C803012160E802B1216BC8026FC
:101D38001215B1802112160A801C1216348017124F
:101D48001620801212156E800D12151B80081214B1
:101D5800E680031214DA12DD1B12DE03121DF312E1
:101D6800B99CA81F08E814C23BB51D02D23B75F008
:101D780007203C0375F009A4FF7E00303C0C74205A
:101D8800303B02743E12D4AB800A740B303B0274B1
:101D98000A12D4C3D8CF12DD1BE51D1000081001AC
:101DA8001010021880B9651F7003751DFF051D808E
:101DB800AE7005851F1D80A7151D80A375F003A4AF
:101DC800227F7B7E0090A37F127735E54824F6407A
:101DD800087E0A90A3E012773522127A377E0574BE
:101DE8005B12D4A77E1D745C02D4A7121DE27E3458
:101DF80090A390027735127A378003121DE27E3164
:0E1E080090A394027735121DE27E3190A485DE
:101E1600027735127A377E008005127A377E2D904A
:101E2600A485027735121E367E31909F990277354A
:101E3600121E197E1A909F9E027735121E1980C0B7
:101E4600121E197E18909F4C027735121E197E1AA3
:101E560090A48A027735121E197E1A90A48F1277E3
:101E66003512DD1BD3100006C310010280F62212C4
:101E76001E197E1A90A034027735121E197E18900C
:101E8600A0500277357F007E2012773502DD1B12C7
:101E96007A3790A495027733127A3790A4A6027700
:101EA6003312BE5E120E94E5BDF55EF56CE5BCF52B
:101EB6005FF56B756A007561FF75A70490070012E0
:101EC600BE08B4FC23E582C313F561E56CF0E56B4F
:101ED600F0E582600F12BD7FE56C655E70E1E56B33
:101EE600655F70DB75A700223024EA0460E7240FE3
:101EF60040D380E1E560758307C333F582E0A3F53F
:101F06006CE0F56B756A0022D2248002C224D214DA
:101F1600C21F121EA7756000E561B4FF1612DEF13E
:101F2600909E337F0A7E0512773512DD1B12DDFC8B
:101F3600020293C210C21112DEF1121DF3301F0A03
:101F46007F07909E4112773380647F007E01C3E550
:101F56006012D4497E0E742812D4A785604874078F
:101F6600F51FFF7E00743E12D4ABE548121EFC122C
:021F7600C7FFA3
:101F78001224D80548C3E5619548FD401CE51F2497
:101F880007F51F24C850E17F387E01ED0412D449BB
:101F98007E0E742912D4A7800DE51F2407FF7E0149
:101FA80090A484127735201F0312251B12DD1B1005
:101FB800001910012C10020280F5120236301F3D64
:101FC800020282101F02D21F021F39E56160F4E588
:101FD8006065617005201FF080E9201FE6056080BC
:101FE800E7E56160DEE56065617005201FD5800961
:101FF800201FD5E560700280CA156080CB121EA72D
:10200800121EFA12C7FF12260F756A1012BDF112BE
:1020180026C6909E48D23C1276F4121D6490202960
:1020280073021F3902330F022049022035121E5C49
:1020380040CB121EFA12BE08C2E2FF12BC2E021FCB
:102048001212DEF17F6490A65E1276F07F7990A678
:102058006B1276F012DD1B75160010000A100109CC
:1020680010020280F505160516C253121EFA12C791
:10207800FF75370A909E61121CFF9020867302201C
:10208800050220AD02227C0222810220710220B4C6
:102098000220B90220710220F70220FB0220FF0271
:1020A800210602210A7F0A12168680BD124868801E
:1020B8000312485D780A1221D9740912DC01122230
:1020C8001812DC1D12225312BDF112BE1912BD40A6
:1020D80012BF30122362D5150C75150A122266122A
:0C20E800248912DC1D100204E57F70DB6F
:1020F400022005780A800678048002780112486874
:102104008009780A8002780112485D1221D9740985
:1021140012DBF6122218E54812DBE2E516540344FA
:102124003012DC03742A12DC0312DC0312DC1D12ED
:10213400225312BDF112BE1912BD4012BF30122338
:1021440062D51548854815122266E51C12DBE2E5C6
:102154001B12DBE2E51B2548F51BE4351CF51CE4EA
:10216400A27792E7A27492E0A27392E112DBE2AD4D
:1021740075AC74AB73E57DC412219AAD78AC77ABC2
:1021840076E57D12219A1224A712DC1D100204E5C3
:102194007F709F022005540F2375F00584F8C3EB6C
:1021A40033FBEC33FCED33FDC3EB33FBEC33FCEDE1
:1021B40033FD20E713EB28FBE43CFCE43D12DBE2B7
:1021C400EC12DBE2EB02DBE2C3EB98FBEC9400FCE9
:1021D400ED940080E88848121E20E4F54AF549751C
:1021E4006A2075150112BDF112BD40D5150E854842
:1021F40015E5492401F549E4354AF54AE57F70E5DA
:10220400744012DC46747812DC03746312DC0374C9
:0F2214002102DBF6122464E56012DBE2121EFAEF
:1022230012C7FFE53A12DBF6E53B12DBF6E53C129B
:10223300DBF6E53D12DBF6E53E12DBF6E53F12DBAE
:10224300F6740112DBE2E54A12DBE2E54902DBE266
:10225300121EFA756A20E4F51CF51BF514F51375C7
:10226300150122753800E51412DBE2E51312DBE2F7
:102273000513E513700205142212486880031248FF
:1022830052121E201223BC12DE07756A2075150137
:1022930075A6FF754A0112BD9912BD4012BF3012D7
:1022A3002362D5150975151E12238612DE11122419
:1022B30089E57912DBE2E412DBE2E57112234712CE
:1022C300DBE2E57012DBE2E57B24ACFFE55F34097A
:1022D30012DBE8EF12DBE2E51520E033857D56E4FF
:1022E30012DBE2E52EC412DBE812DC2C12DE111045
:1022F300021A30559B744012DC03744512DC0374DC
:102303004F12DC03744612DC0312DC2C022005E5B9
:1023130056122321C4FAE57D1223212A80C2FBC46D
:1023230012232E2323CB12232E2B22540FFC24F60D
:1023330050027C0090233DEC932200000101010236
:1023430002030303FA2440400A24804003EA3322B1
:10235300D2E72274FF2220E703C3132224C022E51D
:102363003F701F7F7B7E0078AEE612D433EE2404E9
:01237300FE6B
:10237400743A12D4ABEE2404FEE53E12D42D12DDE1
:102384001B22C015C016D21212A6B6C212D016D085
:102394001578AEE612DBF6E53E12DBF6E53F12DB1E
:1023A400F6E54512DBE2E55212DBE2740A12DBE2E7
:1023B40074C012DBE202DC2C744012DC037454128D
:1023C400DC46744E12DC03743012DC03E51654034D
:1023D400443012DC03122464742112DBF6E53D124E
:1023E400DBF6E56012DBE2121EFA12C7FF78ABE6F9
:1023F4000812DBF6E60812DBF6E60812DBF6E61254
:10240400DBF6E53E12DBF61229EFE51212DBF6E508
:102414001112DBF6740112DBE290A4B71224C97521
:102424006A1012BDF1057F057F787F12DBDB787BB4
:1024340012DBDB787D12DBDB787712DBDBE4FEFF7B
:10244400780712DBDB12DBDBE57412DBE2E57512E5
:10245400DBE2E412DBE2E412DBE212DBDB02DC2C83
:1024640075C70375C6FF75B901C217751D0085BC14
:102474001C85BD1B85BE1A85BF191252E9EE12DBFD
:10248400E2EF02DBE2E57512DBE2E57412DBE2E582
:102494007312DBE2E57812DBE2E57712DBE2E57644
:1024A40012DBE2E51664016011E55E12DBE2E57A17
:1024B40012DBE2E516640260012278BCE612DBE27C
:0A24C40008E602DBE275A700E493CE
:1024CE00700122A312DC031A80F4AF1F7E0478ADD4
:1024DE00E612D42D7E0C742C12D4AB7E0E18E6129E
:1024EE00D42D7E1A78AEE612D42D7E22743B12D4F1
:1024FE00AB7E24E53E12D42D7E2FE54012D4337EE2
:10250E0037743B12D4AB0E0EE54102D42D7532005A
:10251E00121EFA12C7FF857946787A796412C818A6
:10252E0074641256DE8E4712260F756A20D23D1243
:10253E00BDF112BE19122646303D09307406C23D59
:10254E008E1E8F1FE57F602BE54C24FFF54CE54D6D
:10255E0034FFF54D454C600512BD5580D2751D3CBE
:10256E0012BDF112BE1912BD40122646E57F600360
:10257E00D51DED1226A79026BF12D509203D0DAE12
:10258E001EAF1F1226A79026B812D509E546FD707C
:10259E000B90A5ED305D1190A5E9800C04701090A4
:1025AE00A5E9305D0390A5E57F381241B2804BE47A
:1025BE00FFFC7E05305D047E027FB312546FAC06C5
:1025CE00AB071253397F38C23DE51C6007D23D7E02
:1025DE002C12D498E51B203D026007D23D7E3012AE
:1025EE00D498E51A203D026007D23D7E3412D4986D
:1025FE00E5197E3812D4981241B7E53224C850FA44
:10260E0022E54075F03CA42541FFF54CE435F0FE83
:10261E00F54D7C007D1012547C0F8F4BAF4CAE4DA0
:10262E007C007D3C12534F7C00AD4B12547CEE4F20
:10263E0070010F8F4C8E4D2278647973C2D11226A1
:10264E005DFF78677976D2D112265DFE02DE36C343
:10265E00E796FB0809E796FC0809E796FDA2E792C4
:10266E001750031255FE75135A30D10E751320B242
:10267E0017AA47125383AB04AC05E546600B046002
:10268E000BAA4612539AEB03FBEB03FBEB543FFBF7
:10269E00E5132B2017029B9B22EE141430E701E466
:1026AE00FEEF141430E701E4FF2205057088A888B8
:1026BE007005052020F8202075320012DEF17E1EF6
:1026CE007F1C12DE36DFFB12DE367E1E7F1C12DE14
:1026DE0036DEFB7E1D7F1D12DE36DEFB7F007E2189
:1026EE0078ADE612D42D7E29742E12D4AB7E2D1821
:1026FE00E612D42D7E35742E12D4AB7E3918E61226
:10270E00D42D7F077E21745412D4AB7E25744F12C4
:10271E00D4AB7E2D78AEE612D42D7E35743A12D41B
:10272E00AB7E39E53E12D42D78AE1229EF7F0E7EA8
:08273E0021744C12D4AB7E257E
:10274600744112D4AB7E2DE51212D42D7E35743A27
:1027560012D4AB7E39E51112D42D7F157E25744433
:1027660012D4AB7E2DE54012D4337E35743A12D4A2
:10277600AB7E39E54112D42D7F217E0190A5B8129A
:1027860077357E0EAC77AB7612D2DF7E2B85795FFE
:1027960085787B12D8867F287E0190A5BC12773576
:1027A600751D2B751E10E5741229A37E25742F1234
:1027B600D4AB751D2D751E2BE5751229A37F367EAC
:1027C6000290A5A8127735E5721228501228E81251
:1027D6001EFA756A209004E6E56CF09004E7E56B56
:1027E600F0AE4DAF4C7C007D4012547CBF00010F13
:1027F6000FAC07AD07E4FED23D12BDF112BE1912B1
:102806002891E57F602CE54C24FFF54CE54D34FF1F
:10281600F54D454C600512BD5580DE751D3C0E120A
:10282600BDF112BE19122896E57F600612BD40D58D
:102836001DED1228667F7812CA027F767E007430FC
:1028460012D4ABE53224C850FA227E2112CF4F12A1
:10285600D4497E2F90A5C0305D0390A5C50277357B
:102866009004E6E0FD9004E7E0FCC3E56A9420FBF3
:10287600E56B9CFCE56C9DFD50032410FD12556E26
:0D2886009004E8EEF09004E9EFF022DD038D
:10289300AD040E7F78E55E20E72AE57A8549F0A44A
:1028A300A9F0E57A854AF0A429F9E435F0FAE55E62
:1028B3008549F0A429E435F02AFAE55E854AF0A4B7
:1028C3002ACF9FFF12DE36103D18C3EF9B50131B18
:1028D300EF6B600E8F018B0712DE361FEF6970F806
:1028E300AF01AB072290A56D305C0390A586754AB6
:1028F30040754900AF76E577FE20E76B7005EF245E
:10290300105064EF24A8EE34FD401190A572305CA2
:102913000390A58A754A1975499A8075EF2450EE7C
:1029230034FB401190A577305C0390A58F754A0C5A
:102933007549CD805CEF24A0EE34F6401190A57A62
:10294300305C0390A594754A067549668043EF246D
:10295300F0EE34F1401390A57D305C0390A599759A
:102963004A04754944802A8028EF2490EE34E840D5
:102973001190A580305C0390A59E754A0275498F1E
:10298300800F90A583305C0390A5A3754A01754918
:102993009A7F401277337F4612CA027F5F02CA02D0
:1029A300AE1E75F064305C0375F03284C0F0F870CD
:1029B30004EE2404FEE51D12D4ABEE2404FEE8600D
:0129C300070C
:1029C40012D498EE2404FED0E075F00A305C03754E
:1029D400F00584A8F012D498EE2404FE742C12D4CA
:1029E400AB0E0EE8305C012302D498E53E2541F598
:1029F4001124C45003F511D3E63540F51224E850F0
:102A040002F5122212B996C21012DEF17F057E0978
:102A1400909C6A1277027F137E08902A3C12D50993
:102A24007F2B7E01902AA412D50920370A7F277EA6
:102A340027902B1612D50922113007FE1FE001E161
:102A440001F80F00061B00F80C00180E007C1000A3
:102A54007006003C2000E006003E4001E004001E39
:102A64008003C004001F0003C004000F000780009F
:102A7400000F800780000017800F00000027C00FA0
:102A840000000043C00F00100083E00F002003018A
:102A9400F00700C00F01F80383007F87FE01FC00EC
:102AA4000E3E1800000300000000180000030000A0
:102AB40000003800000000000000300000000000AA
:102AC4000000FC761F0E1C6030ECFCBC3F172DF0A0
:102AD400F978613866264F619A706070C60E1EE3FD
:102AE40030E06060C60C1CC360C0E0618C0C18C789
:102AF400C0C0C0E18C1C39C611C0C4C19C993196B8
:102B04003180C8C1FF1E31E7E180F0C0EE1C31C343
:102B1400818006163091882892884924904927900C
:102B24009248A0E3C8BCC2AFD2C075C0107581D8AA
:102B340074FE122B42E4F5F9F5FBC2B480F7D2A679
:102B4400C2A512B97B12DE0302B99C75C703E5481E
:102B540075F004A42480F5C6C23C75B901E5BC0433
:102B64007002D23C22120E76E5BEF54824F65003DC
:102B7400754800753400753704C228D229D22A75E5
:102B8400C703E54824E75003754800E54875F00499
:102B9400A42480F5C6751607751700C23C122BC411
:102BA400122BC4122BC4122BC485175815587559EF
:102BB40000E548B40A09E5586005F46002055922A5
:102BC400203C1D75B90105C6AABCABBDACBEADBFEA
:102BD400EA122BE5EB122BE5EC122BE5ED122BE5BB
:102BE40022203C07F515B4FF03D23C22C0C7C0C65F
:062BF400127D6775A704C5
:102BFA00851683E517C4F8F58275B90105C6E5BCE3
:102C0A00F0C582F82406F92403C582E5BDF0E5BEC5
:102C1A00F0E5BFF075B90105C6E5BCF0E5BDF0E524
:102C2A00BFF08516838982E4F075B90105C685BCB3
:102C3A001385BD14E4F0F08882E5BEF0E5BFF075B7
:102C4A00B901E5BCF0E5BDF0E5BEF0E5BFF075837E
:102C5A0006E51723541E24B0F582E513F0E514F0B7
:102C6A0075A700D0C6D0C705172212BB5E78BEA6CC
:102C7A004808E4F6F55908761808F6D23608760AAE
:102C8A0008F6060876BEC254C25512BE73122B77D6
:102C9A00C229C22AC207C227C268120E67E5BDA2AC
:102CAA00E59243C24AE4F52EF534F536F52F78B6A7
:102CBA00F678B5F678A9F6789EF678B8A65E08A6EC
:102CCA007A12D248C26BC233C238C240C223C2226D
:102CDA00122CF475460278C5A646C23AD221C21908
:102CEA00C226E4F542F541F54022E45407205E0984
:102CFA00B4040040027403801B120E6CC313A9BCF7
:102D0A00600C14A9BD600714A9BE6002A9BFE940FE
:102D1A0001C45407F53722122B69125A3612090CCC
:102D2A0012DEF1121E41E55804700A7F327E0590C8
:102D3A00A3FD12770290A65512874B1208667F727E
:102D4A0090A64A1276F012DD1B10000510020480CC
:102D5A00F8D322C3220200F7120E67E5BD20E70569
:102D6A00122D2140F0754E50122C7412852C754488
:102D7A00031248ED12AEDBD54403022B2A201EF1C2
:102D8A00789F7680754A0012BC8FD210C211C21386
:102D9A00C21212483F75A60C12D99212C47DE5A63A
:102DAA0024FA400612488D75A60C20250CE590548D
:102DBA00057009E53524E25003022E54E532241841
:102DCA00400D75F00C84E5F070D41233D280CFD266
:102DDA001ED2AC306DC87532F012DB98B4E0BF1267
:102DEA004935E53124F39205201203123264122E7A
:102DFA001AC014128E17D014200A03122F3D123350
:102E0A00D212A6851233D212852F1233D2022D9CEA
:102E1A0030122EE54024F0401C7A0AC3E53F954B58
:102E2A006013401E24E2400D305405C254757F01E0
:102E3A0012BCB5DAE679BCE7D2E7F57F09877EC22C
:102E4A007722F40424E250ED80DE12DEF17F2A7E3E
:0C2E5A000E90A4BB12770275A6FFC210F8
:102E66001012137F367E08909F7C12770212DD1BAC
:102E760012DDFC0200F7D22112491112BCBF7F1EDF
:102E86007E0B90A3D812770212DD1B122EA77F3E6F
:102E96007E0790A10912770212DD1B12DDF6022BC6
:102EA6002AD215D21412BE4A120D4675B90575B945
:102EB6000212BE54D25512BD797F0012BC2E12BE2C
:102EC60054E56A600512BD4080F7857A62120E9459
:102ED60085BEBC85BFBD856BBE856CBF75B90575E6
:102EE600B90285BD6C85BC6B756A2012BE4A12306C
:102EF600DE12BE54756A0012BDF1E57064FE7034D0
:102F06007570FC854077854178851F797818797AC0
:102F160012C81812BCEE12DE1112BE54756A1012D7
:102F2600BDF17F087810797212C81A85627C855EB9
:102F36007D12BCEEC2152212486812308A745212F3
:102F4600DC03744D12DC03744312DC031230991255
:102F5600DC3E7441207402745612DC03122FE61212
:102F6600303012DC3EE53C12DBF6E53B12DBF6E5E3
:102F76003A12DBF612306612DC3E744512DC03129E
:102F860030CF12308A744712DC03744712DC0374A4
:102F96004112DC03123099122FE612DC3EE4307443
:102FA600010412DC0112DC3E9004C3E012DBF612CF
:102FB600DC3E9004E4E075F00A84AFF012DBF61212
:102FC600DC42EF12DC01AC5EAB7A1230ABAC5DAB2F
:102FD6005C1230AB12DC3E12DC3E1230CF02483FB0
:092FE6007875C23D122FF17878D4
:102FEF00D23D12DC3E128211303D05E51E12DC018E
:102FFF00E51D12DC01123073E51812DC01E57D20AE
:10300F003D01C4540F12DC0112DC3E303D09744502
:10301F0030170274578007744E301702745302DC56
:10302F0003207408123066123066802775A704904B
:10303F0004BFE0FCE0FB7A1B125371783212551378
:10304F001253391230709004C1E0FCE0FB12533977
:10305F0012307075A7002212DC3EE4F51AF51980C4
:10306F000D12DC3EE51C12DC01E51B12DC01E51A3A
:10307F0012DC0112DC42E51902DC01742412DC03BC
:10308F00744712DC46745002DC0312DC3EE53D123D
:10309F00DBF6E53E12DBF6E53F02DBF612826D1240
:1030AF00DC3EE51D12DC03781CE612DC0118B817B4
:1030BF00F812DC42E412DC0112DC3E744D02DC0338
:1030CF00C038742A12DC03D03812DC1D02DE1178EE
:1030DF00107F0EE4F608DFFCF564F565F567F5681B
:1030EF007515FC751AC0751DC075664075694075FC
:1030FF004A0112BD9930550302319412BD40E5715A
:10310F00B510004002F510E4F511E512207502E547
:10311F0013C395795006207545857913D3E57A95B4
:10312F0014E5156480FFE55E64809F400C857A147A
:0E313F00855E15857B16855F173074B3C2D18F
:10314D007864797312317278677976123172D2D1CF
:10315D0078187973123172781B79761231728091E9
:10316D0085791280B9D3E7960809E7960809E664D0
:10317D0080FFE764809F20D101B3400AE7F618195C
:10318D00E7F61819E7F622E51AB4C00E7873791828
:10319D0012C8187873796412C81878187964C2D176
:1031AD0012320574181256DE8E47AE1EAF1F781BF5
:1031BD007967D2D1123205C3E51F9FE51E9E5004DB
:1031CD008E1E8F1F7EFF7FFFAC1EAD1F12547C7AAB
:1031DD0004EF8AF0A4E5F0CE8AF0A42EFEE435F0DB
:1031ED00BEFF011E60051460057EFF8E1F22EE7E60
:1031FD000020E7F77EFE80F3C3E697FB0809E6970C
:10320D00FC0809E697FD1818191930E7031255FE49
:10321D00C3EB33FBEC33FCED33FDEB33EC33FBED68
:10322D0033FC30D105AA4712539A0BBB00010C7524
:05323D001E03751FFFD8
:10324200EC24FC40048C1E8B1FE627FB0809E637A2
:10325200FC0809E637A2E713F618EC13F618EB138D
:10326200F62210131978B5E624FA401AE57124F60D
:103272004008E57924F6400280360606803212DEE6
:103282000DE59030E2DF753612D22EE4F534F55AB0
:1032920012BEA51232B5C219C257122CF4129146AF
:1032A200129173D212853F4B754C00205E02D228D8
:1032B200022CECD214123304E6F008DFFB857A62AA
:1032C2001232FA7570FE783A797112C81812BCEE91
:1032D2001232FA85627A855E7B120E8A85BC7E8501
:1032E200BD7F7570C012BCEE123304E0F608DFFB3E
:1032F20075A700D254C2142274FF7870F608B88001
:10330200FB2275A7049004F078707F1022121EFA37
:10331200122C7412DEF112DD1BC258C259754A0119
:10332200753901756A2012BD991256DC8E47C2109A
:10333200D211D214D21212BEA51291461291731258
:10334200D99275A6FF753609753200E59020E2061E
:10335200E5352405400CE5905405701FE53524E25F
:103362005019C211C21212DEF112DD1BE4F535F55D
:083372002F7E0612DE09C202E3
:10337A00022005C221E54AB40202D22112BD9912E5
:10338A00A68530260F125A9812852F753606E5360D
:10339A0070FCC22612852C1233D2E54A20E021B4F1
:1033AA000209753900E53670F9808CE53960FAFD55
:1033BA0024E24002053912BD992026C9DDF880E9C8
:1033CA0075390080E475370410003A1001161002AE
:1033DA0016E52F5407600312B99020783D20790A28
:1033EA00207A1F220235C802351CE53760091460AD
:1033FA00091460090236740235E7023645C27902B9
:10340A00369102354FE53724FC500FE537640760E3
:10341A000302370C0236D00234E62011FAE5902076
:10342A00E2028056753400201203D2132278A9E6EC
:10343A007017C226767DE5377005106B02D26BD203
:10344A0077753614D22E02BE9AE53760431460406F
:10345A00B40227200B24E6249B401F2414501C127C
:10346A00914690A3AB7F207E0812770212DD1B756E
:10347A003608D22E78A9E624ECF622241940FB2439
:10348A001450F712914612917390A3B47F2980D7F2
:10349A002028E7E54824F640E1E5580460DC7F5D32
:1034AA007E10E6249B40D324145015C2330559C319
:1034BA00E55895595005855859D22690A39980A95F
:0434CA00241940B6CB
:1034CE00241450B2E55960021559102606E55960CC
:1034DE0002155990A3A2808D10780122753900E54E
:1034EE003424384007754A0175340022700AE54AC3
:1034FE0030E0F2754A0280F0146008754A061291A7
:10350E00738006754A0412914675390180DA3029A6
:10351E0009C229D22A7559008005302A1BD22912D8
:10352E0086FA1286C8E53524AF400475340022753C
:10353E003700C229C22A80F3206841302703D26A9D
:10354E0022D2221238A812DD1B107A0122E5342471
:10355E00384007122CF475340022700FAA37122C43
:10356E00F46A70F27401122CF580EB04122CF5241F
:10357E00FC50E3E537B40706D22880DA8036C2283D
:10358E00E53724FC2324BEF879C4E7F9A74809A738
:10359E005979C4E8F78648088607E537B4050575F6
:1035AE004818D236122B838F59E53764067002D233
:1035BE000702356412388402382EE537601B14601A
:1035CE007614600F146009E53724F9400902378636
:1035DE000236740236BF023753D223124096107948
:1035EE000122E534243840077546017534002278EF
:1035FE00D87020304A0BC24AE624F85004B24380F9
:03360E000AD24A93
:103611007614E54624FE40DDE54660D9154680D89E
:10362100B600D5B40500500C04F54624FA50C9750E
:10363100460580C424F95005127B5B80BB100FB88E
:10364100D20F80B4D223E53464C8600312409610CF
:10365100790122E534243750097011105B32D25BB5
:10366100802E100802D2081240968024100C21D21C
:103671000C801DD22312409610790122D24BE534E1
:1036810024374010C258C259201105D22E75360771
:103691007534002224FD401524037006D258C25906
:1036A10080EEC258D2591460E7D25880E3120E71ED
:1036B100E5BCB2E7F5BC79A1F7124EE680D278B845
:1036C100A65E08A67A2011C8753605D22E80C130B3
:1036D100122B128734055BE55B75F00B84E5F0F581
:1036E1005BE55A24F64009E55A955B5003755B008A
:1036F10012873812DD1BE5346003D534D2753400EE
:1037010022D229D22A75480A0237F4C2401007F1A1
:103711003029030237F41286F612870A102A1BC2D7
:10372100330559C3E558955920E7025008755900EA
:10373100E548B41816E558B4FF0375590012871E01
:1037410012DD1BE5346003D534C122D22A1286FA78
:1037510080EE301223128734155BE55B30E70C7580
:023761005B0A01
:10376300E55A24F64003855A5B12873812DD1BE5C0
:10377300346003D534DA75340022D229D22A75484D
:1037830017804CC2401007F22029441286F6128794
:103793000A102A22C2331559E55930E71C855859B6
:1037A300E558B4FF03755900E548B41802800AD2FE
:1037B3002A1286FA800E855859E558B4FF037559C5
:1037C3000012871E12DD1BE5346003D534B52220B9
:1037D300106220115F7F180548E54864187008F5EA
:1037E3004830270375480A122B4F303C2DDFE88001
:1037F3002620105A2011577F181548E54830E70551
:10380300754817800A640970063027037548171234
:103813002B4F303C05DFE275480A122B83125A36D0
:10382300E532244C50051286C8800312866E753427
:103833000002DD1B12386B7F15E5486B70048A4864
:1038430080020548122B4F303CD0DFED80CC12387C
:103853006B7F15E5486A70048B4880021548122B6C
:103863004F303CB6DFED80B27A007B09E537B40414
:1038730001227A0A7B17B40601227418FAFBF54871
:103883002275A704758307E559C4F582E0E0F57353
:10389300E0F574E0F575E0F576E0F577E0F5787539
:1038A300A700025A36E59020E23EE534243750382B
:0638B3001238EC1238C9C6
:1038B900205E4F7F2C909D20123933909D29806A7C
:1038C900E534243775F009A42435FF205E0624BEAB
:1038D90050027F3EEF249B50027F627E3274891230
:1038E900D4DD2275A7049000317E087F3AE4F0DF29
:1038F900FDE5822446F582E43583F583DEED75A77F
:1039090000227F2C120E6CE5BD12391CE5BE12395E
:103919001CE5BFF8C4123922E8540775F009A490D0
:103929009D0E2582F58250020583EF2409FF027658
:01393900F09D
:108529000285E312DEF1E53724FC40F4B4FE1420A1
:10853900110EE590F45407600122E532247450EFDE
:10854900028E2312DEF112D68012D71212CF5D12DB
:10855900D29E12D0E77E197F3612D03B12DC4B1225
:10856900D051C206E53760051460338053C23A1210
:1085790086871241591242EE1245D41264F41265EB
:108589001C123E04E54864186009E54824F65003C6
:108599001246BF128DB912CDE21241F48014D23ABB
:1085A9001286AD1239421241C312C968128DB9122D
:1085B900CDA3125D7712D759125848125B47801222
:1085C90012869312C8A512D82912C937128DB91269
:1085D900CDBA30101112CFEF800C12DEF1E537243D
:1085E900F9401E1286703022091238A8E53470024B
:1085F900C222302309124096E5347002C22302DDFB
:108609001B121DF375170012DA3C7F1212C9F030E4
:10861900124A75100075A704758306125AF1E51000
:1086290075F009A42415FFF5177E00E512602F7572
:10863900F06484E5F00F12D42D1F7E0EE51112CFE0
:10864900A5751623125CAD0510C3E55A95104006B1
:10865900E51024F550BF3012031287388088745D05
:1086690012D4DD80D5C249302905121DC9800312F3
:108679001DF3909F4212874B202A7602871E3012E3
:1086890023305E2030501D028A2F301217305E06CB
:03869900200B11A2
:10869C0002909012C9E97F1712DD9175172002DA4A
:1086AC003C12D5F712D59830121120510512D6571D
:1086BC00800612CD3D12CB1D1251AB22E4FEFFE51C
:1086CC004824F6400D90A3E01277357E16E548025B
:1086DC00D498B40E0690A3E602773590A3ED1277EA
:1086EC00357E12E54824F702D4337D20800C7D3F83
:1086FC00302A077D633029027D3C7F0080247D2059
:10870C0080127D3E800E7D3CE54975F007A4240661
:10871C00800A7D3FE55975F007A42409FF640270B7
:10872C0001FF7E1CED02D4AB7D2080027D3FE55B1A
:10873C0075F009A42416FF7E09ED02D4ABC24912D0
:10874C0087AFB4FF01227510001287C67920E03084
:10875C00E702792F3049171211AEFAB40408E5106C
:10876C00700C79658008EA14651070027923E97E33
:10877C001812D4AB7E20E51230E708909F7C12775C
:10878C00358016E51112883C125D0D201005201164
:10879C000280063012031287EE0510C3E5589510BF
:1087AC0050A7227E207F001277351286C87E007F6C
:1087BC000690886E12D509E5582275A704758307B3
:1087CC00125AF1E51075F007A42409FFF5177E0085
:0B87DC00E51212D4AB7805EE2404FE79
:1087E700E012D4ABD8F6221288F612890CFD7C0071
:1087F700AE1CAF1B12546FBE003A8F00C3E57A95CB
:1088070013FFE55E9514FE402B7C007D2812547CF7
:10881700C3EF98401F75F0058404FB24F950027BD1
:10882700067E2CAF170F12DE360F12DE360F12DE62
:10883700360EDBEF2264B4602464B475F03284C072
:10884700F012D498CE2404CED0E075F00584C0F0A1
:1088570012D498CE2404CED0E02302D49890886A0C
:108867000277352D2D2D000140FFFFFFE0FFFFFFB1
:10887700FFC25030123F20283CE558F460372048AB
:1088870003200931D250E559F51030330665586099
:108897000205101288C012891C75A7049006DCE532
:1088A70012F0E511F0E517F0E510F075A704900652
:1088B700E0ECF0EBF075A7002275A70475830712AB
:1088C7005AF17813E0F608B819FA9006D07811E64D
:1088D700F008B819FAE51CF516F0E51BF515F012C6
:1088E70088F69006DAE514F0E513F075A70022750F
:1088F700A704758306E51023541E24B0F582E0F51E
:1089070013E0F51422120E71E5BD2487E5BD923BF5
:0289170050020C
:1089190024912212890C75F005A485F012F511E451
:10892900F519FEF51CF51D12BE4AC23DC2567F3C23
:1089390012CA93303D05751900807DDFF3E559654D
:1089490058700A301007EE24D35002D2568C1B8D72
:108959001AE519FD24E250DEAE1CAF1D7C0012544D
:108969006FEFF51924F650CEAC1BAD1A12C9D820F9
:10897900D1108E048F05E51975F0A7A4AEF0FF128A
:10898900546FAC12AB117AA012539AEB33FBEC3350
:10899900FC20D11AEF9BEE9C5014C3E51213FCE5A1
:1089A9001113FBC3EF9BEE9C4004AC06AB072048B8
:1089B90007203B048C128B119006E2E519F0128A0C
:1089C90004AC16AB157AC8125371A912A811125525
:1089D90015ED7005EC249E50057C807B0822C3E5CB
:1089E9007A305602E55C9513FFE55E305602E55D87
:1089F9009514FEC3EF9BFBEE9CFC22AE16AF157CD3
:108A090000E519FD24F6501A12546F7C007D0612F8
:108A1900534F7C007D0512546F8F10EEF51724E932
:098A290050037517FF2212C9E980
:108A3200128A4C128A8F12D24D128AB5204809121C
:108A42008BA3128BD3028C3680747F177E20204832
:108A52000E748A204D101258B5500E742F80077470
:108A62006A305F02746712D4DD75A7049006D0786D
:108A720011E0F608B819FA7F177E00781275190509
:108A8200E60812D4DDEE2406FED519F42275A704F9
:108A92009006D8E0F516E0F515E0F514E0F513E0E0
:108AA200F512E0F511E0F517E0F510E0FCE0FB75DA
:108AB200A700227F187E26AC14AB1302D2DF9006E9
:108AC200E4E0F51CA3E0F51B7F2A304E13120E677B
:108AD200E5BF90A44AB4010390A6441276F0804206
:108AE2000F7E00745312D4AB9005CBE0F830E7054B
:108AF200E53F30E0091F7E00E8540F12D4C3900412
:108B0200EEE0FEF51EA3E0FFF51F128B4BE51E24DF
:108B1200E9500C7E06742B12D4DD7E0C12D4DD12C9
:108B22008B7BC20375172A751627125C7C202415CD
:108B3200205F15D2037F2A7E1E908B69304E0390F0
:108B42008B7202D509205FEB227C007D3C12547CA3
:108B5200A805EF7F2A7E0812D3E67E12743B12D458
:108B6200D97E14E802D3E00707384C9EBAF2643883
:0F8B72000707387CE6C2E67C38AC1CAB1B7A48A0
:108B8100305D027A27125371A91EA81F125515EDE7
:108B91004C60027BFF7F207E28EB12D3EC7E3902F2
:108BA10091237F2B90A3F3127733E517F46022AE64
:108BB10017AF107C007D3C12547CA805EF7F2A7E04
:108BC1000C12D3E67E16743B12D4D97E18E812D368
:108BD100E022AE12AF117C007D0A12547CA805EF91
:108BE1007F207E3012D3E67E3A742C12D4DD7E3C97
:108BF100E812D4C30F7E29744502D4AB7485800773
:108C0100748720560274867E2912D4DD30170774CA
:108C11002D7E3A12D4DD227C007D0A12547CA805F7
:108C2100EF7F2A7E3012D3E67E3A742C12D4DD7E99
:108C31003CE802D4C3128D67E54824F65005128C36
:108C41001880B9E559046558600D128C18128BFD16
:108C5100E559655860AA22A217923D8E1E8F18858C
:108C610015179006D0E0F51185581015101245B46E
:108C7100C3E51195105002F404F924A65005C374FC
:108C8100B399F9E975F00584F924EE500279119050
:108C91008DA7E993F5F0120920E5CC7004E930E7DE
:108CA10002747F23A4A9F0E51B2517FDE51C3516E9
:108CB100FEC3ED99F515EE9400F51675A7007583C1
:108CC10006E55823541E24B0F582E0A3F513E0F520
:108CD10014128D67203D2C201729120E71E5BD2439
:108CE10087E5BD5002249175F007A4FB9518E5F0C6
:108CF100951E400FEB9FE5F09E4008EF9518EE950D
:108D01001E500EA23D9217AE1EAF18128C18028B88
:108D1100FD306B10128D04E53F20E00774867E2242
:108D210012D4DD2275A7009006E0E516F0A3E51543
:108D3100F0128C18128C0174857E2312D4DD8558B3
:108D4100101288C0128A4C128A8F8C168B15128AC7
:108D5100B51289CA1288B212D24D9006E2E0F51915
:108D6100128A04028BA3C3E57A305602E55C95139F
:108D7100FFE55E305602E55D9514FE921750031231
:108D810055E6AC16AB157AC8125371A906A807129D
:108D910055157E037FE7ED700CEB2418EC34FC4095
:108DA10004AE04AF032200172E43576C8092A4B681
:108DB100C5D3DFE6EDF3F8FD305E4F30504C75A7BB
:108DC100009006E0E0A3FCE0FBECA2E79217402054
:108DD10024FE50047F3B8022AE04AF037C007D144F
:108DE10012547C74542F2017029F9FFF7462800CD1
:108DF1001255F6EC24FE50E07F6D743D7E0012D4D6
:108E0100AB7E017D197C03128E0C227F3D12DE3672
:108E1100EF2DFFDCF822E537B40206E534243750A4
:108E2100292212DEF112D68012CF5D128FA312C851
:108E31003312CDCA128FFB125B477F207E2B12D0DB
:108E41003B12D71212DC4B1238A812D173128ED1F9
:108E510012514502DD1B20041EE579FD24A05002BC
:108E61007D5FED24CD401E744520750C2DFFF5125C
:108E7100128EA61FBF44F922C39DFFF512128EA6C2
:108E81000FBF46F92220750EED2413FFF512128E45
:108E9100A60FBF78F922C374779DFFF512128EA633
:108EA1001FBF12F922EF24BA40082433FCC37432E5
:108EB1009C1404FC24D750047C238009EC2375F016
:108EC10005842413FC7E0512DE360EECB506F8226D
:108ED100E59020E206E53424374003128E577F45A2
:108EE1007E047D1212DE360EDDFA7F437E0074644D
:108EF10012D4AB7F4F7D12128F8C7F3B7D12128F6C
:108F01008C7F597D16128F8C7F317D16128F8C7F4D
:0F8F1100637D1A128F8C7F277D1A128F8C7F6DD4
:108F20007D1E128F8C7F1D7D1E128F8C7E057F19FA
:108F300012DE360FBF72F97804E57924CD5002783D
:108F400009E8305C0123F87F1B128F7B7F6B128F47
:108F50007B18305C01187F25128F7B7F61128F7B1D
:108F600018305C01187F2F128F7B7F57128F7B1870
:108F7000305C01187F39128F7B7F4D7E00E875F0E1
:108F80000A847004E802D498E802D433EF651260D2
:108F90000C7E04EE20E00712DE360EDDF62212DE35
:108FA0006680F790A50A7F287E2C1277357E3B12CB
:108FB000D2F6AC5EAB7A7F307E19C23D12D33590CB
:108FC000A3F77F5D7E2D12773578B9C3E57A9618C1
:108FD000FBE55E96FC7F507E19D23D02D335E5114C
:108FE00064B4700122E51112DCBB7831790F7D0B7E
:108FF00012DDB91F1E90908B02D509E5716012E554
:109000007012DCBB7831790F7D0412DDB50DBD0A1D
:10901000F97F011290637F1D1290637E2312906D81
:109020007E3F12906D7E247F171290777E397F02EB
:109030001290777E247F071290817E397F1C1290D8
:10904000817E317F0212DE367F1C12DE367F0F7E7C
:109050002412DE367E3E12DE367F0C7E2E90D7FE48
:1090600002D5097E2A12DE360EBE39F9227F081299
:10907000DE360FBF17F9227D0612DE360E0FDDF940
:10908000227D0612DE360E1FDDF9220303E0A0E08A
:1090900012C9E97F18909D5E1277337F217E01749B
:1090A0004112D4AB7F2A7E01745312D4AB9005BE1B
:1090B000E0F51AA3E0F519A3E0F51EA3E0F51D8580
:1090C0001A1C85191B751720129140E519251DF5ED
:1090D0001BF51DE51A351EF51CF51E751729129195
:1090E000409005BA129130AC1AAB19751720129046
:1090F000FE9005BC129130AC1EAB1D751729EC70AB
:1091000006EB24CD4001227A48305D027A271253C3
:1091100071125515ED4C600122AF177E07EB12D38B
:10912000927E1A0F90A5CD305D0390A5D0027735C1
:10913000E0FEA3E0FD12BFA0C3EB9DF8EC9EF92278
:10914000751627025CAD12BFA075A7049005B47810
:10915000737F06E6F008DFFBECF0EBF0E0E0E0FC0C
:10916000E0FDE0FEE0FFEF2DFFEE3C9005C0F0EFEC
:0B917000F0801275A7049005BAE0FB28
:10917B00E0CBF0EBF0E0E0E4F0F075A7002275A790
:10918B00049005B478647F06E0F608DFFB75A70052
:0E919B00125EBC9005BEE51CF0A3E51BF022A1
:10393A00D23C799E77008002C23C12BE4AE4F5105E
:10394A00F511F512F513F514F515F516F517C23D2F
:10395A00123C8A203D1F123C8A203D19E51F30E5A2
:10396A001130E40E1239B1303C08799EE724F55043
:10397A000122D510DBAE14AF157C00AD12125449EA
:10398A008F55AE16AF177C00AD1312546F125670D6
:10399A007E00E55530E7011E2DFFE43E30E7027F49
:1039AA0000740A2FF55622C235E51CAF1DBFFF056C
:1039BA000FD235F404FABF003F532CF8E518AF19BB
:1039CA00BFFF050FD262F404BF002D20E72A205B57
:1039DA000123FF24AA4021E51AAE1BBEFF050ED221
:1039EA0061F404BE00128547F0A4E5F020E709203F
:1039FA005B0123FE24AA5001227C807B8030516621
:103A0A00302163C006C0078AF0E545A4AEF0FFE5A1
:103A1A0056205B011375F009A4ACF0FD12546F74C3
:103A2A00FFBE0001EFFA24C050027A3FD007D00649
:103A3A00E55212DCBB303504B2D5B2D1EA8CF0A41F
:103A4A0030E70205F0748025F020D10495F095F056
:0A3A5A00FCEA8BF0A430E70205F04F
:103A6400748025F030D50495F095F0FBC3EC2F203D
:103A74006203C39F9FFFEB2E306103C39E9EFE2013
:103A84003C64200C05123B1E4064123B00405F1254
:103A9400DE36E51EFD24FB50550E12DE36ED24F60F
:103AA400504C1E1F12DE36ED24F150421E0F12DE62
:103AB40036ED24EC50380F12DE36ED24E7502F1F7C
:103AC4001F0E0E12DE36ED24E250231E0F0F12DEFF
:103AD40036ED24DD50180E12DE36ED24D8500F1EBC
:103AE4001E1F1F02DE36123B004003799E0722E9A7
:103AF400242AFFE82461FE123B1E401DEF2460408F
:103B040018243F5013EE2460400F243F500AEF2442
:103B1400D6FFEE249FFEC322D322532CF8432C0459
:103B2400EE10E706D2E7F404D261FE24D340EAEFB4
:103B340010E706D2E7F404C262FF24D340DBEFB5FA
:103B440006005003CED26070057480FE8062FF24AC
:0D3B5400FD5060903C0A938EF0A4AAF0335F
:103B6100CA33CA33CA33CA33CA33FA903C34938F47
:103B7100F0A433C5F033CA903C5593FB123BD29568
:103B810070500224B412DCBBEA8BF0A430E70205CA
:103B9100F0C3748095F020D50425F025F0FEEA8C61
:103BA100F0A430E70205F0C3748095F030D104250C
:103BB100F025F0FFC3227A01EE6F70097B16BF0278
:103BC100BB7A0380B7BF01047B0080B07B0D0A8004
:103BD100ABE52C540723C3903BDC73800E800E8031
:103BE10024801E8010800A80108012EB22742D9B8D
:103BF10022742D2B22745A9B22745A2B2274879B78
:103C01002274872B2274B39B22FFFFCCAA9280716E
:103C1100665D554E4944403C383533302E2C2A28B8
:103C2100272524232221201F1E1D1C1B1A1A1918A7
:103C31001817178181818282838384858687898A87
:103C41008B8D8F90929496989B9D9FA2A4A7A9ACCF
:103C5100AFB1B4B400010203040405060708090A60
:103C61000A0B0C0D0D0E0F0F10111112131314145A
:103C7100151516161612BD8212BC10E4F5F7C2B264
:103C8100C2B2E5F7D2B264C022203D07123C767081
:103C910003D23D22056D056D12BC107D008DF7C26A
:103CA100B2C2B285F71F8DF7C2B2C3E5F79573F5BE
:103CB100188DF7C2B2C2B2E5F79574F5198DF7C246
:103CC100B2C2B2E5F78DF7C2B2C3E5F79576F51A40
:023CD1008DF76D
:103CD300C2B2C2B2E5F79577F51B8DF7C2B2C2B295
:103CE300E5F78DF7C2B2C2B2E5F7F51E8DF7C2B2A2
:103CF300C3E5F7957AF51C8DF7C2B2C2B2E5F78D2D
:103D0300F7C2B2C2B2E5F7D2B2543F30E50244C0C3
:103D1300955EF51D156D156DE51024784001227E25
:103D230000AF55EF30E7011E0512E51FA2E592D55E
:103D3300400EE515951EF515E5149400F514800B5A
:103D4300E515251EF515E43514F5147800E51E6018
:103D53000620D50318F404C39FF5F0E89E30E7016D
:103D6300220513E5F0A42517F517E5F03516F5162A
:103D730022303D03D23D22123C7660F8123C76603D
:103D8300F3E546600A123C7660EA123C7660E5058C
:103D93006D056D056D12BC107D008DF7C2B2C3E5D4
:103DA300F79573F5188DF7C2B2C2B2E5F79574F5BE
:103DB300198DF7C2B2C2B2E5F78DF7C2B2C3E5F708
:103DC3009576F51A8DF7C2B2C2B2E5F79577F51B72
:103DD300D2B2156D156D156D2230742412BE4AC210
:103DE3003D75101E123D74203D167902123E484067
:0A3DF3000CA806A907123AF34003DA
:103DFD0012DE36D510E422200F4030123D2006CFC2
:103E0D00304806200C03204FC6E546790260147930
:103E1D000614600F791614600A79361460057976E8
:103E2D0014701712BE4AC23D7896123D74203D0A99
:103E3D00123E48400312DE36D8F022532CF8AB1850
:103E4D00E519FC339262123E9ABC002BEB89F053BC
:103E5D00F00784FF24DF401FAB1AE51BFC33926192
:103E6D00123E9AAA4712539ABC000CEB89F053F0FC
:103E7D000784FE24DF5002D32274562F2062029F46
:103E8D009FFF741F2E3061029E9EFEC322500312AF
:103E9D0055F6E920E40122C3EC13FCEB13FBE920FA
:103EAD00E50122C3EC13FCEB13FBE920E60122C371
:103EBD00EC13FCEB13FB2274542F2062029F9FFF27
:103ECD00741D2E3061029E9EFE2279B4203249204F
:103EDD001D46EFB506009260AC06AB074004AC077B
:103EED00AB06903F26EC2304938BF0A4A9F0EC23B2
:033EFD00938BF0B4
:103F0000A429F9903F8693C9904086E52C540793E5
:103F100013E95001F490408EF9E52C54079329756C
:103F2000F0B484A9F022FFFFFFFF7FFF55553FFF4C
:103F300033332AAA24921FFF1C711999174515556E
:103F400013B1124911110FFF0F0F0E380D790CCC60
:103F50000C300BA20B210AAA0A3D09D8097B0924BF
:103F600008D30888084207FF07C107870750071CC6
:103F700006EB06BC06900666063E061805F405D15B
:103F800005B005900572000000000001010101016B
:103F90000101010102020202020202020203030302
:103FA00003030303030304040404040404040405D6
:103FB00005050505050505050606060606060606A9
:103FC000060607070707070707070708080808087E
:103FD0000808080808090909090909090909090A55
:103FE0000A0A0A0A0A0A0A0A0A0B0B0B0B0B0B0B2A
:103FF0000B0B0B0C0C0C0C0C0C0C0C0C0C0C0D0D02
:104000000D0D0D0D0D0D0D0D0D0E0E0E0E0E0E0ED9
:104010000E0E0E0E0F0F0F0F0F0F0F0F0F0F0F0FB4
:10402000101010101010101010101010101111118D
:10403000111111111111111111111212121212126A
:104040001212121212121213131313131313131347
:104050001313131313131414141414141414141426
:104060001414141414151515151515151515151505
:1040700015151515151616161616161616161616E5
:1040800016161616161600FFFF00FF0000FF002E82
:10409000B5875B2D5A88E537607414603EB40258CA
:1040A0007F347E12E5342437400810644B90A3CA55
:1040B000801AF89041E012D509E824FD501179A149
:1040C000E77E0590A20D20E70390A2170F803A2407
:1040D000040F7E2312D4CAD26480627F357E02E54B
:1040E000342437401410641090A10030081B12775C
:1040F000027E1A90A3C9801122700590A112800936
:10410000909D8B200C03909D9712770280C97F357C
:10411000E5342433402A2404501B7D0F600C7D1E9F
:104120001460077D3C1460027D78ED305D02C3139E
:104130007E2B12D3927E0090A11312770202DD1B18
:104140007E0524FE5005909F698009909D6E200F8A
:1041500003909D7A12770280E4E546604A14603C41
:1041600014602E14602014601290A601205D41900E
:1041700041D97F367E3412D509803C90A601305D4E
:104180000390A5FD802A90A5FD305D0390A5F980E0
:104190001F90A5F9305D0390A5F5801490A5F5302A
:1041A0005D0390A5F1800990A5ED305D0390A5E930
:0241B0007F3658
:1041B2007E331277357E3C7422305D02748302D4E2
:1041C200DD305D0890A5D9305BE4800690A5E12042
:1041D2005BDC90A5DD80D70508B28D8DB5BA0910DC
:1041E20006000A10F248922492249224F2480A10FD
:1041F2000600305E5220434F20284CE55864FF6091
:1042020046E54824F640407F3FE55804F9C23D1296
:10421200424A1211AE601AB404047401D23D75F020
:1042220003A4243CB5070A7E3A303D027E36124290
:104232004C0F0F0FD9D7E55975F003A4243EFF1296
:10424200424A0F0F12424A227E3D12DE360EBE4015
:10425200F922C248C249305E56202853E55864FF0D
:10426200604DE54824F640471211AE6042D249B48F
:104272000402803B1465597036D248304E31E559FC
:104282006558602B3074281242B7120E67E5BFB42E
:10429200011DE5BD20E618202416205F129006E4D9
:1042A200E0700CA3E024CE400624255002055922DA
:1042B200305FFC80E820113375A7009006E4E070BF
:1042C20028A3E0302402F404305F02F4042404F949
:1042D20024F74015E924FC4003D26C2270012230FD
:1042E2006C097536A7D22ED22FC26C22305E0830EE
:1042F2007405E558B4FF0122C244C24D780075A787
:0B4302000475830712463688188A1ED7
:10430D008E168F17C23EC23BE54824F6500302437A
:10431D00C7D23EE55860F7E8655970F22048EF12B4
:10432D00447C30D13BAE16AF17A818E54670551238
:10433D000920E5CC49604DD244E5CC7033E924CD5C
:10434D00402EE975F038A4ACF0FB12558512558559
:10435D00EBFDF5111243DD304D2CC206C23B8043FF
:10436D00E546705C120920E5CC7005E924CD50506E
:10437D00124F7C75A704758307A8181246368A1E3E
:10438D008E168F178037120E67E5BDA2E0B3923BF4
:10439D005011307428123AF34026A907A806D20608
:1043AD0012CA7A1243F91243F0124439890788066A
:1043BD001E1F90463112D509800630D103124411CB
:1043CD00A81808C3E55898400302430075A70022BA
:1043DD0074562F2062029F9FF9741F2E3061029E2A
:1043ED009EF822E51865586001227D057A00EA12D3
:1043FD00DCBB12DDB90A0AED24F240020A0AEA24F6
:10440D004C50EB22AE16AF17123EC41E303E021EAC
:10441D001EE51E12D4ABEE2404FEE51212D4AB3011
:08442D003E09EE2404FEE51334
:1044350012D4AB22E5186558603CC001C000C0121B
:10444500C0138518101245B4D013D012D000D00176
:10445500E510303B07C39570500224B412DCBB2035
:104465003B07AE16AF171243DDE5112402FD7A06B0
:1044750012DDB91DDAFA221211AEB40457E87054F0
:10448500120E85E5BD604D78C6A61308A61208A6CE
:104495002C12C82775A704758307751001125AC217
:1044A50012C8211510125AC21256DC8E628F631281
:1044B50057648B1C8A1B12C82D20320E12456420AE
:1044C5003B08D24D1266FF1244DA78C68613088679
:1044D5001208862C22120E85AABD7C027BB31253CC
:1044E5009A8C128B13AA1DA91F1253DCA91CA81B99
:1044F5001255158C1D8B1FAC12AB13AA19A91A12D4
:1045050053DCA91CA81B1255158C198B1AE56E25B1
:104515001AF9E56D3519F8C3E56E951AFBE56D9544
:1045250019FAC3E554951FFDE56F951DFCE5542566
:104535001FFFE56F351DFEE52C23652C30E206ECEB
:10454500CEFCEDCFFD75A7049005C2E8F0E9F0ECCF
:07455500F0EDF0EAF0EBF0DD
:10455C00EEF0EFF075A70022D23BC3E5649573C56E
:10456C00659574F564E5669575600404600822E54C
:10457C006424E0500822E5642420400122C3E5674E
:10458C009576F567E5689577F566E5699578600940
:10459C0004600122E566F48002E5668562F0A4748D
:1045AC00E025F04002C23B2212C82775A704758390
:1045BC0007125AC212C8210510125AC2C02C125A24
:1045CC00DBD02C891002C82D30125120064E7800F9
:1045DC0075A70475830612463630D139123EC4E5F0
:1045EC004624FE500A0E0F90462C12D5098026EA5E
:1045FC007007745D12D4A7801C75F06484ADF070E4
:10460C000FED75F00A847008E5F00E12D498800551
:10461C001EED12D42D08C3E55A9850B475A700228C
:10462C00030340A040030340E040D2D1E8C4F5822C
:10463C00E0FA797312468F30D146AF06532CF8ED61
:10464C00BFFF07F40460390FD262BF00331247C3B7
:10465C00402E797612468F30D126E5822403F582DE
:10466C00E0F512E0F513EEA2E713FEED13BEFF0723
:0A467C00F404600C0ED261BE0006CB
:104686001247E0400122C2D122C3E09709FDE0971C
:1046960009FEE097600904700AEE30E7068007EE2F
:1046A60030E703C2D122E546600E14600BF9EDCE69
:1046B600A2E713CE13D9F8FD227C007B44E54660C1
:1046C600207C007BCC1460197C017B981460127CE2
:1046D600037B3014600B7C067B601460047C0C7BCF
:1046E600C08C148B157AE9125371A8471255138C96
:1046F600168B1775C70075C6047510DF75B901E509
:10470600BC20E76FF51385BD1205C605C675B90150
:10471600532CF8C3E5BE9573FBE5BF9574FC05C63F
:1047260075B901E5BC9575FD5005D2621255FEC3FB
:10473600E5159BE5149CE49D40338C198B18C3E565
:10474600BD9576FBE5BE9577FCE5BF9578FD5005F2
:10475600D2611255FEC3E5179BE5169CE49D400DFC
:104766008C1B8B1A12478AE5322428401305C6E5AE
:10477600C68006E5C62404F5C6700205C7D5100135
:0F47860022024702AE19AD181246ACED1247C31E
:10479500AE1BAD1A1246ACEE13ED131247E0123EF6
:1047A500C4E54624FB50080E0F90463102D5091E7C
:1047B500E51312D4ABEE2404FEE51202D4AB75F07A
:1047C500067FFDA946B9000575F0027FFF84C5F097
:1047D5002F500205F0C5F0FF24DE228547F0A430F6
:1047E500E70205F0E5F0A946B9000280050475F079
:1047F5000384FE24E022E537B4020122E537700286
:10480500D23964027002C239E53724FC799EE7602B
:1048150005640B600C22D27E20081E401C107F1000
:1048250022D27F2008134011107E01227537012204
:104835007537002039037537022275F9FF75FB00BE
:10484500800E75F9FF75FBFF801C2053F512487D1E
:10485500759E85759D2D801412487D759E84759D68
:104865002D800912487D759E83759D09C2AC75988A
:1048750052C26DC26EC26F2212166EC253E4F5F9B2
:10488500F5FB30340215FB22D2A47F3212DE13C2AF
:10489500A412D99212DD1B12DDFCC214C2151248F6
:1048A5003F74C012DC4674A312DC03748F12DC0360
:1048B5001248D374C012DC4675A7049048DD7F10FA
:1048C500E49312DC03DFF91248D375A70022E5381B
:0548D50012DC0374CAAF
:1048DA0002DC03A29494859C8080808080818380FE
:1048EA00819E8075A60A12489FD269D2ACE5A62499
:1048FA00FA500C306DF712DB98B4E0F1124935C268
:10490A00ACC26975A6FF22D21EC274C273E4FDF559
:10491A0071F570C22D12483FD2AC12DB98C5F07007
:10492A0005DDF7C2AC22C5F0B4E0EFF538E4F532A4
:10493A0012DB93A2E19273A2E2927475A704900427
:10494A00B4F012DB93C2D1124B1C20690330740BF2
:10495A008D758E748F73E514C4F57D124B9C124BC2
:10496A001C20690330740C8D788E778F76E51425B8
:10497A007DF57D124B9CD2D1124B1CEEF0F55DEF0A
:10498A00F0F55C207303E4FEFF79BCA70609A707CC
:10499A0012DB937D0A124B898F71EE60037571FFEA
:1049AA007D14124B89C22DED24F150010F240A50B7
:1049BA0002D22DBFB4027F008F7012DB93F054072E
:1049CA00C52E54F8252EF52EE571700EE4F571F515
:1049DA0070C22D9004BFF0F0F0F012DB93E538605E
:1049EA0009D21EC27412AEDF8005C21E12AEDB12DD
:1049FA00DB93B4E1FA75A7049004C412DB93F012B6
:104A0A00DB93F0F53A12DB93F0F53B12DB93F0F50A
:0B4A1A003C12DB93F0F53D12DB93F043
:104A2500F53E12DB93F0F53F12DB9312DB93B4E214
:104A3500FA12DB93F07E0C12DB93FF12DB9312DB91
:104A45009312DB9312DB9320E1027F00EFF012DB80
:104A550093DEE412DB93B4E3FA12DB93FF12DB93EC
:104A6500CF60027F7F9004E4EFF0E4F012DBC390A7
:104A750004D8124B8912DB93B4EAFAC2AC75A704C9
:104A85009004DAE561F0E560F0E55EF0E57AF0E5E1
:104A950079F0E52EF0E55FF0E57BF0E551F0207467
:104AA50012E4F571F5709004B4F09004BDF0F0F0E7
:104AB500F0F0F075A70078ABA63A08A63B08A63C2F
:104AC500120E7BE5BF253D240C75F0188478AEA643
:104AD500F0186005640260182216E670121816E6D2
:104AE5007004760C181678ACE6904B0F9308F622F6
:104AF5000618E608904B0F930466700D76011806AC
:104B0500E6640D70047601180622001F1D1F1E1F86
:104B15001E1F1F1E1F1E1F12DB93FC12DB93FD12AF
:104B2500DB93FE12DB93FFECA2E692E7921713FCF0
:084B3500ED92E713FDEE92E79B
:104B3D0013FEEF92E7301701F4F513ECA2E713FC27
:104B4D00ED92E713FDEE92E7301701F4F512ECA2AA
:104B5D00E713301701F4F510ED92E7301701F4F576
:104B6D00111255A620D10E8C1C8D1D8E1E8F1F125D
:104B7D00B2E71255A630170312B2C12212DB93C34E
:104B8D0013FEF012DB9392E7FFF07C0002547CAC35
:104B9D001CAD1DAE1EAF1F30170312B2C1ECF0EDF0
:104BAD00F0EEF0EFF022124BBC0202C612BC4FC267
:104BBD00101248F07F5A7E0590A3D812770212DDAD
:104BCD001BD214D215C255122CEC789F7680087624
:104BDD000012BC8F1232FA7570FE853A71853B72E8
:104BED00853C73853D74853E75853F7612BCEE120E
:104BFD0032FA7570C0757B03757A54E4F57FF57ED6
:104C0D0012BCEE751421751348755F01757B007527
:104C1D00750475745275780175776CE4F57DF551F1
:104C2D00757F0190DF5C85836E85826DC23D124C70
:104C3D009A851C1D75A6FF305505C221022EA7129F
:104C4D004C9AE572A2E59275A2E79277D274D2736F
:104C5D00E51275F008A4AEF0FF2075031255E612AB
:104C6D00C77712C7C0124D1DE51C251D13F57185A3
:054C7D001C1D12BC67C4
:104C820012BCBF757F02E56A70B57F5A7E2FE5417F
:104C920012D39212DD1B80A7856E83856D82C25569
:104CA2007873124CFE7876124CFEE493F570B4B42D
:104CB20002D255A3E493F51CA3E493F512A3203D7D
:104CC2000FA97BE493F57BC399502A20E702055F85
:104CD200A385836E85826D103D16D23DE582240543
:104CE200F582E43583F583E493F52654F0F57222D8
:104CF200E526C480F630E7D8155F80D48601E493B8
:104D0200F6A308C399500A20E70606B60002080671
:104D12002230E70616B6FF0218162230750DE5138B
:104D22002579F513E43514F514800DC3E51395794F
:104D3200F513E5149400F514AE14AF137C007D0A4C
:104D420012547C8E5E8F7A22124DDF851617203D1B
:104D520001227F5A909C831276F07F64E5166404E8
:104D6200700C909C9B12773312DD1B02DDF6909C37
:104D72008F1276F07F6E7E0890A5C9127702121EFE
:104D82000312DD1B7515B87514047F6E7E20C224D4
:104D9200A815E82404F9C23DE7124E27203D06E695
:0A4DA20012D4DD8008E6128460E8F8
:104DAC00A815F60515EE2406FED514DA851716128D
:104DBC001E5112DD1B10000510018D80F878B81201
:104DCC000E8F86BC0886BD0886BE0886BF124EE6CE
:104DDC0012DEF1120E8FC23D75160078B87F4B7E35
:104DEC000890A5C91277027E20E5BC12D4DD124EC4
:104DFC001E7E26E5BD12D4DD124E1E7E2CE5BE12A3
:104E0C00D4DD124E1E7E32E5BF12D4DD124E1E02D0
:104E1C00DD1BF608080808F618181824D0500524CD
:104E2C00F64001220516D23D2275C70375C6FE1247
:104E3C00766E124EE675C6FC75BC2675BD6475BEE5
:104E4C00A975BF70124EE675C6FB12766E124EE651
:104E5C0075C6FA75BC1475BD1475BE0075BF0C1201
:104E6C004EE675C6F975BC4E75BDBF75BE0075BFF7
:104E7C0019124EE675C6F875BC0A75BD7E75BE0076
:104E8C0075BF01124EE675C6F775BC0175BD23756D
:104E9C00BE4575BF67124EE675C6F675BC0275BD8C
:104EAC00AB75BE0175BF01124EE675C6F512766E76
:104EBC0075BE0275BF0A124EE675C6F412766E7593
:104ECC00BCE1124EE675C6F312766A124EE615C6B2
:104EDC00124EE615C6124EE615C675B90575B90221
:104EEC0022751500127D6775B901E5BC64816003FC
:104EFC001276510515E515242050E975C70375C6C2
:104F0C008075B90505C6E5C6241C50F5124F1E0266
:034F1C007BBDE476
:104F1F00F5C7F5C6742612766F75BD4E124F38124F
:104F2F004F35E4124F3512766F124EE605C6227FCB
:104F3F00357E00E54B12D4497E10E54C12D4497EE4
:104F4F0020E54D12D4497E30E54E12D449227F46DA
:104F5F007E00E56C12D4497E10E56B12D4497E2099
:104F6F00E56A12D4497E30E57F12D44922207401BC
:104F7F0022D24475A700758307E559C454F024075E
:104F8F00F582E0F51A244C40E7A3E0F512A3E0F513
:104F9F00131209208938120E67E5BDA2E0923BE596
:104FAF001A40069570500224B4F51A203B05D2061C
:104FBF0012CA7AE51A1250DFE5152437F51DE435CC
:104FCF0014F51CE5172437F51FE43516F51E85CCAF
:104FDF0012853813AC12AB137A0412536375380170
:104FEF0024FA401A05382402401405382401400ED3
:104FFF000538053824014006053805380538C3E55E
:10500F001A945A500224B4F51AC23BC23CC23D75E1
:10501F001B00A23B823C406D203B2CE51A75F0082B
:10502F00A4951BFBE5F0303D04940180029400FC35
:10503F005008EB24A0FBEC3405FC1250E6125095FF
:0A504F00923B40031250B8203C2CA5
:10505900E51A75F008A4251BF9E4303D010435F083
:10506900FAE994A0FBEA9405FC5004AB01AC0212E6
:1050790050E6125095923C40031250B8E51B253872
:10508900F51B5094203D04D23D808D22E51F251744
:10509900FEE51E35167016EE24914011E51D251505
:1050A900FFE51C35147006EF2491400122D3228EAE
:1050B900027C8A7B3B125371ED2402FE8F027C8AAB
:1050C9007B3B125371ED2439FF02DE361256CF8035
:1050D900311256C2804675F008A4ACF0FB75190070
:1050E900C3EB9468F9EC9401FA40080519AC02ABDA
:1050F9000180ED8C108B11531903E51920E0CD12B5
:1051090056C212513AAF05E51924FE50031255E66D
:105119008E168F17E51920E0B81256CF12513AAF03
:1051290005E5191460061460031255E68E148F15EF
:1051390022AC06AB07AA12A9130253DC125227208C
:105149003D4974857F227E0812D4DD7E0830173CE4
:10515900AC1EAB1FEB2418EC34FC402F125342E574
:105169001B60077F207E0812D4F87F207E10E51A85
:0951790012D4F87F237E17742E76
:1051820012D4D97F207E1BE51B7011E519C2E012F3
:10519200D4F8227F207E0E740A02D4F8E51975F045
:1051A200058475F005A402D4F8125227203D5E74DE
:1051B200857F227E3A12D4DD301753AC1EAB1FEB33
:1051C2002418EC34FC4046EC7033EB249C402E7ED9
:1051D2002D125219125585C0E07F2A7E2EEB12D471
:1051E200F87E39D0E0C2E012D4F87F347E3712DE86
:1051F200361E12DE361F12DE360E02DE367E30120A
:105202005219125585EB7F2A7E3112CE1C227F2A3B
:105212007E39740A02D4F87F2912DE660FBF34F990
:105222000EBE40F322D23D301266120E71E5BDF57C
:105232001C75F00AA4F824E15002781EE4FCFBFE7F
:10524200FFC23D12BE4A125293203D44D8F8751D4A
:10525200CEE51C146009751D9C146003751D6AC29D
:1052620017EC30E705D2171255F68C018B00E9488E
:105272007003D23D22EE7008EF251D4003D23D227D
:10528200AC06AB077A1C1253711255158C1E8B1F7C
:1052920022203D07123C767003D23D22056D12BCDE
:1052A20010E4F5F7C2B2C2B2ADF7F5F7C2B2C2B2BC
:0252B200E5F71E
:1052B400FAD2B230E4E3ED2FFFE43EFEE56D2408BC
:1052C400F56D12BC10E4F5F7C2B2C2B2ADF7D2B2BA
:1052D400EA30E508EB2DFBEC3400FC22C3EB9DFB2C
:0552E400EC9400FC2227
:0100030055A7
:10DF5C0069FC362E06FD69FC372F071169FD383038
:10DF6C0007FD69FD3931061169FE383107FD68FE80
:10DF7C003732091168FF373008FD68FF372D07115C
:10DF8C006800362909FE680036290C116801372B08
:10DF9C000CFF6801372F0A116802383009FF68023C
:10DFAC00372E08116803372C0AFE6803372E081128
:10DFBC006704373208FE67043633091167053535B7
:10DFCC0005FF6705353303116706362F02FF670619
:10DFDC00362B05116707362B07FF6707352F051101
:10DFEC006708353104FF6708332E0511670931289E
:10DFFC000700670931250A11670A35240B01670AE6
:10E00C003A240A11660A3C210801660B3D1E0B11CD
:10E01C00660B3D1E0C00660B3D200A11660C3B2165
:10E02C000CFF660C39220E11660C37231100660D9D
:10E03C0036240D11660D34260F01660E3226111191
:10E04C00660E32251401660F35251311660F37271E
:10E05C0016016610392918116610392B1502651135
:10E06C00392D11116511372E0C026512332F081141
:10E07C006512312F07026513302C0A1165132D29F7
:10E08C000E0265132A271011651429270E02651438
:10E09C002C290C1165153129080365153726071134
:10E0AC006515321F09036516411B09116516411CC4
:10E0BC0008036416461F081164164D2105046416E6
:10E0CC005922031164166425040563156A2407118B
:10E0DC0063156D23090663156C230D1163156C25EF
:10E0EC00130762146E2B151162146E2F1406621333
:10E0FC006E30161162136E30150761136F311211E9
:10E10C0061126F350F0761126F380D116011723A81
:10E11C000A086011763F0611601079420209600FFF
:10E12C007A3A0533600F7832040A5F0F742C01338E
:10E13C005F0E722B030A5F0E732E08115F0E743084
:10E14C00050C5F0D722C02135E0D6C2B010C5E0D19
:10E15C00622C05315E0D5F2B030D5D0D5E290833BE
:10E16C005D0D5F23030B5D0D5F1B01335D0D5A16B7
:10E17C00020A5D0D521B00115C0D4D26000C5C0E4D
:10E18C00462802335C0E3926040C5C0F2C2B08330A
:10E19C005C0F23320C0F5D0F172E0A335D0F0C2E04
:10E1AC0009105D0F043507335E0FB23C080F5F0F8B
:10E1BC00AB4209335F0EA43E070F5F0EA2430B3335
:10E1CC00600EA746120B600D9F490C73610C9C49A5
:10E1DC000F0C610B97460973610B8B440A0C610A97
:10E1EC008B420B336109843A080C6108823A043380
:10E1FC0061087934030C60086F2F063360086228BD
:10E20C00050C6008572505336008511F040D5F0885
:10E21C004E1B05335F08491B090D5F094120103760
:10E22C005F0938270D0D5F0A302F06335F0B2B3239
:10E23C00070F5F0B282F0A335F0B262E0E0E600C78
:10E24C0023361137600D1F3F160F600D18411277E2
:10E25C00610D0F320A13610D042B0633610D022E72
:10E26C00040E620D043A0231620E0343050D630D78
:10E27C00B1470113630DA94A000B640CA14D0511A4
:10E28C00640C9B44070E650B99490911650A944768
:10E29C00090D65098E49021365088848060D650845
:10E2AC0081400E336407793B130F6407722F187784
:10E2BC0064076D231A106407692911776407651CBC
:0DE2CC00080F63075D180B33630751190D30
:10E2D9000D630746220E336308402B110F6308387C
:10E2E900291837630932271B0D6309312B1477620B
:10E2F9000A372C0F0A620A3C280973620A441E0B6A
:10E309000C620A48150E33620B46190C0A620B4758
:10E31900260D33610B4C280C0B610B54251037610A
:10E329000B5E24170C600B63291A77600A66361492
:10E339000A600A68390B735F0A6C2C100A5F09724C
:10E349002015775F097422120A5F0873300F775F0F
:10E35900087639140A5F077D3816775F0785370F06
:10E36900095F068D3B0D735F058B4410075F048BB6
:10E37900490C735F048E3F0C075F03863604335FD5
:10E389000394280708600299300E1160029E400527
:10E39900076102A34A0C336101AA4810086201B15E
:10E3A90042127762020131150A6202062B13776362
:10E3B900020830110C63020B361277630310331114
:10E3C9000C6403182B147764032223110A640426AE
:10E3D90023107764042226110A64051C2715776423
:10E3E900051D251508640521271277640628270FBE
:10E3F9000764062F1D11776406350F140764063E5E
:10E409000A19776406401216086407431B117763DB
:10E41900074A22120663075228127763075A2713FD
:10E429000662075E2314776206612011076206649B
:10E439001E0E7362066A1E0E076206742110376289
:10E44900057828130661057A2F157761047A332038
:10E459000661047A301B7761037A281B0761037F01
:10E4690023187761028429160661028832177761B9
:10E47900018D371305610193340C7362009A2E09DB
:10E489000562009D2E043362009D370C0663FFA0D0
:10E4990040103763FFA844140564FFAF4612776440
:10E4A900FF014511056500043F12776500053E101F
:10E4B900076600073F117766000B430D07670110D8
:10E4C9003D117367011539120767021A321277670E
:10E4D900021A2C12076702192C107768031B2E0FDA
:10E4E9000668031F2C117768042729100468042E75
:10E4F9002A0F776705322F130467053330127767C0
:10E5090006362D140567063B291677670643231B34
:10E51900046706471E16776607491E150366074CEA
:10E529001B157766074C2217046607522214776574
:10E53900075B26150265066229157765066D291799
:10E549000165067529137765057D281A0265058217
:10E5590028187765047F1F160265048F2A117765CD
:10E5690003953211006602993D157766029C401C9D
:10E57900FF6602A13E1F776701A43F1CFF6701A741
:10E589004314776801AB4710FF6901B1490F7769F7
:10E5990001024911026A0207490D736A020B480C0C
:10E5A900056B030F480B336B03144A0D026B0419F7
:10E5B9004914376B051F491CFE6C06224824776CE9
:10E5C90006233F21FC6C07203023776C0721272184
:10E5D900FC6C07262420776C08292812FC6C082873
:10E5E9002C0F776C0927230CFF6C09251802316C55
:10E5F90009350F05FC6C094C1401116C09561D01F4
:10E60900FC6B095F2003136B086B2108FB6B087413
:10E619002509336B08772507FC6B0778210D336BC8
:10E62900077A1E0AFB6B077F220C336B06832E0ABF
:10E63900FA6B05853C09336B0489410EF96B048C2F
:0DE649003E10376B038D3C0FFA6B038D40C4
:10E6560013776B02904112FA6C01934110776C01AB
:10E66600984410F86C009B471A776D009F461EF879
:10E676006DFFA24519776EFFA14019F86EFFA640FF
:10E6860014776FFEAA4417FA6FFEAF4A127770FE30
:10E69600B34D18FA70FF024B1B7771FF054718FD43
:10E6A60071FF0942177772000E4012FD7200163D87
:10E6B6000C7372011B3510FA7201232E1577720244
:10E6C60029321AF872032C371D7772032F3014F88B
:10E6D600720336210F77710346190DF87103502026
:10E6E6000B33710353290EF87003572B143770033D
:10E6F600612712F870036F2911777002793017F7C6
:10E706007001803722777001843D1FF67000883FC4
:10E71600197770FF8D3F11F670FF933D0C7371FEF4
:10E72600973D0EF571FE9B3E0C3372FD9F4310F62E
:10E7360072FDA448127773FDAB4C13F573FDB14F10
:10E74600167774FD034F14F775FE074C127775FEA6
:10E756000A4510F975FE0E400F7776FF124111F843
:10E7660076001745167776001C4614F67601214288
:10E7760017777602263D17F3760229382177760336
:10E786002A3315F276032B3009737604302A07F004
:10E79600760439220A337604472110F07504512590
:10E7A60012777504552416F1750459210F777504EF
:10E7B6005F2111F0740463231477740468240EF245
:10E7C600740370230933740379270AEF74028030C7
:10E7D6000B33740185360DEF74018B3913377400D2
:10E7E600903D1BF075FF94441E7775FF984823EF04
:10E7F60075FE9B46207776FE9F4221F076FEA13F6E
:10E80600177777FDA44313EF77FDA747157778FDB4
:10E81600AA4915EF78FDAD4C157779FDB04D19EE87
:10E826007AFDB34D1C777AFD024E19F07BFD054F3C
:10E836001B777BFE094F24F37CFE0D531D777CFF6F
:10E84600114619F37CFF173F12777C001F3810EF33
:10E856007C00263613777C012B3115ED7C012F2B9E
:10E8660015777C02332513ED7C02392214777C025E
:10E87600402110EE7C0249210B737B02531F0FEBE4
:10E886007B02601E15777B026A2214EA7B017428DC
:10E8960019777B017B2D1AEA7B00833122777B0077
:10E8A6008A3320EB7BFF91371A777BFE953C1FEA74
:10E8B6007CFE983C26777CFEA74621EC7CFD9939A8
:10E8C60023777CFC9A3B1FEA7DFC9A3F1C777DFBF5
:10E8D6009A401EE87DFB9B3F20777EFA9B3F1FE612
:10E8E6007EFA9C431A777EF99E4717E57FF8A04A81
:10E8F6000E737FF8A34A0AEA80F8A548073380F822
:10E90600A94402EA81F8AE46041182F8B24C00E747
:10E9160082F80351021183F8085304EA83F90E4D75
:10E92600061183F914430CEC84FA1A400E1184FB89
:10E93600203F0AE884FC2540061384FC2B4008E6A9
:10E9460084FD3039073383FD36300EE483FE3C2BDD
:10E95600193783FE402A1EE783FE3D25187783FE7E
:10E96600371B16E783FF3114137783FF35170FE440
:10E9760083FF3E220D738200412C15E58200432C55
:10E986001A77820046251BE782004C201577810006
:10E99600552116E581005E2510778100682718E469
:10E9A60081FF72291E7780FF7A2E22E580FE7E3057
:10E9B600277780FE812B22E680FD85251C7780FD4A
:0DE9C600882618E281FC8A2F187781FC8DCD
:10E9D3003821E181FB903F287781FA924025E0813D
:10E9E300FA943D237782F9973C18E082F99A3F1510
:10E9F3007782F89E4412E083F8A347107783F8A741
:10EA03004A0CDF84F8AA4D133785F7AC5214E2851C
:10EA1300F7AF56107786F7B2580DE087F802560223
:10EA23003387F8055002E388F8094C051188F90C7F
:10EA33004E02E489F91052011189FA155004DF8955
:10EA4300FB1D45041389FB233304DE89FB292306BD
:10EA53003389FC2B1F05DE89FC2F23093389FD3302
:10EA6300280ADC89FD3B23103788FD471E0EDD880D
:10EA7300FD511E0E3388FD53200CDD88FD54210B00
:10EA83003387FD57200DDD87FD5C20093387FD5D4E
:10EA93002403DE87FD5B29013386FD592C04DE86C2
:10EAA300FD5D2C093385FD622F0CDC85FD652D0B87
:10EAB3003385FC672908DF85FC6722093385FC6BF6
:10EAC300210CDD84FC72280A3384FB783005DD8455
:10EAD300FA7C37073384FA7E390ADC84F9813B06F2
:10EAE3003384F8843F05DB84F8873F023384F78A55
:10EAF3003C04DB84F78D390A3384F6903908D985D1
:10EB0300F5923F113785F595430FD985F498440A5B
:10EB13007386F49B440AD986F39C440C3386F39C96
:10EB23004507DA87F29C47063387F19E4C0AD9885A
:10EB3300F1A251103788F1A65516D989F0A7571FAE
:10EB4300778AF0A9541BDA8AF0AA4D12778BF0ACBE
:10EB5300460DDB8BF0AC4906338CEFAB4D05DB8CFC
:10EB6300EFA95002318DEEA85209E28DEEA7530EA4
:10EB7300118EEEA75316E58EEDA44A20118FEDA05A
:10EB83004423E28FEC9C4821118FEB9A4A22E090B8
:10EB9300EB95411D1190EA8E391DDF90EA893621EC
:10EBA3001190E9873223E590E9852C2C118FE87DBC
:10EBB3002A26E08FE8762124118FE8662122E08F50
:10EBC300E856221F118EE947201DE08EE9392116F0
:10EBD300118EE9302518E28EEA2D2917118EEB30BC
:10EBE3003213E18EEB333711118EEC373C10E18E8B
:10EBF300ED393E07138DED3B4203DD8DEE3B3E09C0
:10EC0300338DEE3B310DDE8DEE392812378DEF3823
:10EC13002319DC8DEF382A18778DF0372A12DC8D13
:10EC2300F0382214778DF0361B0EDC8DF1361B0C79
:10EC3300338CF1371F0DDB8CF136250E378CF23414
:10EC4300270CDC8CF22A270D338DF31F2A0CDC8D65
:10EC5300F3173409338DF4143A08E48EF4123A0CA2
:10EC6300338EF4103D11EA8FF50E411A778FF50CB0
:10EC73004917EA90F50A50157790F5054F13E79178
:10EC8300F5B24F107792F5AD5408E492F4AB5A0104
:10EC93003393F4AB5C05E893F4A9500A3394F3A4DB
:10ECA300450CE094F3A041093394F29A3A05E295B6
:10ECB300F29734043395F1913208DC95F19E310DCE
:10ECC3003395F08A320CDA95F0872D0B3395EF806C
:10ECD300250EDE94EF73220C3394EF6C2412DD9433
:10ECE300EF6928157794EE6B2812DF93EE69280EEF
:10ECF3007393EE64270DDF93EE5C260B3392EE578E
:10ED0300270EDB92EE5828123792EE5E2610DB9226
:10ED1300EE64240D7391EE6C2108D991ED722304F6
:10ED23003391ED782904D991EC7C320A3391EB7F4E
:10ED33003A08D891EB833D093391EA883C0CD7918B
:0DED4300E98D3B103791E9903E12D792E820
:10ED50009143137792E794420ED792E7993E073397
:10ED600093E7A03901D993E7A63B0A1194E6A83F9F
:10ED70000CD794E6AB490E1195E6AE4F07D695E653
:10ED8000004D011396E6034601D996E6033E0811AD
:10ED900097E7043D0ED997E70740151198E70C4314
:10EDA00012DA98E812460F1198E918490CDA98E936
:10EDB0001D44081198EA243D05D898EB293A03111F
:10EDC00098EB2C3707D898EC2D38093398ED2E3D69
:10EDD0000ADC98ED2E3E0A3398EE2D3F0BDB98EFC0
:10EDE0002C420C3398F02B430ED998F02B3D113761
:10EDF00098F12D3710D898F130340D7398F23433E0
:10EE00000FD698F237330F7798F339331CD597F331
:10EE10003C32167797F43E2F11D797F440280973A8
:10EE200097F4422109D797F4461F0AB396F44B2171
:10EE300008D796F45325083396F45C2505D796F445
:10EE40006723023395F4722503D695F3782B0231AC
:10EE500095F37B3102D695F27E31063395F1832FFF
:10EE600004D695F18A2F023395F0913201D596F0B0
:10EE70009638061196EF9A3F02D497EF9D450213FC
:10EE800097EE9F4704D497EEA247073398EEA64427
:10EE900008D398EEAA430B3399EEAD440CD499EE07
:10EEA000B1400D339AEE013F11D39AEE054512772A
:10EEB0009BEE064A15D59BEE064712779CEF05425E
:10EEC00012D79CEF063E0F779DEF084111D39DEFBF
:10EED000094619779EF00B4718D39EF00D431C7717
:10EEE0009FF10F4015D69FF1114113779FF2134602
:10EEF0000ED9A0F2174A0B33A0F31C4A08D4A0F491
:10EF000023420333A0F42A3305D3A0F53127071198
:10EF1000A0F5382300D29FF53D2702339FF6442900
:10EF200003D39FF64F2808119EF55E2807D19EF562
:10EF30006C2D04119EF4752F01D09EF47C2D0433AA
:10EF40009EF3822B04D09EF3872E05119EF28B3503
:10EF500007D09EF2903D01119FF1954203D09FF0A2
:10EF600094400333A0F09F3F0BD0A0F0A13D0F379A
:10EF7000A0EFA33C0DD1A1EFA43C0C33A1EFA43C26
:10EF80000AD0A1EEA53D0533A2EEA63C00D1A2EE2B
:10EF9000A8390211A3EEAA3C04D0A3EEAD3F05119F
:10EFA000A4EEB24008D0A4EE03410C11A5EE064138
:10EFB0000AD2A5EE08450711A6EF094A05D2A6EF29
:10EFC000094C0111A7EF0A4807D3A7F00B420B1118
:10EFD000A8F00B420DD4A8F00D461311A9F111466B
:10EFE00014D9A9F1173F1B11A9F21E381ADAA9F397
:10EFF00021381811A9F31F3A17DFA9F41839151190
:10F00000AAF4163A1DDCAAF5183C1A11AAF51C3A06
:10F010001AD9AAF61F391A11ABF6203615D9ABF753
:10F0200021341711ABF8203B19D9ABF81E3F17114B
:10F03000ACF91D4011D9ACF91E3F0E11ACFA1F40BE
:10F040000CD6ACFB22410D11ACFC23450FD6ADFC18
:10F0500023490B11ADFD214A0DD6ADFE2047091104
:10F06000ADFE21450CD6ADFF22430E11AE00224568
:10F070000CD8AE01214B0A11AE0220500DD7AF03C0
:10F080001D4F0B11AF031A5109D9AF04174A0D11C7
:10F09000B00418470BDBB0051A500A11B0061C5516
:10F0A0000ED7B1071C560B11B10719470ED9B1087D
:10F0B000173C0C11B208183D0CDCB2091C490E11AA
:0DF0C000B20A1E4E0AD9B30B1D500B11B33E
:10F0CD000C1A5109D9B30C174F0711B40D17490B71
:10F0DD00DBB40D17480D11B50E19490ADCB50F1922
:10F0ED004F0B11B50F185605DBB61017550711B696
:10F0FD0011174C0ADBB61116430B11B711173F0D43
:10F10D00DDB71219430C11B7131A480BDCB8131ADB
:10F11D00450F11B81419410DDCB81418400B11B975
:10F12D001518430DDBB91618470F11B91618490DEF
:10F13D00DBBA1718470A11BA1717450CDBBB1814A1
:10F14D00460F11BB18134C0EDBBC1912510A11BC22
:10F15D001A125007DBBC1A12470B11BD1A10400DC5
:10F16D00DCBD1B10400A11BE1B124509DCBE1C156F
:10F17D00490B11BE1D184A0ADBBF1D1B4A0811BFE2
:10F18D001E1B480CDBBF1F1A470E11BF1F1A490B60
:10F19D00DBC0201B4B0D11C0211C4910DBC0211DF4
:10F1AD00470F11C1221D4711DBC1231C4B0F11C18C
:10F1BD00231B4B0EDBC22419441111C224193D0F20
:10F1CD00DBC2251B3B1011C2261D3F0DDAC2261EC8
:10F1DD00411011C3271D3F12DAC3271C3D0F11C368
:10F1ED00281B3D10DBC4291C401111C4291C450FDF
:10F1FD00DCC42A1C460E11C42A1B4510DCC52B1974
:10F20D00431111C52C184511DDC62C164A1011C617
:10F21D002D174A11DEC62D18491211C72E19471088
:10F22D00DEC72F1A460E11C72F1C4410DFC7301F23
:10F23D00471111C731214B0CDBC832224D0E11C8BD
:10F24D0032224A10DAC83321471111C83420460F33
:10F25D00D9C83520461111C93521430CDBC93623D8
:10F26D003F0F11C937253D11DBC93725400E11C997
:10F27D0038254211DCC93925431311C939254312EB
:10F28D00DCC93A25431111CA3B24400DDCCA3C248C
:10F29D00411011CA3C23400EDCCA3D22401111CA57
:10F2AD003E20420FDECB3E20451011CB3F204714B0
:10F2BD00DECB4021441211CB40213F10DFCB412248
:10F2CD003C0D11CB42234011DFCC42233E1111CC1A
:10F2DD0043202F0EE0CC4319221211CC43122011E2
:10F2ED00E3CC4311250E11CD43132B10E3CD441266
:10F2FD002D1111CD440F2B0FE3CD44092B1211CE3F
:10F30D004404320FE2CE4401360E11CF44B3370D13
:10F31D00E0CF44B3330E11D04401370EE0D0440595
:10F32D003D0D11D0450A3B0CE3D14512330D11D1E2
:10F33D00451A2D0EE3D1461E2B0F11D1461D2E0F52
:10F34D00E4D1471D300F11D1471E320EE3D24821B3
:10F35D00330F11D248233510E2D24923350F11D284
:10F36D004A20360EE3D24A1D360E11D24B1B3410F5
:10F37D00E3D34B1B320F11D34B1B300EE4D34C1B7D
:10F38D00340D11D34C1B3A0DE5D44D1A3B0E11D44F
:10F39D004D1B360AE6D44E1D340E11D44E1E360DBD
:10F3AD00E5D44F1F360C11D5501F350EE5D5501F26
:10F3BD00340D11D5511E340EE5D5511E370C11D516
:10F3CD00521E390EE5D652203B0F11D653223C0F5B
:10F3DD00E4D65423391111D654243710E3D65524CD
:10F3ED00360F11D655253310E3D65626330D11D6CB
:10F3FD005627350BE2D657273A0C11D658273C0F16
:10F40D00E2D75827391011D75927370FE2D75A2786
:10F41D00381011D75A283B0FE2D75B293C1111D771
:10F42D005C2B3C12E2D75C2D391111D75D2C3910B4
:0DF43D00E3D75E2B3C0F11D75E293B0EE399
:10F44A00D75F27371011D75F26360EE3D760273CE0
:10F45A000E11D761284310E3D76229451111D762EB
:10F46A00293F0FE4D763283A1011D763293A11E4E8
:10F47A00D7642A3E1011D7652C4211E4D7662E4272
:10F48A001011D7662D3F11E4D7672F3A1011D768AC
:10F49A002D3B0CE4D7682E3D0711D7692E4204E4B0
:10F4AA00D76A2E470111D76B2E4702E4D76B2D403E
:10F4BA000513D76C2B3503E4D76C2A2B0711D76DAC
:10F4CA002B2909E5D76D2B300611D76E2A3A04E4A9
:10F4DA00D76F28400611D76F283E08E4D77027381F
:10F4EA000C11D87026320DE6D871252F0911D87162
:10F4FA0024310AE9D87221340811D8721B3A08EA71
:10F50A00D9730D420A11D973104909EADA730C4505
:10F51A000811DA730A3B06E8DB74093D0211DB7451
:10F52A000A4003E9DB740B3C0213DC75103406EA6B
:10F53A00DC7517350333DC761A3F06EADD771C469D
:10F54A000433DD771F4001E8DD7824360731DD78A2
:10F55A002C3206E7DC7933320413DC79373409E7D5
:10F56A00DC7A3A340C33DC7A3C3508E7DC7B3D370D
:10F57A000233DB7C3C3A05E7DB7C3C3D0333DB7D35
:10F58A003B3A04E7DB7D3B320331DA7D3E2D09EA63
:10F59A00DA7E43270D11DA7E4D230AE9DA7E5726F1
:10F5AA000B11D97D5E2C0BE9D97D61300C11D97D07
:10F5BA00632F08EAD87D662F0511D87C683005EAE2
:10F5CA00D87C6D330611D77B733608E9D77B7C3834
:10F5DA000511D77A853A04E8D8798B3B0711D8798F
:10F5EA008E3809E9D8788F371011D878903B0BE814
:10F5FA00D87791420D11D976954A08E7D976984974
:10F60A000411D9759D4008E8DA75A23A0B33DA7508
:10F61A00A53C0AE8DB75A8430031DB74AA4603E976
:10F62A00DC74AF460213DC74004A02EADD75054C4D
:10F63A000333DD75084D00EDDE75084B0533DF76C3
:10F64A00064902EDDF76044A0131E076044902EA0E
:10F65A00E076044C0513E176045006EAE176014DA2
:10F66A000D33E276B1450FEAE276AD3F1077E375E6
:10F67A00AB3F0DEAE375AC430A33E475AE4604EAE0
:10F68A00E475B0400131E575B23908EAE575013C27
:10F69A000611E675054607ECE6760A4B0311E7768E
:10F6AA000F4604EEE777163B0611E778203405EC9F
:10F6BA00E77827350611E7792D3409ECE7793234F2
:10F6CA000B11E77A3B260AECE67A45250B11E67A16
:10F6DA004D230BEAE67A56250711E67A5F270AEAEE
:10F6EA00E579672A0C11E579731F0AEBE578792E1B
:10F6FA000811E578843302EAE5778D3B0313E67651
:10F70A00954104EAE676993F0733E6759A3801EAA5
:10F71A00E67595310531E6748F3202EAE6748E3564
:10F72A000111E773923301EAE77398310413E77220
:0AF73A009D3304EBE872B4370911A7
:00000001FF
